:020000040800F2
:1000000000500020116D0108FF050108D505010809
:10001000FD050108FB050108F905010800000000C5
:10002000000000000000000000000000F7050108CB
:10003000F505010800000000F30501087328010818
:10004000B16D0108B16D0108B16D0108B16D010814
:10005000B16D0108B16D0108B16D0108B16D010804
:10006000B16D010881280108B16D0108B16D010869
:10007000B16D0108B16D010879F20008B16D010898
:10008000211F0108B16D0108B16D0108B16D0108B2
:10009000A5060108B16D0108B16D0108B16D010837
:1000A000B16D010875EE0008B16D010885EE00081C
:1000B00065EE000855EE000845EE00087966000878
:1000C0007D6600087366000877660008B16D010858
:1000D000B16D010871F20008B16D010869F2000804
:1000E00085280108B16D010849520108000000008F
:1000F0000000000000000000000000000000000000
:0C01000000000000000000005FF808F1A3
:100110002DE9F04F684B694EA3B033600023736044
:1001200011F0CCFA18B911F0EBFA0BF0F9FF0CF062
:100130009DF8634A634C137843F001031370624ADD
:10014000002393460A930B930C934FF4E0130D9303
:100150002368107B43F480332360A36943F01003CA
:10016000A361236803F400330B930A9B01330A93C2
:100170000B9B1BB90A9BB3F5A06FF2D123685149C1
:1001800013F4003301D0022315E00A6842F00102A3
:100190000A600A93236803F002030B930A9B01335E
:1001A0000A930B9B1BB90A9BB3F5A06FF2D123688E
:1001B0009A0739D501230C93444B45491A6842F0FC
:1001C00010021A601A6822F003021A601A6842F0DC
:1001D00002021A606368636063686360636843F483
:1001E000806363603B4B1A68043B22F070425A60A4
:1001F000394A0A60626822F47C1262605A6842F0EE
:1002000000425A60DA6822F40042DA609B681B04FC
:1002100049BF324B4FF4E0130B604FF480130D9342
:100220000C9B012B01D117E0FEE7022B18D168B11E
:100230000D9BB3F5801F02D14FF4A01305E00D9B79
:10024000B3F5E01F02D14FF400130D930D9A6368CC
:10025000134343F4803302E0636843F46013636044
:10026000236843F0807323602268164B9701FBD507
:100270005A6822F003025A605A6842F002025A6039
:100280006368104803F00C03082BF9D14268144B43
:1002900002F00C02042A03D0082A03D00E4A29E0F7
:1002A0000A6827E042684568C2F38342ED0302F121
:1002B000020219D40B491CE0D7B900081004002031
:1002C000B0240020001002406C2A002000200240D0
:1002D000440000200410014000127A00001BB70007
:1002E000A003002000093D0040680968800348BF62
:1002F00049084A431A6062684D4FC2F30312B95C61
:100300001A68DFF85CC1CA404FF6FF711A60494AAB
:100310000593CCF80820484A22ADCCF80C20A269FD
:10032000CDF810C042F00102A261626ADFF83481A8
:10033000B260626ADFF8309142F080726262A26954
:10034000404642F01C02A26125F82C1D00222946DD
:100350008DF85E20039211F0D9FE4846294611F02F
:10036000D5FE3648294611F0D1FE10218DF84210F5
:1003700002218DF843100DF1880A4FF400712AF81C
:10038000481D4046C8F81010514611F0BFFE2C48D9
:10039000416841F00071416028460AF0BEFA1799A1
:1003A0002848059BB1FBF0F12748039A01602749D3
:1003B0001B680A604A604FF47A71B3FBF1F3244979
:1003C000DDF810C0013B4B60F0238CF8233007238D
:1003D0008A600B60DBF808101E4A1F4B116007F1A2
:1003E000100103C985E80300A169049341F00801E5
:1003F0000392A1610821C9F81010179818A911F0EB
:1004000085FE039A049B1168CDF80C8011F0080F4B
:10041000904631D093F89021012A2DD893F891215C
:100420000E4B9B6813F0805300F00D8624E000BF54
:10043000B8AA0108000000080005FA0500100140F4
:100440000000014040420F003C2700200827002008
:1004500010E000E0283500206C2A00201004002065
:1004600000ED00E000080140000C0140AB4B002211
:1004700083F891210CF0CCF8642012F0F0F9A0225E
:10048000A74800211AF082FAA64A536823F4406371
:1004900043F0706343F400635360E369002243F068
:1004A0000703E361A36943F4006343F00C03A36112
:1004B0009D4B4FF0000903F10C0102F8019001324D
:1004C0000C2AF5D1FF221A765A769A76DA76974B6D
:1004D000974AD8F800401A609648494630221AF0E8
:1004E00055FAC4F380180423934A924919F802007C
:1004F0000C2202FB09F25054B8F1000F06D11E285D
:1005000001BFFF2003F1FF335054DBB209F10109B1
:10051000B9F1040FE8D1894A9BF805901370884B14
:10052000884983F80090884B7F4AF361C0330B60A1
:10053000864BA10603EBC9035B7848BF0123136216
:10054000002340F2DC51824A22F813100133082BB9
:10055000F7D1504600211C221AF018FAB9F10E0FFB
:1005600003D009F0EF03082B02D101238DF852309C
:10057000C4F340038DF84630C4F340338DF8403067
:10058000C4F3C0338DF8433014F400638DF8498010
:1005900004D09BF88431581E434243418DF84430C7
:1005A000C4F300438DF84A30336ABBF8441100337A
:1005B00018BF01238DF84B30C4F300538DF84C3035
:1005C000BBF84631ADF85610ADF85030BBF852319B
:1005D00004F00109ADF84E30C4F380438DF8473084
:1005E0009BF85431C4F3C0081A1C18BF0122E1045F
:1005F00048BF4A498DF8482048BFB1F84C11BBF8B4
:10060000502148BFADF85610B2F5FA7F8DF84190F1
:100610008DF84280ADF8542002D90BB9ADF85630B0
:100620009BF855419BF8D631003418BF0124494846
:100630000021642286F824308DF84D401AF0A6F986
:100640009DF85230002B0CBF00230223B9F1000F9C
:1006500002D1B8F1000F00D001339B003B440CB134
:100660009B6900E09B6AA3F1020B163304934FF0E1
:10067000000A4FF6FF733BF8022F9A4200F0028205
:100680009DF84500D3B2120AD1B218B1981E0128C4
:1006900040F2F4819DF8490030B12F4C18012458E4
:1006A0002E48844200F0EA819DF84A0030B12A4C7D
:1006B000180124582948844200F0E0819DF8460042
:1006C00050B1254C039F04EB03146068B84203D17A
:1006D0002089012800F0D2819DF8430050B11E4CC2
:1006E000039F04EB03146068B84203D120890228F9
:1006F00000F0C4819DF8440050B1174C184F04EB32
:1007000003146068B84203D12089022800F0B68142
:10071000022A27D19DF8402028E000BF6C2A002043
:100720008427002000000140100400205C320020DB
:10073000602C00206432002054E70108BE14002021
:10074000000C0020A02800207C2A0020C8B001084E
:10075000FC1300204C130020ACCD01080004004025
:10076000000C0140012A04D19DF84120002A00F02C
:1007700085819DF84B209D481F015AB19DF852205C
:1007800042B9A3F10802012A04D8C259984CA242E6
:1007900008BF04219DF84C2032B19DF852201AB9AF
:1007A000043B032B98BF04219DF84030C419A3B12A
:1007B000CB1EDBB2012B08D8C359B3F1804F00F038
:1007C0005D818C4A934262D158E1022940F02E812A
:1007D000C259894B9A425CD150E1012957D19DF809
:1007E0004730DFF8248223B9BDF85430B3F5FA7FDF
:1007F00006D9814BC2599A4204BF032388F8253099
:100800007A4AFF23D11991F80DE088F86C3088F806
:100810006D30486801F1080309894FF00009ADF80F
:100820005C1002218DF85F1088F870902946C8F896
:100830007C408DF85EE00692059388F82890C8F811
:100840002C90C8F83090C8F83490C8F8689088F8B0
:100850006E9088F86F9011F059FC059B069A997874
:10086000D0594A460CF02BFD2046494601220EF095
:1008700057FC624B6249C8F88030624BC8F88890D8
:10088000C8F8843020460A1D0EF092FCF6E00229DA
:100890004CD15FFA8AF31C2101FB03FC5A4B4FF049
:1008A000000803EB0C09012389F8703006934F4BC5
:1008B00089F871A0D91991F80DE001F10802486892
:1008C000098989F87280ADF85C1002218DF85F10FB
:1008D00089F87A802946C9F87C40CDF81CC08DF88B
:1008E0005EE0059211F012FC404B059AD8599178C0
:1008F00042460CF0E4FC069B20461A4641460EF0A8
:100900000FFC424A404BDDF81CC0C9F8802003EBC5
:100910000C013F4A8031C9F88420C9F888802046FC
:100920000A1D0EF045FC0AF1010AA7E0032940F078
:1009300080809DF84730374F03B39DF84830DFF88B
:10094000E08097F8019053B1334BBDF85420204616
:10095000B3FBF2F2082192B2BDF8563003E0204614
:100960004FF6FF7208210CF0FFFC2C4B48F82900D1
:10097000C360BB78192207EBC3032DE0BDF85420F8
:1009800097F80180B2F5FA7F13D9234B2046B3FBC9
:10099000F2F2082192B2BDF856300CF0E5FC204B83
:1009A0000D2243F828001F4BC360BB7807EBC3033D
:1009B00012E01D4B2046B3FBF2F2012192B2BDF8CA
:1009C00056300CF0D1FC164B092243F82800134B8B
:1009D000C360BB7807EBC3035A71BB787A7807EB27
:1009E000C3010A7101328C607A7045E0ACCD010818
:1009F000002C0140000400400008004031CD0008F8
:100A0000900400201DCE000810040020F9D2000838
:100A100009CD00084C13002000127A002DCE0008EA
:100A2000502700203DCE000840420F0001293FF42E
:100A3000D6AE042922D1664FBDF84E20BB7897F878
:100A4000008007EBC30383F80480624B012193FB12
:100A5000F2F2204692B2BDF850300CF085FC5E4BAD
:100A60000A2103EB8803C3F85001BB7807EBC302EC
:100A700051713A7801323A700133BB70049B9B4547
:100A80007FF4F7AD524A554B1278002786F8702153
:100A9000534A1F7092F800804F4CA8F11702022AA7
:100AA00099461AD8E3690021D85903EB070A15F0D3
:100AB00081FD10B1336A6BBB27E04A4B07EB030E95
:100AC0009AE80F008EE80F0099F8003010370133D4
:100AD000C02F89F80030E5D1ECE7434B13F838C05C
:100AE00003EBC803D3F804A089F800C0BAF1000FE3
:100AF000E0D06745DEDA3B4A3B0103EB020E53448C
:100B00000FCB01378EE80F00F3E7384F3B68DE0468
:100B100024D41DE0364B374A13F8380003EBC803E2
:100B20005E681070002EF0D000238342EDDAC3EB34
:100B3000C3017218D2F800C0DFF8C4E0013341F8F5
:100B40000EC001EB0E079188B9809279BA71ECE77B
:100B500008F0EF03082B284B25D127E099F8003047
:100B6000012BF5D9254E06EB031303F110091036BE
:100B70004E45EDD056F8100C4FF07C5115F086FB29
:100B80004FF07C5146F8100C56F8140C15F07EFB13
:100B90004FF07C5146F8140C56F80C0C15F076FB0F
:100BA00046F80C0CE3E7B8F10E0F09D11A78B8F14A
:100BB000180F42F010021A7024D112F0E5F821E06B
:100BC0001A78B8F1190F22F010021A70F4E700BF7A
:100BD0004C13002040420F0010040020802700200A
:100BE000000C0020340B0020C8B00108283500207C
:100BF00030B901082C280020481400203C0B0020AC
:100C00002D28002012F0A4F83B68C44E58035EBFA4
:100C1000C34B01221A70C34A4FF0020A13782946C7
:100C200043F004031370C04B8DF85FA093F8552177
:100C30009846012ABD4A14BF4FF400430423138091
:100C4000ADF85C3014238DF85E30B369B84843F0DA
:100C50000403B36111F05AFAB64AB74B00201A6088
:100C600011F012FEB54B4FF0030993E80300B3698E
:100C700085E8030043F00803B361179818A911F041
:100C800045FAB369182243F48053B361F368A84866
:100C900043F48053F3602946A0238DF85E2005922B
:100CA0004FF0040BADF85C308DF85F9011F02EFA28
:100CB00040239F482946ADF85C308DF85EB011F0B6
:100CC00025FA10239A482946ADF85C308DF85E303D
:100CD000049311F01BFAF1684FF0070C41F48051B6
:100CE000F160F168059A21F48051F1609449088817
:100CF00000F4415040F4457040EA09000880888BB8
:100D000020F400600004000C8883A1F810C008885B
:100D1000CDF80CC080B240F040000880F16941F489
:100D20008041F161316941F4804131618DF85F901A
:100D3000DFF814928DF85E2048464FF42042294691
:100D4000ADF85C2011F0E2F94FF4804248462946A4
:100D5000ADF85C208DF85EB011F0D8F9049B4FF42B
:100D6000805B484629468DF85E30ADF85CB011F0E6
:100D7000CDF93369DDF80CC043F480433361336946
:100D8000504623F4804333616E4B1A8802F441527B
:100D900042F4457242F003021A809A8B22F40062F8
:100DA0001204120C9A83A3F810C01A8892B242F06F
:100DB00040021A80C9F810B009F0EEF8002801F0DE
:100DC00075824388002B01F071823F68DFF89091B3
:100DD00007F40063484600211022039319F0D6FD62
:100DE0004FF6FF73ADF83C30022307F4004B4FF091
:100DF000000A1F408DF83E308DF83FA00FD001272C
:100E000022A921F84C7D4A4809F014FC072389F8EF
:100E100000A089F801A089F8027089F80330BBF1BD
:100E2000000F12D0022322A921F84C3D404809F0BE
:100E300001FC0123FA1889F8043089F806300723E9
:100E400089F8057089F80730D7B2039B9BB102235C
:100E500022A921F84C3D3C4809F0ECFB0923012272
:100E600089F80C3089F80E207B1C072289F80D7058
:100E700089F80F20DFB27368344843F4404373604D
:100E80007369DFF8C8A043F001037361B36943F4E9
:100E90000073B36109F0B5FD284609F087FD2C4BBE
:100EA000012F17932B4B4FF00006189394BF334636
:100EB00080231C934FF480731D934FF480631E9323
:100EC000202329461F9350464FF400531A9720932E
:100ED00019961B96219609F076FDDAF800301E4A25
:100EE00043F00103CAF800305368012F23F4702344
:100EF00094BF0021012123F4807343EA012353604E
:100F00009168164B013F0B4043F4602343F002030A
:100F10009360D36AFFB223F4700323E00010024011
:100F200068100020B02400206C2A00201027002028
:100F300000080140DD2501089C350020F0AA0108C9
:100F40000030014000380040000C01400800024021
:100F50004C2401405817002000240140FDF7F1FF08
:100F60004817002043EA0757D762012309EB06021E
:100F70009178002952D019F80600591C0928C9B2E5
:100F8000D278C84F10D9A0F10A05D7F80CC005EBEC
:100F900045054FF0070E0EFA05FE2CEA0E0EAA408C
:100FA0004EEA0202FA600CE03D6900EB400C4FF0A3
:100FB000070E0EFA0CFE25EA0E0502FA0CF22A4381
:100FC0003A61062BB74D0CD8013B6F6B03EB8303E3
:100FD0001F229A4027EA020200FA03F313436B63CD
:100FE0001BE00C2B0CD8DA1F2F6B02EB82021F23A5
:100FF000934027EA030700FA02F33B432B630CE01C
:10100000A3F10D02EF6A02EB82021F23934027EA4D
:10101000030700FA02F33B43EB620B460436102E43
:10102000A4D1A04B9A6842F480729A609A6842F008
:1010300001029A609A6842F008029A609968994A97
:10104000090733D5FAE7013A092A3FF615AAF86DE0
:10105000294628604846049311F058F84FF400627E
:10106000C9F810203C2011F0FAFB049B9BF8912159
:101070009342BFF6FBA9DFF8589208214FF40062B3
:1010800006937820C9F810100591C9F8142004922D
:1010900011F0DAFB0599049AC9F814107820C9F800
:1010A000102011F0D1FB069B0133DFE7936843F07A
:1010B000040393607B4B9A6812F004020392F9D107
:1010C0009A68B8F85A0142F4A0029A60764B002858
:1010D00041F0F180B3F95C21002A41F0EC80B3F9D2
:1010E0005E31002B41F0E780DFF8E8816E4DD8F8E3
:1010F00000300021B3F856300C226C480493DFF81E
:10110000CCB195F8619195F8697195F86A6195F897
:1011100063A119F03BFC00211422654819F036FC4C
:10112000002384F8713119468BF872310C220BF5CB
:10113000BA70059319F02AFC5E4A2320C4F8802176
:1011400011F08DFB752001210DF1270205F020FA29
:10115000B8B1594A059BCBF87821584A1846CBF8C4
:101160007C2143228BF8742101210EAA05F010FA8C
:101170009DF8383003F07E038DF83830002847D1D1
:101180004FE04F4A6B201388802123F040031B045B
:101190001B0C138013884FF0060B23F038031B043D
:1011A0001B0C43F03003138013889BB243F04003C1
:1011B000138005F0C9FA962011F051FB752001212A
:1011C00017AA05F0A6FA9DF85C30682B05D00BF144
:1011D000FF3B1BF0FF0BEED183E00C20012117AA8F
:1011E00005F097FA9DF85C30142B7AD3182B02D9AE
:1011F000543B062B75D8032384F87131432384F8BC
:101200007431304BC4F878312F4BC4F87C3168E02E
:10121000682B06D101238BF871311D238BF87431B3
:101220005FE09DF8273003F07E03682B8DF82730B0
:1012300052D10223062084F871310146D4F8783166
:1012400017AA98479DF8611001F001029DF85F1000
:1012500001F001014B0043EA82019DF85D2002F09C
:1012600001030B430AD05BB2012B01D1002302E042
:10127000022B0FD1012384F8723132E0134B0C2082
:10128000D3F8783101210FAA98479DF83C3013F02C
:101290000F0303D1032011F063FB22E0042BE9D1FB
:1012A000E4E700BF002401406C2A0020342900201C
:1012B00008340020F8AA0108916500086966000852
:1012C000003001401367000849670008100400203F
:1012D000000C01400C140020702B04BF042384F880
:1012E0007131CA4A0023137094F87131032B13D162
:1012F000C74BC849C8481960C8495960C849D9602E
:10130000C849196104231370C74A06231168037082
:1013100041F00103136003E0012011F021FB47E2DB
:101320004B4640F2023C0A2B28BF00234FF0010E2F
:101330000EFA03FE0EEA0C0CBCF1000F16D11EF0E3
:10134000FD0F13D0B94BDFF81CE341F00301C3F8E4
:1013500000E0DFF814E31160C3F804E0B44B4FF091
:10136000040E83F800E00723437006E0012B4FF0E2
:101370000009D5D8AE4B83F80090042E00F2768198
:10138000DFE816F005007D016E0005000D010A2062
:1013900011F065FA7720A02101220FAB05F038F893
:1013A00000285DD01E210122772005F0FBF84FF4C4
:1013B0002F6011F049FA4FF00009A9F160010026F1
:1013C000C9B2022217AB77208DF85C608DF85D60A2
:1013D00005F01EF89DF85D309DF85C2043EA02227E
:1013E000944B03F5C27129F8012009F10209B9F102
:1013F000100FE2D1B3F892114FF0010E01F00F007F
:1014000001F47F41A3F89211334626F001022244F1
:10141000B2F88421002A18BF4FF0000E16F0010F19
:1014200003D0D2B25340082202E083EA1223FAE743
:1014300013F4004F18BF83F4C053013A4FEA43033B
:10144000F6D10136102EE0D17A4A0143A2F892116A
:10145000BEF1000F04D1C3F30333984200F00787B5
:1014600094F89431734E002B40F0AA87142011F0A9
:10147000F6F97720D02101220FAB04F0C9FF002834
:1014800000F08D809DF83C300322552B86F8AF315B
:10149000A6F8B82140F08380D12101220FAB77203C
:1014A00004F0B6FF9DF83C30772003F00F021B09D3
:1014B00086F8B02186F8B131162217ABAA2104F0C4
:1014C000A7FF9DF85C209DF85D3043EA0223A6F853
:1014D00098319DF85E209DF85F3043EA0223A6F81C
:1014E0009A319DF860209DF8613043EA0223A6F806
:1014F0009C319DF862209DF8633043EA0223A6F8F0
:101500009E319DF864209DF8653043EA0223A6F8D9
:10151000A0319DF866209DF8673043EA0223A6F8C3
:10152000A2319DF868209DF8693043EA0223A6F8AD
:10153000A4319DF86A209DF86B3043EA0223A6F897
:10154000A6319DF86C209DF86D3043EA0223A6F881
:10155000A8319DF86E209DF86F3043EA0223A6F86B
:10156000AA319DF870209DF8713043EA022341F2C0
:101570007072A6F8AC31304B1A8046F678125A8059
:101580002E4A5A602E4A9A602E4ADA602E4A1A6112
:101590002E4A5A61012386F8943100F011BF94F865
:1015A000BC91244EB9F1000F40F07386142011F065
:1015B00056F906F2BD137620D021012204F028FF4F
:1015C00096F8BD31582B5AD106F5E07388211822C0
:1015D000762004F01DFF31227620F42104F0E2FF92
:1015E00001231B4A86F8BC31134B9A60194AA3F8B1
:1015F00000905A6045F6D8125A80174ADA60174AA6
:101600001A61174A5A6100F044BE00BF6809002001
:1016100008340020756700089B03002089610008DA
:101620006961000890C1793DC01300203429002071
:10163000C135002010040020DC2400206166000871
:101640006965000849660008296500088D60000882
:10165000896000088B60000841660008DD640008AE
:10166000C95E0008B9630008D1610008012E06D0E8
:101670003F4B404A9E70136843F0040313603D4E95
:1016800033689B0702D53C4B1B689847BAF1000FA3
:1016900007D133687D2113F00E0F0CBF04220822FE
:1016A00002E001224FF47A71013AD3B203FB011137
:1016B00084F8DC31314B50461960314B1B68984738
:1016C000304A00231370914617B1022F40F0E48591
:1016D0002D4A002422ABC2F8E04103F82C4D1E2015
:1016E0000A21012204F094FE88B19DF85C30482B59
:1016F00040F06986254B264A1A60264A5A601C4BE0
:101700000222DA70336843F00803336002E00446D3
:1017100000F059BE95F856310BB11F4A137095F879
:1017200057310BB11D4A137095F858310BB189F838
:10173000003033681A4E13F0080F37D0BDF91090FF
:10174000642799FBF7F4204614F04CFD824607FB12
:10175000149000B214F046FD124914F097FD0146B2
:10176000504614F08BFC104914F090FD30601FE0DF
:101770009B030020C01300203429002020350020C6
:1017800008340020BD350020100400202826002049
:1017900071210108A91E010868090020C135002037
:1017A000B80A00208988883C00002041002333606B
:1017B000A84A0A24137843F002031370A64B0822A8
:1017C0001A61A54E1920F368013C83F00803F36009
:1017D00011F045F8012011F057F8192011F03FF8E9
:1017E000002011F051F814F0FF04EAD1082333610E
:1017F0009A4B1A681E4612F0080F05D0984B1B68CA
:101800009847984B01221A70974B984C1B68187B8D
:1018100014F0E8FC964914F039FD0AF025FC954BCC
:1018200093491860944B186914F030FD934B18607D
:10183000934B188814F0D6FC0146924814F0DAFD58
:10184000914914F0D7FD914B186011F0DFFA204652
:10185000FF211C2219F09AF8204636688C4B012291
:1018600016F0020F18BF62701A701FBF03221A70A1
:101870000222A27000211A78770721704FF01B0412
:10188000845402F1010144BF814C0232C9B2197083
:1018900041BF2270754A0324545416F00A0F0CD02D
:1018A0001A7804218154511CC9B205244454D11C16
:1018B00002321970D2B206218154764C21688E060C
:1018C00041BF1A78561C1E70072648BF86540A0668
:1018D00008D51A7809268654961C01321E70D2B299
:1018E0000A2686546E79082E01D00E2E04D11A785D
:1018F000571C1F700B2787541A7811F4803F4FF044
:101900000C0E00F802E002F101071CBFDFF880E1D5
:101910000232FFB21F701FBF8EF80020534A4FF0F3
:101920000E0E02F807E04A0748BF1A784FF0120E71
:1019300041BF571C1F70102787541A7811F4806F0D
:1019400002F10107FFB21F7000F802E00ED095F817
:1019500018E2BEF1000F09D0DFF834E102328EF850
:101960000020424A4FF0130E02F807E08F0541BFF6
:101970001A78571C1F70152748BF8754182E0DD191
:101980001A7816278754571CFFB24FF0170E00F82D
:1019900007E0D71C0232D2B21F7086540E0341BF3B
:1019A0001A78561C1E70192648BF8654CA0541BFB6
:1019B0001A78511C19701A2348BF835400219822A9
:1019C000354818F0E3FF12F02AFD3449344B35480E
:1019D0001960B5F84E21344B016034491A80002358
:1019E000334AD8F800900B70B5F8961113809370B5
:1019F0001FFA81FC09F179022E4E2F483768DFF873
:101A0000BCE007F5967720F813C04EF82370013339
:101A1000122BF1D1D4F800E009F1C9071EF4805F60
:101A200008BFB5F89EC1A0F806C01378002B55D1A9
:101A300092F802C0D3789C4550D2BCF1000F3FD041
:101A40000CF1FF3C0CEB8C0C0CEB8C0C0CF561736B
:101A50003DE000BFB0240020000C0140C013002076
:101A60002826002040260020340A0020CD13002024
:101A700035FA8E3CBC0A002008340020A80A002059
:101A8000080000200AE81C4100401C4604260020F3
:101A9000CC13002028350020D4290020F42B00206E
:101AA00088110020243500208C11002054110020C2
:101AB0003435002058290020943200200C110020D9
:101AC000013303EB830303EB830303F5617392F8A4
:101AD00001C09BB20CF1040C20F81C300432BA4255
:101AE000A3D11EF0080F00F0D78095F89031072B96
:101AF00000F2CC80DFE803F004070E354F6F6FACC7
:101B000045F2F05201E042F6F8228A4B1A8012F0B8
:101B100024FDBAE042F6F822864B09011A800A2316
:101B200091FBF3F10023A1F5B061834A42F8231041
:101B30000133122BF9D1814A814940201160814A39
:101B4000137010F071FD002800F0A08001234FF009
:101B5000070990F9000040218DE808027A4A7B4B82
:101B60008EE042F6F822734B40201A80784A734B7D
:101B70001A60744B10221A7010F056FD002800F005
:101B8000858001234FF0000C90F9000040218DE882
:101B90000810704A72E042F6F822664B40201A8024
:101BA0006D4A664B1A60674B08221A7010F03CFDB4
:101BB00000286BD001234FF0000E90F90000402167
:101BC0008DE80840654A4FF4E13308F0FDF8644BB6
:101BD000C3F8E40156E042F6F821564A062B11807C
:101BE00058494FF00C025F4F5F4D6048DFF8ACC1C1
:101BF000DFF8ACE10A700ED000232B703B7003704D
:101C00001B238CF800305A4B8EF8002005221A70E6
:101C10004FF4E1350BE000218EF80020544A297082
:101C200039700170534D21218CF800101370524A05
:101C3000424B40201A6010F0F7FC38B30123002714
:101C400090F9000040218DE888004C4A2B4617E0AF
:101C500044F62062374B40201A80494A374B1A60BD
:101C6000384B08221A7010F0DFFC78B101230025F0
:101C700090F900008DE82800424A40214FF4E133FA
:101C800008F0A2F8003018BF012028B908200AF097
:101C900015FA3D4A294B1A6023682A4A13F4804FEB
:101CA0001FBF122111703948244918BF086042F241
:101CB0000101194099B144F620601E49088098043A
:101CC00041BF0821117032481C4948BF0860D9073C
:101CD00041BF0C2111702F48184948BF0860117886
:101CE000043951701A0640F194801D48DFF8B49011
:101CF0000027294DC0F8E8913946152200F5F67005
:101D0000DFF8A4A06F706F60AF6018F03FFEA9F11C
:101D100005033846CAF800300CF08AFD336802200B
:101D2000EB6010F081FC002840D180200AF0C6F959
:101D300067E000BFDE0A00204C340020440300208E
:101D4000595201085432002065530108A086010051
:101D50002DA30008B952010815A30008BDA400086E
:101D60001004002036160020D9160020D8160020B6
:101D7000DB16002090D0030029A200088DA30008E4
:101D800019A2000841A30008B552010885520108B4
:101D9000A55201089552010844260020DA160020B9
:101DA00035160020602C00206426002046796B78D0
:101DB000CE490C2202FB03125278B24204D0013306
:101DC000DBB2042BF4D900236B70DAF800306A78A8
:101DD0001B7890F90000002B4FF00C0303FB02135B
:101DE00014BF0326012600225B780096019202218F
:101DF00007F0EAFFBE4B1860002896D001200CF0D7
:101E000017FDD8F80000BB4B00F5C5721A600CF046
:101E100031FEB94BB94ABA4D1360BA4A80331360E8
:101E20002368002613F4803F2E7017AF00F0C280A5
:101E300040F22A3A0BF01CFEDFF810C3DFF810B3B3
:101E40004FF00108604652463146CDF810C085F883
:101E5000008018F09BFDDBF818304FF0100943F0BC
:101E60000803CBF8183018238DF83B30A64803231D
:101E70000EA98DF83A30ADF8389008F0DBFBDBF8AE
:101E80001C30A24943F00203CBF81C30A04BA14DFB
:101E90001B68ABF6947BB3FBF1F32988013B21F47B
:101EA0005C7101FA09F121FA09F129809BB21D2127
:101EB000A9852B85A5F814802B8C23F0010303FA48
:101EC00009F323FA09F32B842B8CA888298B23F0A0
:101ED000020321F0730101FA09F103FA09F321FA6F
:101EE00009F123FA09F341F0600180B243EA0803E3
:101EF000A8802983AE862B842B8B23F0080303FA5A
:101F000009F323FA09F343F008032B83B5F84430AF
:101F10006FEA43436FEA53439BB2A5F84430DBF8C2
:101F2000A83F43EA0803CBF8A83F584608F069FDEC
:101F3000384608F03BFD784BDDF810C0179380233E
:101F40001C934FF480731D9358464FF40053394649
:101F50002093CDF860C0CDF86490CDF868A01B96B2
:101F60001E961F96219608F02EFDAB890FA89BB2F6
:101F700043F40073AB81DBF8003043F00203CBF88D
:101F800000308DF83C908DF83D808DF83E608DF8E6
:101F90003F8012F04DF9614B03991A68604B43F88A
:101FA00021200B460133202B0393F4D10FF0D0FFF7
:101FB0000FF0CEFF23685B0556D55A4D5A4BD5F826
:101FC0002C850420C3F8008010F02EFB0421C5F8F6
:101FD000300508F097F8554B85F834050820C3F80C
:101FE000008010F021FB524B0821186008F08AF89D
:101FF000504E85F83505002130462C2218F0C6FCDD
:102000008E2373704FF07C0AE0234FF07D09F3704C
:1020100086F800A086F82B90474E2C2200213046EF
:1020200018F0B4FC8A2373701020A023F37086F894
:1020300000A086F82B90C5F8388510F0F5FA10212D
:10204000C5F83C0508F05EF885F840052020C5F885
:10205000448510F0E9FA2021C5F8480508F052F847
:1020600085F84C050BF094FB344E00253388322064
:1020700023F040031B041B0C338033884FF480583B
:1020800023F038031B041B0C338033889BB243F0CE
:10209000400333809F238DF83C308DF83D508DF800
:1020A0003E508DF83F5010F0DAFB8DF85D50164D24
:1020B0000FAA0423C5F814803046394604F0DFFA2D
:1020C000C5F810809DF85E209DF85D30120242EA4E
:1020D00003429DF85F301A43194B9A42194B4DD079
:1020E0003ED819498A4242D034E000BF04BB0108FF
:1020F000D0220020EC110020942C00208415002018
:102100001818002008230020000C014000366E0142
:10211000A0030020000400403404004010AB01087C
:102120001A18002010040020D814002014150020D4
:102130005C150020E4140020181500200038004031
:1021400018BA20000C0000201520200011060020E5
:102150000010024001F51A4102318A4209D01CE008
:102160009D498A4205D001318A4207D015E02022DC
:1021700000E080221A804FF4807202E04FF48072F7
:102180001A805A809A88198812029A604A43DA6043
:10219000924A012182F84D1504E000221A805A80EB
:1021A0009A60DA60DE6816B3F60AB0464FF00009AE
:1021B000B14509DA09EB06056D10E802394610222F
:1021C00010F0D2F80F2807DC0CF0C2FD834A4FEA6A
:1021D000C823C2F850350AE0002357F82320013203
:1021E00060D10133042BF8D12E46A846E0E72068E1
:1021F0007B4B10F4002218BF01221A70794B5A79D8
:102200001946052A02BF784B4FF4C8721A80774BE3
:102210004FF47A721A80764BC8221A80754A137866
:1022200043F008031370744A137823F00203137009
:1022300040F6020303406BB1704A714B1A60714B58
:1022400003221A70704B01221A70704A0023138007
:102250006F4A13808B68012223606E4B1A706E4A9E
:10226000137863F07F03137023B0BDE8F08F42F260
:1022700010726A4B03261A805A80694A5A60694A6A
:102280009A60694ADA60694A1A61694A5A61FFF7D5
:10229000EFB90426FFF7ECB9012F7FF63BAA1F46E2
:1022A000FFF70EBA05F1010945469EE7012010F03F
:1022B00085F8FEF78ABD5F4B00221A7000B213F05A
:1022C00091FF5D4913F0E2FF464D0746B5F95C0109
:1022D00013F088FF584913F0D9FF0646B5F95E019F
:1022E00013F080FF544913F0D1FF0546384609F03A
:1022F000BBFE8146384609F046FE0746304609F0E7
:10230000B3FE8046304609F03EFE0646284609F0F8
:10231000ABFE8346284609F036FE494682465846BB
:1023200013F0B4FF49460490504613F0AFFF5946EE
:102330000590384613F0AAFF51460690384613F030
:10234000A5FF41460790584613F0A0FF3B4D51466C
:10235000286008F1004013F099FF31466860AE60D4
:10236000069813F093FF0146059813F087FE314657
:10237000E860079813F08AFF0146049813F07CFE8A
:102380004146286107F1004013F080FF3146686143
:10239000049813F07BFF0146079813F06DFE314659
:1023A000A861059813F072FF0146069813F066FEC7
:1023B0004946E861404613F069FF2862FEF794BE83
:1023C0000226FFF755B9012F7FF6A4A9002789F847
:1023D0000040FFF77DB900BF1740EF001004002058
:1023E000691000206C2A0020A0110020B0350020C8
:1023F000B235002048140020B8350020E62B00201C
:1024000044170020322900209F030020E4280020E8
:10241000E628002068100020B0240020DC240020E2
:1024200039660008CD64000831660008BD64000804
:102430000D5D00084800002035FA8E3C2017002072
:102440002DE9F04FAB4D99B02B780C2B9FBFAA4ACA
:10245000342101FB03239E6A88BF0026A74C11A8E4
:10246000E36898479DF84430A54F23B12B780C2B97
:102470000CD900230FE010F0CBF9A24B1B68F31A24
:1024800018443B6864339842E8D3EFE79A4A342112
:1024900001FB03239B6A9C4A3868138013F09EFE5D
:1024A0009A4913F0F3FE9A4B9A4D18606368994865
:1024B000984730B9984C2368980700F1DE8000F007
:1024C000DFBD964F284629463A7808F039FB97F841
:1024D0000180B8F1000F30D0BB78B3B9884A1268D8
:1024E0005AB37B607C688D4E022C0BDC06F108032E
:1024F000242101FB043140460022013409F0A5FAF1
:102500007460EFE70123B37017E000237B607C6801
:10251000824E022C11DC35F9140013F063FE06F133
:102520000803242101FB043109F05CFA15F046F898
:1025300025F8140001347460E9E7794EDFF8F4817E
:102540003388002B72D07B6FA8F13C041B78A8F174
:10255000480704934FF00009338835F91900B3F5A3
:102560007A7F069302BF00233B6023613B684FEAFA
:10257000490A03443B6013F035FE23690133012B04
:10258000236104D1002360602060A3602AE0D4F8B6
:1025900000C00A936146CDF820C0099013F06CFD8D
:1025A0000A9B8346184613F01DFE0146584613F059
:1025B00021FFDDF820C00146604613F05FFD0346B1
:1025C000099A194660601046089313F055FD0146BC
:1025D000584613F05BFEA16813F050FD089BE060C5
:1025E0002360A060002325F80A3028F80A30069BF3
:1025F000012B26D12069012807DD013813F0F2FDF7
:102600000146E06813F0F6FE00E0002015F02CFA19
:10261000049B834663B1184613F0E4FD0146584617
:1026200013F0F0FF20B14FF47A733380002319E0E8
:102630003B684FF47A7203F5FA7393FBF2F328F8D0
:102640000A3009F10109B9F1030F07F1040704F198
:10265000140481D13088012801D110F031F9338878
:10266000013BE2E735F8132038F81310521A25F829
:1026700013200133032BF5D11CE72A4B1B78002BC9
:1026800000F0FE8410F0C4F8244E0027D6F8C830BD
:10269000C6F8C800C31A0A93D6F8CC301F4A06936E
:1026A0001B78002B48D092F8D03002F1D4087BB1CF
:1026B0001D4B33F9170013F095FD242101FB078111
:1026C00009F090F914F07AFF184B23F8170039E05D
:1026D0001F46069B08EB07011878154A243709F0B6
:1026E000B4F96C2FF5D10D4B012283F8D0200327CC
:1026F00028E000BF9A030020640000200834002076
:1027000020350020DC250020BC130020BD37863595
:102710001C340020F0130020C013002068090020A2
:10272000B03500209035002060350020EA130020ED
:1027300000007A44280A0020664B33F81720664BC5
:1027400023F817200137022FA6DD6349B1F802A054
:10275000B1F800900FFA8AF252430FFA89F303FBA3
:1027600003228B8864210B93BDF92C3003FB0323D8
:1027700001FB03F2594B1B885B4392FBF3F3226886
:10278000523B11070D9309D5554BB3F9001029B1F0
:10279000B3F9021011B1B3F904307BBB514B197876
:1027A00001F0100000F0FF0360B312F0200329D005
:1027B00001F0020202F0FF0322B34B4B1B78042B03
:1027C0001FD94A4B1B88B3F5967F1AD3484BB3F9F0
:1027D000040013F007FD474B0446188813F002FD70
:1027E000454913F007FE0146204613F045FC4349D6
:1027F00013F04CFD00240746012305E000230124CB
:1028000001E000231C4600270A980F9313F0E6FC12
:102810003B4913F03BFDD6F840610490B5F9000048
:1028200013F0E0FC314613F031FD0890B5F90200D9
:1028300013F0D8FC314613F029FD0990B5F90400D6
:1028400013F0D0FC314613F021FD2549834608984A
:102850000B884D88B1F8048001460C9313F016FDE7
:1028600006460998014613F011FD0146304613F063
:1028700005FC59460646584613F008FD0146304609
:1028800013F0FCFB15F0F0F80F9B0E90002B3FD0DF
:1028900038461C4913F0B6FE28B138461A4913F0E1
:1028A000EBFB0746F4E73846184913F08DFE28B1D4
:1028B0003846154913F0E2FB0746F4E74FF07C5128
:1028C000384613F0E3FC09F05EFB002113F0D6FB61
:1028D00006461EE060350020EA13002008000020B4
:1028E000F61300204814002049140020561400203C
:1028F00028140020581400200000204135FA8E3C96
:10290000BD378635DB0F4940DB0FC940DB0F49C0BF
:102910000026002C00F0A380BDF9300013F062FC0B
:10292000074628B213F05EFC05460FFA88F013F054
:1029300059FC39460446384613F0A8FC294680461F
:10294000284613F0A3FC0146404613F097FB2146AE
:102950008046204613F09AFC0146404613F08EFB59
:10296000A349804613F04EFE002878D0404615F06B
:102970007BF801464FF07E5013F03CFD8046384610
:10298000414613F083FC41460746284613F07EFC7F
:1029900041460546204613F079FC964C8046216856
:1029A000384613F073FC61680C90284613F06EFCF7
:1029B0000C9B0146184613F061FBA1680C90404641
:1029C00013F064FC0C9B0146184613F057FBE168BA
:1029D0000C90384613F05AFC21690746284613F03C
:1029E00055FC0146384613F049FB616905464046EF
:1029F00013F04CFC0146284613F040FB0C9B0546A7
:102A00001946184613F042FC29460746284613F09B
:102A10003DFC0146384613F031FB15F025F8014620
:102A2000284613F033FC00F10048A169404613F03A
:102A30002DFC002113F022FBE1690746404613F00C
:102A400025FC002113F01AFB216A0546404613F0CD
:102A50001DFC0146304613F011FB064601E000253F
:102A60002F460D9B262B00F286800FFA89F013F07B
:102A7000B9FB81460FFA8AF013F0B4FB0446BDF9A6
:102A80002C0013F0AFFB49468046484613F0FEFB8E
:102A900021468246204613F0F9FB0146504613F0CA
:102AA000EDFA41468246404613F0F0FB014650469F
:102AB00013F0E4FA4E49824613F0A4FD00285AD0E0
:102AC000504614F0D1FF01464FF07E5013F092FCB7
:102AD00082464846514613F0D9FB5146814620466E
:102AE00013F0D4FB51460446404613F0CFFB414B54
:102AF00082461A6A20461146D3F81C800C920D9328
:102B000013F0C4FB41460B90504613F0BFFBDDF8B9
:102B10002CC00146604613F0AFFA0146384613F068
:102B2000ADFA0D9B07469B69504619460B9313F06F
:102B3000ADFB0C9A82461146484613F0A7FB0146AE
:102B4000504613F099FA0146284613F097FA414689
:102B50000546484613F09AFB0B9B804619462046D3
:102B600013F094FB0146404613F086FA01463046C6
:102B700013F084FA0646069B4FF00009D3F8048050
:102B80004946404613F03EFD1B4C002838D00E98B5
:102B90001A4913F019FD002838D03946404613F081
:102BA00075FB049913F072FB0146D4F8440113F04D
:102BB00065FA2946C4F84401404613F067FB0499BE
:102BC00013F064FB0146D4F8480113F057FA31467C
:102BD000C4F84801404613F059FB049913F056FB22
:102BE0000146D4F84C0113F049FAC4F84C010DE049
:102BF0000AD7233CB028002068090020C2B8B23EA2
:102C0000C4F84491C4F84891C4F84C91069B986864
:102C1000064B1B785B0705D4054B1A6844F61F6307
:102C20009A4207D94FF07E5105E000BFB835002029
:102C300058290020A64913F029FB3946804613F095
:102C400025FBD4F8441113F019FA0146089813F043
:102C500015FA29468146404613F018FBD4F848116E
:102C600013F00CFA0146099813F008FA31460746AA
:102C7000404613F00BFBD4F84C1113F0FFF901465A
:102C8000584613F0FBF94FF07C518246049813F03C
:102C9000FDFA05464846294613F0F8FA2946064645
:102CA000384613F0F3FA29468046504613F0EEFA00
:102CB000884B8246D3F800B0874B3146D3F800905A
:102CC000864B09F100401F68854B1D6813F0DEFA42
:102CD00041460890384613F0D9FA089B0146184639
:102CE00013F0CAF951460890284613F0CFFA089B12
:102CF0000146184613F0C0F90146584613F0BEF9D4
:102D0000744B314618600B90584613F0BFFA514689
:102D10000890384613F0BAFA089B0146184613F09B
:102D2000ADF941460890284613F0B0FA089B0146D9
:102D3000184613F0A1F90146484613F09FF9664B77
:102D4000414618600990584613F0A0FA5146089081
:102D5000484613F09BFA089B0146184613F08CF97D
:102D600031460890284613F091FA089B0146184610
:102D700013F084F90146384613F080F9574A51465A
:102D800010600890584613F081FA41468246484642
:102D900013F07CFA0146504613F070F93146804634
:102DA000384613F073FA0146404613F065F90146C0
:102DB000284613F063F9DDF82CC0494B61461860D2
:102DC0000546604613F062FA099A06461146104617
:102DD00013F05CFA0146304613F050F9089B0646A2
:102DE0001946184613F052FA0146304613F046F9D8
:102DF00029460646284613F049FA0146304613F0A4
:102E00003DF914F031FE01464FF07E5013F0F2FA16
:102E10000546304B2946186813F038FA2D4B2946E1
:102E200018602D4B2F4E186813F030FA2A4B2946A4
:102E300018602A4B186813F029FA284B29461860A5
:102E4000274B294D186813F021FA254B18600FF015
:102E5000DDFF296AE86914F07DFC244913F016FAB5
:102E600014F0ACFB3080A86900F1004014F022FCA3
:102E700001461F4813F000F91C4913F007FA14F03B
:102E80009DFB29687080E86814F064FC174900F124
:102E9000004013F0FBF9D4F8501113F0EFF814F0E0
:102EA0008DFB83B213F4004F16BF00F56160B38051
:102EB000B0802C462E6A0F4D3046D5F8541113F0D1
:102EC000A1FB0D4B1A78C8B142F0080218E000BF10
:102ED0000000204160000020A4280020A828002035
:102EE000AC28002028140020B02800204C3D0F44BE
:102EF000DB0FC93F680900204814002022F00802B7
:102F0000AE4F1A70B7F9000013F06CF98146B7F9AB
:102F1000020013F067F98046B7F9040013F062F974
:102F200021680746484613F0B1F961688246404679
:102F300013F0ACF90146504613F0A0F8A1688246A0
:102F4000384613F0A3F90146504613F097F8A169EB
:102F50008246484613F09AF9E1698346404613F0E9
:102F600095F90146584613F089F8394683463046AC
:102F700013F08CF90146584613F080F8E1680646D4
:102F8000484613F083F921698146404613F07EF9E3
:102F90000146484613F072F861698046384613F0DE
:102FA00075F90146404613F069F8069B00F10047A9
:102FB0005B78012B18D1824B1B7859070ED4D5F8BA
:102FC0005801402390FBF3F3C01A13F00BF931467C
:102FD00013F054F813F020FBC5F85801D5F8580148
:102FE000402390FBF3F001E0764B188813F0FAF8D9
:102FF0000146304613F040F8D5F8601106460498B3
:1030000013F03CF80146049813F0F4F9D5F85C414C
:1030100080462146304613F02FF80146404613F013
:1030200035F90146204613F029F8C5F85C0106463B
:10303000504614F0C3FAD5F86451634C297808F06F
:1030400093FF236818442060384614F0B7FA2978B3
:1030500008F08AFF636818446060304614F0AEFAE6
:10306000697808F081FFA368584A18440A991368E0
:10307000A06019441160564A13680133136004E0DC
:10308000544B00221A805A809A80534BB3F9062081
:10309000524B1B6859898A420EDBB2F5FA6FD87918
:1030A000BFBF531A4343A1F5FA6093FBF0F0ACBFE6
:1030B000C0F16400643000E06420494B4949B3F832
:1030C000967193F96031D1F800909BB2049300217E
:1030D00040F2E634404B4FEA410E33F911C0C7EBE2
:1030E0000C0303F2F315A54203D8002BB8BF5B42D3
:1030F00001E04FF4FA7302294FF064053A4C22D0F4
:1031000099F811611EB1B342CCBF9B1B002393FB06
:10311000F5F6DFF8E0B06FF0630A3BF816800AFBC3
:10312000063A01363BF916300FFA88F69B1B03FB73
:103130000AF393FBF5F52D4B4544BC4524F80E509E
:10314000585427DB2CE099F812611EB1B342CCBF72
:103150009B1B002393FBF5F8254E6FF0630B06EBEA
:10316000480A0BFB083306EB4806BAF968A1B6F922
:103170006A61BC45CAEB060606FB03F393FBFBFB47
:10318000049BCAEB0B0A0AFB03FA184BA4F804A031
:103190009D7008DA144D3EF805305B422EF805307C
:1031A0000131032994D10E4DB5F898118A4223DBE1
:1031B000B2F5FA6FA8BF4FF4FA621EE0EA130020DE
:1031C000B835002008000020F825002094350020A4
:1031D000F4250020603500209432002044140020A3
:1031E0006C2A00200C140020B83200208433002008
:1031F000680900202C2700200A46521A4FF47A73DF
:103200005A43C1F5FA61B2FBF1F2642392FBF3F188
:10321000DFF818E36FF063003EF8117000FB012245
:1032200001313EF9111038B2091A4A4392FBF3F307
:103230003B44E380A94BAA4E1F887A0640D5A94B90
:103240000A20B3F9043093FBF0F0A74B1B88C01A97
:1032500000B212F0C7FFA54913F018F8804608F035
:1032600003FF8146404608F08EFE8046B6F9020014
:1032700012F0B8FF8246B6F9000012F0B3FF4946DB
:10328000834613F003F841460490504612F0FEFFC7
:10329000049B0146184612F0EFFE13F0BDF94946B3
:1032A0003080504612F0F2FF41468146584612F0F7
:1032B000EDFF0146484612F0E1FE13F0ADF97080D3
:1032C00095F89C310BB9002F6AD0894E96F8783169
:1032D000B6F8768143B9012006F5BE71002208F0E8
:1032E000B4FB012386F87831824B814F188812F0A5
:1032F00075FF07F5BE7108F075FB13F0B3F980B2E6
:10330000B8FBF0F07C4B00F1010E1B781FFA8EFE2B
:10331000A6F8A0E11BB3B7F9A2910021744E34F8CE
:1033200011C006F5D27838F9112006F5D67709FBD9
:1033300002F237F8113027F811C0C3EB0C0A0FFA6C
:103340008EF392FBF3F3534428F811300131042932
:10335000E4D1694B00221A70A6F8A20104E0B7F884
:10336000A231013BA7F8A231614A0023B2F9A201C0
:10337000002813DDB2F9A0416049A1F1080232F939
:10338000132031F81310424392FBF4F28A1A544985
:1033900021F813200133042BEED101E0A2F8A23171
:1033A00095F89D01002862D04C4B1B885B065ED4CB
:1033B00012F018FF4D4912F069FF12F0F3FA0646B9
:1033C0000F4614F035F8464C8046B4F900008946A3
:1033D00012F0D6FACDE904013046394614F06EF801
:1033E0000646B4F904000F4612F0CAFADDE90423D8
:1033F00082468B464046494612F028FB5246CDE9AC
:1034000006015B463046394612F020FB02460B4669
:10341000DDE9060112F068F912F0B2FD384DB0F5A1
:10342000FA7FA8BF4FF4FA70A842B8BF28464946B1
:103430002080524640465B4612F008FBDDE904233B
:10344000804689463046394612F000FB02460B465C
:103450004046494612F048F912F092FDB0F5FA7F65
:10346000A8BF4FF4FA70A842B8BF2846A080254BE9
:10347000254D1A7812F0040F03D0244B08225A610C
:1034800065E023490968CF075CBF42F001021A706A
:10349000204A2149127816075EBF1A7822F00102ED
:1034A0001A702A6812F0040F02D01C48008870B904
:1034B0001B48008808B1940709D41A4A12880032C0
:1034C00018BF01221AB918480088642830D902228E
:1034D0000A701A7822F001021A702FE0C41300203B
:1034E000B832002028140020E611002035FA8E3C66
:1034F00068090020BC13002074120020140B002067
:103500000CFEFFFFB8350020C0130020000C014066
:10351000C81300204814002058350020B235002080
:10352000A0110020B03500203029002014270020F1
:103530001B78D80756BF02230A700B700FF068F98A
:103540008B4B1B68C01A002801DB11F0A3FF894BCD
:103550009B680BB1884898472868884B012210F077
:10356000080F1A70864CDFF860823BD08549864F81
:103570008E8806F10E039BB21C2B844BB3F90430EA
:103580002CD8834A1288520728D50A2293FBF2F2DC
:103590003B88D21A92B293B21FB2B337BCBF02F5C6
:1035A000B47293B21AB2B32A7A4AC8BFA3F5B473FD
:1035B0001278C8BF9BB2120794F8607112D57FB21F
:1035C0007F427B43D8F800201BB2527A53436FF0FE
:1035D0001D0293FBF2F31E448E8003E00A2293FB4C
:1035E000F2F33B8010F0140FDFF8E09174D0684BD9
:1035F0001B8803F40273002B6ED0664B614A1B7864
:1036000003F0100303F0FF0643B1634B94F9EE019E
:103610001968538800FB013353805DE0D9F8B80185
:103620005E4FC1785E4B807839B3B3F900E0B7F9EB
:103630000630CEEB03010029B8BF494281420FDDBD
:10364000584973450E604FF00101C8BF434289F8E5
:10365000BC11D188CCBF9BB283B20B44D3803BE07A
:1036600099F8BC312BB1504B89F8BC6119684F4BAC
:103670001960494B1B68734423E0B3F90060B7F944
:1036800006309B1B83EAE377A7EBE37787420ADDEB
:10369000022193FBF1F346490B60464901230B706D
:1036A00089F8BC310AE099F8BC313BB13E4B89F84E
:1036B000BC1118683D4B18603E4B1970364B1B68A7
:1036C0003344D9F8C001018840888B4203DB834230
:1036D000A8BF03461946D180374B1B78B3B12F4B97
:1036E000B3F90620B4F898319A420FDC244B5B7989
:1036F000012B01D0192B02D194F8E82132B90E2BFD
:1037000004D0082B1EBF1F4B00229A80D8F800302F
:1037100093F81871002F60D01D4B1B8898075CD060
:10372000264B27491E6A304612F058FF00284FD119
:10373000304613F0BFFFD9F8C41112F0A7FD13F003
:103740003DFFB0F5617FA8BF4FF4617012F04AFDF4
:103750001C4912F04FFE08F016FC0646384612F0DF
:1037600041FD314612F092FD13F028FF80B230E0A7
:103770005C350020083400201C0B0020751200204E
:103780006C2A0020B8320020E41100202814002008
:10379000C4130020481400201C260020943200206E
:1037A000761200201826002030140020701400200B
:1037B000983500202026002002000020B02800209C
:1037C0008FC2753CEFB6B0440C140020680900208D
:1037D00000209D4AD3881844D0802B68990640F178
:1037E00099809A4B1B8803F03003002B00F09280E5
:1037F000974B1B78DA0740F18D80964BB3F90400A4
:103800000A2390FBF3F012F0EDFC934912F03EFD19
:10381000054608F0B8FB0746284608F025FC8F4B04
:1038200006461B688E4AD9788E4D00293FD0DFF8B6
:1038300074B2B2F90200BBF802A006910FFA8AF343
:10384000C01A04920BF0BEF80699049A4B429842B3
:1038500003DB8842A8BF084600E01846BBF800C05A
:103860008244B2F900000FFA8CF21FFA8AFA801A29
:103870000893CDF810C00691ABF802A00BF0A2F8A7
:10388000089BDDF810C0984204DB06990346884285
:10389000A8BF0B4663449BB2ABF800300FFA8AF026
:1038A000049312F09FFC049B834618B208E0B2F91F
:1038B0000200049212F096FC049A8346B2F90000CA
:1038C00012F090FC31468246584612F0DFFC394631
:1038D0000490504612F0DAFC049B0146184612F0A0
:1038E000CBFB614912F086FD12F096FE3946288026
:1038F000584612F0CBFC31460746504612F0C6FC43
:103900000146384612F0BAFB574912F073FD12F027
:1039100083FE6880554B1B784BB1554B00221A60D3
:103920005A609A60534B00221A605A609A60524B58
:10393000D8F80000B4F86C210093504B1C68504B31
:10394000196800F15803A0474E4B4F49DB780693A6
:103950004E4B93F80080B8F1030F16D9D9F8C8314F
:103960005C88B4F5FA7F10D2374BB1F90450B3F943
:10397000040062420028B8BF4042131A9D4203DB94
:103980002318AB42A8BF2B468B80414B1B6813F01A
:1039900000630BD0D9F8C82100254B880F8804920A
:1039A000B1F904A03B4E2C46AB46B2E09B463A4AE6
:1039B000D9F8C8711370244A4D88B2F806A00E8851
:1039C000B1F90490354CC34504F1100480F08281B4
:1039D0000FFA8AF012F006FC54F8181C12F056FC8C
:1039E000049028B212F0FEFB54F8101C12F04EFCAA
:1039F000049B0146184612F041FB049030B212F0CD
:103A0000F1FB54F8141C12F041FC049B01461846CB
:103A100012F034FB049097F90000404209FB00F0DB
:103A200012F0E0FB54F80C1C12F030FC049B014631
:103A3000184612F023FB12F0EFFD194B23F81B0080
:103A40000BF1010BBFE700BFB8320020C413002008
:103A5000481400202814002035FA8E3CEC11002078
:103A6000F6110020B43500200000204104000020A1
:103A700078330020FC330020F42B00209403002036
:103A80004414002034350020AC330020802700206F
:103A9000C8130020340B0020BF3500203C0B002051
:103AA00010140020F211002018B2099312F09AFBB2
:103AB000B16812F0EBFB089038B212F093FB71681A
:103AC00012F0E4FB089A0146104612F0D7FA049B64
:103AD000089093F9000040420AFB00F012F082FBCC
:103AE000F16812F0D3FB089A0146104612F0C6FAAC
:103AF00012F092FD11AA80B222F81B0021B202B28C
:103B00008A42099B08DD0446284605460BF1010B55
:103B10001036C345C8D304E029B28A42F5DB2046FB
:103B2000F1E79F4B9F49DF880B68641BDB04A4B25D
:103B300022D59D4BB3F906209C4B1D68A888EB88C5
:103B4000C61AB24205DC9A4B2E881B681D880123D9
:103B500007E003449A42964B6D881B685E8803DB3E
:103B6000002389F88C3200E02F46A9F88E62A9F86C
:103B70009052A9F8927203E08D4B1B681D885E88F5
:103B8000B2B21FFA85FECEEB020080B203B224B2BD
:103B90009C42DFF838C24FF0000311DD01228CF89F
:103BA0000020434516D20DF1440E3EF913C002B277
:103BB00002FB0CF292FBF4F22EF813200133F0E733
:103BC000022694FBF6F40EEB0405161B8CF800306D
:103BD000ADB2B6B20A68754902F48053089399F8F9
:103BE0008C32DFF8ECA10A93714B0024D3F800B0BB
:103BF0000B68049302F010036E4A0E93127802F0E1
:103C00000402D3B2684A0B93B2F906300C93D9F888
:103C100094320D934FEA48030F930F9B9C4259D067
:103C200011A9085F12F0DEFA099038B212F0DAFA40
:103C3000614951F8341012F029FB804628B212F085
:103C4000D1FA81464046494612F0BEFC48B930B22E
:103C500012F0C8FA81464046494612F0D3FC00B93A
:103C6000C1464946099812F009FA12F0D5FC069BA4
:103C700080B22AF8020F00B213B1BBF804100EE0B4
:103C8000089B53B10A9B2BB1049BBBF80010B3F8FF
:103C900000E006E0049B598801E0BBF80010BBF887
:103CA00002E0884203DB70450146A8BF71460E9BC7
:103CB000AAF8001063B10B9B53B1089B43B90D9B4D
:103CC000198A0C9B8B42BCBFBBF80410AAF80010E9
:103CD0000234A2E737490A788B4602F0040202F068
:103CE000FF0312B9354A127888E0354B1B6813F090
:103CF000006308D0334890F89832013BDBB2182BB0
:103D000000F29D8185E0274ADFF8B0801668DFF871
:103D1000B8E016F4805A17D1BEF8003098F80000C9
:103D2000012181421AB207D23EF9113001319A4283
:103D3000B8BF1A4693B2F4E71D49096849888A4218
:103D400004DD5B1A9AB202E01A4600E00022164B2C
:103D50001D49B3F906401B4BD3F894C2134B1D68A1
:103D6000134B186898F800300EEB430E7145C1D024
:103D7000BAF1000F40F043840B88069F9B1A9BB258
:103D80000B80B0F802801BB227B3B0F804904B450B
:103D900003DB4345A8BF43469946A1F800902BE0BA
:103DA000B83200202835002094320020242800203A
:103DB00028280020B8350020340B00208027002060
:103DC000C81300206809002010140020BF3500200F
:103DD0000E140020B0F800904B4503DB4345A8BF0C
:103DE00043469946A1F80090BCF810309C4203DA93
:103DF000F70601D583880B800231B7E79342BFF401
:103E000079AFC44931F81300C34921F813000133D5
:103E1000F4E701229A40C14B1340002B00F00F81C0
:103E2000BF4BC0491B8813F4807F08D0BE4B1A8853
:103E3000ADF844205A889B88ADF8462015E0BB4B6E
:103E40001A88ADF844205A889B88ADF84620B84AB5
:103E5000ADF848301268D40409D5D0F89422B1F9ED
:103E60000640D289944202DA5B42ADF84830B14D47
:103E70004FF47A72B5F902304FF4616403F5E163EF
:103E8000534393FBF4F3A3F5FA73ADF85C30B5F943
:103E9000003003F5E1635A4392FBF4F29E4BA2F526
:103EA000FA721B88ADF85E20A3F2DC53ADF84A30FD
:103EB000D0F894320A88DB89D21AADF84C204A88AF
:103EC000D21AADF84E208A88D21AADF85020CA888E
:103ED000D21AADF852200A89D21AADF854204A8974
:103EE000D21AADF856208A89D21AADF85820CA895C
:103EF000D31AADF85A3000238F4A002122F813104C
:103F00000133082BF8D18D4B8D491B688D4D0493DF
:103F10008D4B1B6806938D4B1B78C3EBC30301EBE2
:103F20000308414573D00B7833B103F11502012327
:103F30009340049A134066D0069B11F806EC0E27B6
:103F400007FB0E37B7F90020B7F9023064209B1A3F
:103F500011F9022C9BB25A4392FBF0F211F805AC16
:103F60004FEA530911F8034CC9EB02024FEA4A0623
:103F700018A892B211F801CC064414B936F81C0CFA
:103F80000CE0B5F9000036F91C6CB04208DA0444C4
:103F9000844203DBA6423046A8BF2046288008E0C2
:103FA00007DD041BB44203DB8442A8BF0446264657
:103FB0002E80D7F80A40012000FA0AF02042B5F915
:103FC000006011F9040C12B200FB06F04FF0640619
:103FD00090FBF6F014BF4FF0FF34012490420ADB4F
:103FE0004FFA8CF25A4392FBF6F2C9EB020212B27C
:103FF0008242A8BF0246504B33F81E9002FB049445
:1040000023F81E4000E02B800235073189E74E4B34
:104010004F4E1F6800250E2303FB057393F90640DE
:1040200036F9023FE8B26343642493FBF4F434802E
:104030000EF0D2FE01352044082D3080EBD13C4FEC
:104040003D4D3B68404E13F0200F33D000200EF062
:10405000C3FE2880044601200EF0BEFE374B688068
:104060001B68190626D53B4B324AD3F8BC321B7865
:10407000012B23D13168B2F9003091F914E04FF0EF
:10408000320C03FB0EF393FBFCF31FFA83FE91F952
:104090000630B2F902205B4253436FF0310193FBCB
:1040A000F1F193FBFCF30EEB0102A118734429809C
:1040B00018446880D6F800E0002319E0D6F800E044
:1040C000B2F902309EF906105943322391FBF3F105
:1040D000214429809EF91440B2F9001001FB04F23A
:1040E00092FBF3F21044E4E70133082B2A5333D058
:1040F0000E2101FB03E135F91300B1F900205C004A
:104100009042B1F90210EFDB0AB28242A8BF024628
:10411000EAE700BF0A290020101400209920980126
:10412000C413002094320020B8320020AC330020A9
:104130002835002028140020FC130020C81300207C
:1041400033280020020C00200C2300202C28002003
:10415000FA13002068090020AA4CD4F8C89199F9F4
:104160000830A3B994F8988208F1FF33182B72D85D
:10417000DFE803F03571714F7171714871717171C0
:10418000715971717171714F657171593500DFF835
:1041900094A24FF000089C4B882000FB08303AF9AD
:1041A000021FB9F906200EF02DFC32680E2303FB26
:1041B000082280B2AAF80000B2F9003000B298429A
:1041C000B2F9022003DB13B28342A8BF034608F111
:1041D0000108B8F1080FAAF80030DCD1C2E799F85D
:1041E000043013B10020698908E09BF8003003F027
:1041F000040303F0FF00002BF4D1014609F0A8F8F6
:10420000012629E00020E98809F0A2F80120298987
:1042100005E00020298909F09BF86989012009F04F
:1042200097F8022618E00226B01E35F81610C0B224
:10423000013609F08DF8082EF6D106260CE003268B
:10424000F01E35F81610C0B2013609F081F8072EBD
:10425000F6D1042600E000263B689A0602D4B8F1A5
:10426000050F0AD13046298809F072F8701CC0B2D7
:10427000698809F06DF80236F6B23B68DB0205D4B6
:1042800094F800377BB10EF0EDFC0CE0DFF898817C
:1042900000257019C0B238F8021F09F059F80D2D29
:1042A000EED00135F5E7594B1878002840F0CB8166
:1042B0003B681D0340F1C78194F80137023B052B91
:1042C00020D8534B93F8D83733B1012B0AD10AF0D9
:1042D0007DFDC0F17F0005E04A4BD3F80407036879
:1042E0009B689847D4F8083794F80C271344B3F523
:1042F000807FA8BF4FF480738342D4BFC4F80837CF
:10430000C4F8080794F80137023B082B00F27081CB
:10431000DFE813F00900400062008C00A500B70040
:10432000340152015F013B4B1A68D4F814376433EF
:104330009A4240F25D8140200DF016FC002840F0CA
:1043400057814027344BD4F810272E4E985C1D46D9
:1043500078B106F0ABFDD6F80837013F03F1FF3323
:10436000C6F80837D6F8103703F10103C6F810373E
:10437000E8D1D4F81027234BAA5C002A40F03881FA
:10438000C3F810274FF0FF32C3F81427032283F835
:1043900001272DE129230093204B492003F10C0232
:1043A000019302925021A3F10A02023307F05CF953
:1043B000002840F01D813B684FF0FF3213F080036E
:1043C00005D0C4F81007C4F814270423D3E0C4F8B8
:1043D0001037C4F8142740E0114A0223002100934B
:1043E00001910291482002F1080307F03DF90028ED
:1043F00040F0FE804FF0FF33C4F81437C4F81007C4
:104400000523B8E068090020280C0020BA350020F8
:104410006C2A002058290020E0AB01084AAC0108B2
:104420002CAE0108FA1300209A32002007230093D3
:10443000864B472003F10C02019302920021A3F165
:104440000802043307F010F9002840F0D1804FF043
:10445000FF33C4F81007C4F8143706238BE07C4AF6
:1044600005230021009301910291532002F10803DA
:1044700007F0FAF8002840F0BB80C4F810070723C3
:1044800079E040200DF070FB002840F0B180D4F8B6
:1044900010370C2B66D8DFE803F0070B0E12192536
:1044A0002A2F3337455054006A4812F029FE53E052
:1044B00069486A4913E06A486A496B4A4AE06B4BAB
:1044C0006B4893F8D61793F8D72743E0674B0C2136
:1044D00093F8B027674801FB023393F8B21712F044
:1044E0000FFE39E0614B6448B3F84011F7E75F4BCA
:1044F0006248B3F84211F2E7614B62481969EEE78E
:10450000614B62481988EAE7D4F81837D80404D513
:10451000564B5F4893F87A11E1E75E4B0B22C3F8E4
:10452000102719E0514B5C4893F87E1193F87F21D6
:1045300093F87D3112F0E4FD0EE05848B4F81C17F2
:10454000CDE73B68190507D5484B5548B3F88211AC
:10455000B3F9802112F0D4FDD4F810370133C4F838
:10456000103745E00DF060FB002841D04FF4805338
:10457000A4F81E37092384F8013739E0494B1B683A
:104580009A0116D5B4F82037424D93B9D5F824379F
:104590000E201193444B11A91B68129306F070FD75
:1045A0004FF48053A5F81E37092385F8013706F02C
:1045B000BFFD06F047FD1BE094F82837002BF6D02E
:1045C000384B1B689B01F2D4324B082283F8012739
:1045D000EFE7364B1A68D4F81437C8339A4203D938
:1045E0000DF008FB0123C6E70DF01EFB0028F7D1F4
:1045F0000DF0EAFA38B3012384F8013723E0BCF860
:104600000E80EB88C3EB08094C4502DD43449C4215
:1046100013DB4445C8BF6B88B1F90080D6BF8388DF
:10462000B0F80290B5F800909845FFF6E4ABC845A5
:104630004346A8BF4B46FFF7DEBB4445CCBF6B8863
:104640002B88FFF7D8BB19B0BDE8F08F44AE010846
:1046500090AE01086CCE010886CE01089BCE010801
:10466000A3CE0108B7CE0108C3CE01086C2A0020F2
:10467000CCCE0108DDCE0108E7CE0108F6CE010858
:104680000834002005CF01080800002015CF0108DC
:104690001FCF0108680900202CCF010845CF010871
:1046A00050CF0108C8130020DC2500205829002025
:1046B0002DE9F04F9F4FA04C3A6889B002F59C431A
:1046C000203323609D4B1E78CEB19D4909688A42F4
:1046D00040F20781013E1E7003E1DFF88482072D5E
:1046E000D8F800308CBF2946595D964B96481B6818
:1046F0009847032D09D904EB4505A880013610F031
:104700005DFEF5B28542E8D320E0D8F8002005F13F
:104710000E0302EB8303D9881A890028EBD04FF4EB
:104720007A73401A5843531A90FBF3F040F6C903CA
:1047300000F57A70984205DC40F2EE239842B8BF4B
:10474000184601E040F6CA0080B2D4E742F2010AFE
:104750007E4B7F4E1B68D6F8008003EA0A0ABAFA3D
:104760008AFA4FEA5A1A7B4BBAF1000F05D194F836
:1047700028201A70784A517811701B782BB1764B2B
:1047800093F8009089F0010900E099460F23DFF8C3
:10479000E8B184F82930002510F010FE854267DA70
:1047A0006B00B9F1000F03D06C4A32F8150000E03D
:1047B00048466B4ADFF8C4C111684FEA850ECA8AC1
:1047C0008242684A02D8098B81421CD25CF80E00F2
:1047D0005949804501D2D05A19E0E8B203920293B8
:1047E000019110F003FE032D029B039A0FDC019947
:1047F0004FF0010E91F829C00EFA05FE2CEA0E0EBC
:1048000081F829E003E008F596714CF80E10BAF132
:10481000000F28D194F8BC100322B1FBF2F202EB96
:1048200042028A1AD2B203EB050E724404EB420232
:10483000508594F8BD202AB9022913D93E4A012196
:1048400082F8BD10BBF800203BF8020C1044BBF806
:1048500002201044444A80B2D05200B2032290FB9E
:10486000F2F080B23F4AD05201350BF1060B93E7CC
:1048700094F829203D4BA2F10F014A424A4184F8A5
:10488000D6206AB13A4A1268520109D43268D9680E
:104890009A60521AC82A1FD9012283F821201BE0EE
:1048A0002D4A01215170117032689968DA605B6895
:1048B000521A9A4282BF2D4B002283F821200025F4
:1048C00010F07CFD854207DAE8B210F08FFD254B31
:1048D00023F815000135F3E794F8BC30013384F870
:1048E000BC301A4E3368DD0405D5214B1B68D80750
:1048F00001D40BF039FE1A4B3F681A68907A0028F1
:104900003ED01849137B013831F810001BB1C0F5B7
:104910003B60083080B200B2A0F57A70B0F57A7FC3
:10492000A8BF4FF47A7020EAE07011F05BFC1149E7
:104930005BE000BFDC25002098100020303500200F
:104940002C3500204403002054320020283500205C
:1049500058290020AC180020000000209C100020E6
:1049600024350020943200205611002034350020D8
:10497000C813002000007A44C41000200C1100204D
:10498000336819043AD5D4F8D830934DFB1A002B6C
:1049900034DB07F59C432033C5F8D8308F4BD27AEF
:1049A00059798F4B33F8113095F8DC109BB293FB9B
:1049B000F2F3013101F00F0285F8DC202A4482F87D
:1049C000DD300346874A825C0130134410289BB2D5
:1049D000F8D11BB293FBF0F000B26428A8BF6420AA
:1049E00020EAE07011F0FEFB7F4911F003FD7F49E2
:1049F00011F04CFC11F036FE7D4B188033687D4D74
:104A000013F4807F00F00F817B4BDFF8F0919F4221
:104A100005D999F8022012B9012289F8022099F8E3
:104A20000220002A00F0FF80744A95F8008092F876
:104A30002170C8F380087A1E57425741704A002FF0
:104A40009246116818BF4FF0000BC1F380630193C9
:104A500008BF4FF0030B99F82020052A00F2DD80F3
:104A6000DFE802F0034E537988A5B8F1000F3AD081
:104A7000D4F8F000B4F8F4100DF087FE012809D145
:104A80006049614A09681268C988642000FB0122F4
:104A9000C9F81020019B6BB15A4A126812794AB1C9
:104AA00010F068FA032289F820204FF47A72C9F8CE
:104AB0001C20D0E7002F40F0B080534AD9F81010E6
:104AC00010684E4A88420AD9029210F053FA029AAC
:104AD000032182F8201040F6B831D161BBE70121F3
:104AE00082F82010B7E7019B4FF4806013B107F004
:104AF000D5FA01E007F0C2FA0022C9F810208CE0D4
:104B0000002F49D110F036FAA5E727B1052289F820
:104B10002020012000E03846B8F1000F0CD0D4F876
:104B2000F0204FF0020BD189384A118051809180DA
:104B3000344909684988D180334A1168D9F814206A
:104B4000914202D8B8F1000F64D147F23052C9F84F
:104B50001C20032221E02A7842F002022A700BF086
:104B600003FD294AD9F81C1012680A44C9F8182014
:104B7000042212E0244A9FB11168D9F8182091420A
:104B80004BD9234A92781AB9DAF80020D30744D4D3
:104B90002A7822F002022A70052289F820205AE79A
:104BA0001268D9F81C100A44C9F8182035E01549D4
:104BB000154A09681268C988642000FB01224FF475
:104BC0008060C9F81020002289F8202089F803208D
:104BD00007F054FA3FE700BF981000204817002064
:104BE00058170020751100200000C84200C07F4403
:104BF0003C140020B8350020404B4C0034350020D8
:104C0000C81300204434002058290020943200208A
:104C10000000002000287FF41EAFBBF1000F02D07F
:104C200058460DF04DFEDFF8C082A44F08F5C47061
:104C3000B8F84E110DF0A9FDCDF80480814628BBCF
:104C40009F4B1B6813F0006808D0FB7833B90FF056
:104C5000F7FC9C4B012818BF002018702B785807D0
:104C600007D53368D90604D4B8F1000F01D0FB781A
:104C700053B3954B01221B683A7103F57A73C4F85C
:104C8000F830904BFA7000221A701DE03368DA0693
:104C900015D42B785B0712D5894B1B6818010ED5EC
:104CA000FB7863B1884B1A68D4F8F8309A4209D976
:104CB0000FF0C6FC30B9834BF870187002E0814BDE
:104CC00000221A7000233B712B78590735D53368C1
:104CD000DA0632D57D4B1B78DB062ED4BB789BB130
:104CE000019B93F8E231B9F1000F15D17BB1764BFE
:104CF0001A68D4F8FC309B1A002B08DA0BF034FC4D
:104D0000734B83F8009118E0B9F1000F0DD110201A
:104D10000DF0D6FD01230EE03BB16B4A4FF47A71E2
:104D2000126801FB0323C4F8FC3094F8003123B16E
:104D30000DF0B0FD002384F80031019B002293F8B0
:104D4000E0B193F8E111B3F898E1B3F89AC11346D2
:104D5000DFF898A19B083AF9120001327045C4BFF0
:104D600063F07F03DBB26045B8BF43F04003042A21
:104D7000EED194F8012156489A4205D190F80221CB
:104D8000F92A04D8013200E0002280F8022184F8D8
:104D90000131BB784E4ADFF8288133BBD8F80000D8
:104DA000C0070AD582F80331B9F1000F1DD12B7865
:104DB000DB071AD50BF004FA17E02B78580714D547
:104DC000444B1B788BB1444BDB7873B992F80331B9
:104DD0000133DBB2032B82F8033106D911B10BF09A
:104DE000C3FB02E0B9F1000FF9D094F80231384A60
:104DF000142BDFF8FC9040F0A480BB781BF1000B73
:104E000018BF4FF0010B6BB392F801315F2B11D13A
:104E10002B7803F0040303F0FF0113B10BF0A4FBA4
:104E200008E00B20039102920DF04AFD029A0399CB
:104E300082F80211BBF1000F14D094F801317D2BE0
:104E400010D12B7803F0040303F0FF0213B10BF031
:104E50008BFB07E00B2002920DF032FD1C4B029AF7
:104E600083F802212B7803F0040303F0FF01002BE9
:104E700067D194F80131164A572B10D1174B4FF4D4
:104E80007A721A8033681B0601D509F043FE144B71
:104E90001B685F0755D5134B0A221A8051E0306812
:104EA000400734D55A2B32D192F8043113B3012381
:104EB00082F8041182F8053143E000BF00000020B1
:104EC000C8130020C03500205829002048140020B5
:104ED00098100020AC18002034350020B035002098
:104EE000C0130020B23500206C2A0020943200202C
:104EF0000C14002092F8063183F0010382F8063189
:104F00000BB10C2000E00D200DF0DAFC19E05D2B58
:104F100000F029855B2B00F028855E2B02D1032051
:104F200000F024BD562B01D107F072FBBB78002B9B
:104F300000F0308594F801316F2B40F025850BF09F
:104F40003FF93368580738D594F80631B64A9BB113
:104F50002B78590710D5019BBAF90610B3F8983190
:104F6000994209DDD8F8003013F0010302BF322165
:104F7000A2F80A1182F80631D8F80030DA030DD50C
:104F800094F80C21A84B2AB993F8042112B93222C3
:104F9000A3F80A21012384F80C310EE094F80431BF
:104FA000A14A53B12B7803F0040303F0FF0123B9A6
:104FB000012382F8041182F80531D9F8009000230A
:104FC000C8F8003009F17B0709F1CB0A3A787B7801
:104FD00017F8010C9A420DD239460DF08DFB48B1FD
:104FE00017F8022C012303FA02F2D8F80030134319
:104FF000C8F8003004375745E8D18C4B1B784BB1CB
:105000008B4BDFF848921A68984612F0020F40F076
:10501000308328E309F1CA0709F589783A787B7863
:1050200017F8010C9A4225D239460DF065FB08B3FA
:1050300097F804C00C21BB7801FB0C417D4A013B71
:1050400003EB43031344D1F8142197F803909A42D9
:1050500075480FD0C1F81431002390F84021C1F8F1
:105060001831012303FA0CF322EA030381F81091AB
:1050700080F8403106374745D0D16F4BDFF8D0A1DB
:10508000D3F800806D4B4FF0000B1B6802936C4B04
:105090001B780393DAF80030002B00F0DB8293F8E2
:1050A0000090B9F1000F00F0D582DAF804200299DF
:1050B0008A1A002A0CDB01F5FA72CAF8042094F867
:1050C0004011012202FA0BF221EA020284F8402187
:1050D000039A002A00F0BE821AF8042C5978043290
:1050E000D2B2002940F07782564931F91210564A5F
:1050F000B2F8962102F1C800814201DD9F7814E0E8
:10510000C83A914202DA99784F420EE094F8402171
:10511000012303FA0BF322EA030384F84031029BD4
:1051200003F5FA73CAF8043094E294F8403143FA74
:105130000BF3DB0700F18E82002FCCBF0220012091
:105140000DF0F6FB09F1FF32374B132A00F27A8299
:10515000DFE812F0140023003200440061008000F8
:10516000E5004A01AF01E201110278024400550056
:105170008000E5004A01B7001C01810198F8001089
:1051800040460F44FA2FA8BFFA2727EAE77788F8A6
:1051900000700DF097FA01201EE098F801104046CB
:1051A0000F44642FA8BF642727EAE77788F80170C7
:1051B0000DF088FA02200FE098F8031040460F44E3
:1051C000642FA8BF642727EAE77788F80370D3F82D
:1051D00044110DF02FFA03203946C9E198F8051063
:1051E0000D2039446429A8BF642121EAE17188F8BF
:1051F00005100DF0F9FAB9F10D0F00F0238298F8BF
:1052000004100E2039446429A8BF642121EAE17109
:1052100088F80410ACE198F806100520394481F3B1
:10522000080188F80610A3E198100020BA35002084
:10523000C8130020B8AE01084414002058290020EB
:10524000AC180020943200206C2A0020C0130020EB
:10525000AC110020D3F848311A78022A22D13846FE
:10526000049310F0BFFFA94911F0C4F8049B596AD8
:10527000059310F003FF0021049011F0A5F9059BA0
:1052800048B9049AA149104611F0BCF9049A059B4B
:1052900010B19E4A00E000225A620F2011460DF024
:1052A0008FFA0AE099780F203944C829A8BFC8218D
:1052B00021EAE17199700DF097FAB9F10F0F00F042
:1052C000C181934BD3F8489199F80030022B1AD141
:1052D000384610F087FF8D4911F08CF8D9F820106E
:1052E00010F0CCFE0021074611F06EF930B93846B7
:1052F000864911F087F910B1844F00E00027C9F802
:105300002070122057E199F8011012203944C82961
:10531000A8BFC82121EAE17189F8011028E1D3F87A
:1053200048311A78022A22D13846049310F05AFFE5
:10533000764911F05FF8049B196B059310F09EFEFF
:105340000021049011F040F9059B48B9049A6F4977
:10535000104611F057F9049A059B10B16B4A00E012
:1053600000221A63102011460DF02AFA0AE0197B78
:1053700010203944C829A8BFC82121EAE171197356
:105380000DF032FAB9F1100F00F05C81604BD3F8E8
:10539000489199F80030022B1AD1384610F022FFBC
:1053A0005A4911F027F8D9F82C1010F067FE0021A7
:1053B000074611F009F930B93846544911F022F97D
:1053C00010B1524F00E00027C9F82C701320F2E012
:1053D00099F80B1013203944C829A8BFC82121EA25
:1053E000E17189F80B10C3E0D3F848311A78022A2A
:1053F00022D13846049310F0F5FE464910F0FAFF2A
:10540000049BD96B059310F039FE0021049011F034
:10541000DBF8059B48B9049A3C49104611F0F2F8B4
:10542000049A059B10B1394A00E00022DA6311208A
:1054300011460DF0C5F90AE0997D11203944C829BB
:10544000A8BFC82121EAE17199750DF0CDF9B9F134
:10545000110F00F0F7802E4BD3F8489199F80030E7
:10546000022B1AD1384610F0BDFE2A4910F0C2FFB7
:10547000D9F8381010F002FE0021074611F0A4F808
:1054800030B93846214911F0BDF810B11F4F00E086
:105490000027C9F8387014208DE099F815101420F1
:1054A0003944C829A8BFC82121EAE17189F815103B
:1054B0005EE0D3F8489199F80030022B1AD13846B3
:1054C00010F090FE114910F095FFD9F8281010F057
:1054D000D5FD0021074611F077F830B938460B4961
:1054E00011F090F810B1094F00E00027C9F82870BA
:1054F000092060E099F8031009203944C829A8BFA1
:10550000C82121EAE17189F8031031E00000C842A6
:105510009810002000007A44D3F8489199F80030A0
:10552000022B1AD1384610F05DFEB54910F062FF2B
:10553000D9F8341010F0A2FD0021074611F044F80C
:1055400030B93846AE4911F05DF810B1AC4F00E00B
:105550000027C9F834700A202DE099F80D100A20B0
:105560003944C829A8BFC82121EAE17189F80D1082
:105570000DF03AF966E0D3F8489199F80030022B23
:105580001DD1384610F02EFE9E4910F033FFD9F899
:10559000401010F073FD0021074611F015F830B9E6
:1055A0003846974911F02EF810B1954F00E00027CA
:1055B000C9F840700B2039460DF002F942E099F825
:1055C00017100B203944C829A8BFC82121EAE1716E
:1055D00089F81710CCE7012934D198788A4B33F930
:1055E0001230B3F5617F05DB40F633029342A8BF6A
:1055F000134601E04FF46173B9F10C0F22D14FF45F
:10560000966292FBF0F0A3F5617393FBF0F37F4A8F
:10561000DFB21378BB4215D0042F34BF3B460223C0
:105620001370019A09FB0323794A03F2B2731360E2
:105630000CF021F8484639460DF0D6F8781CC0B277
:105640000DF076F994F84021012303FA0BF313438C
:1056500084F840310BF1010BBBF1040F0AF10C0A85
:105660007FF418ADCCE43368D8050FD5694BDB78EF
:1056700063B1D9F80030990708D5674B1B8813F040
:10568000010708D1012006F009FD04E0012006F021
:10569000F5FC012300E00023D8F8002052070BD5C9
:1056A00053B1012006F0EAFC5B4B1B889B0706D434
:1056B000022006F0F3FC02E0022006F0DFFCD9F83D
:1056C000003013F00A0F32D0D8F80030DF060FD5C3
:1056D000514B1B8858070ED4042006F0DFFC4F4BBB
:1056E0000A22B3F9043093FBF2F3A4F84C3102E040
:1056F000042006F0C3FCD8F80030990607D5464BC5
:105700001B885A0606D4402006F0C8FC02E0402060
:1057100006F0B4FCD8F800305B0641BF3F4B0A22CC
:10572000B3F9043093FBF2F348BFA4F84E31D9F833
:1057300000309F0609D4D8F80030180540F1B88031
:105740004FF4807006F0AAFCB6E0354BDFF8C8A035
:105750001B7813F0020F6DD0324B1B78042B69D9E4
:10576000D8F8003013F4007B0FD0BAF80030D90617
:105770003AD4102006F092FC202006F07FFC2A4844
:10578000011D09F031F902232AE0BAF8007007F090
:105790001007BFB22FB1102006F070FC012784F86B
:1057A00050B1D8F800305A0512D5D4F854311F49F9
:1057B0005A89B1F90030002BB8BF5B42934207DA37
:1057C000B1F90230002BB8BF5B429342C0F2258191
:1057D000BAF800309B0608D5202006F04FFC0023C5
:1057E00084F85031012700E0002794F8583193BB2A
:1057F0000E200DF065F80E4B012283F858212AE0A7
:105800000000C84200007A44943200200829002099
:105810004414002034350020C41300202814002034
:10582000481400204914002060140020B8320020E1
:1058300098100020BAF8003003F03003002B3FF43A
:105840007AAF102006F01AFC202006F017FC002387
:1058500084F8503102E0002F3FF46DAF002217466C
:105860007A4B002023F81700794B191D03F10A0E1B
:1058700021F81700002142F80E109644CEF80400DB
:10588000CEF8081023F8170003F1320E5A3342F80D
:105890000E10D15096441344CEF80400CEF80810F0
:1058A000586099601432002F7FF445AF0127D7E785
:1058B0004FF4807006F0E2FB664B5A791F46082AC7
:1058C00001D00E2A02D1402006F0D8FB33685805DB
:1058D00019D597F818321BB92B7813F0040F03E091
:1058E000D8F8003013F4002F09D05B4B00221A7057
:1058F0003C200EF073FE30B10EF02EF8F8E707F002
:1059000047FF0EF08CFD012384F8DC3194F8DD3183
:10591000002B00F09880D9F80030590740F19380AF
:10592000D8F800301A0705D4082009B0BDE8F04FB8
:1059300006F0A4BB494B1C8804F00804A4B2002C58
:1059400040F08180082006F0A9FB454B1A68454BC2
:105950001A60454BDA88454BA3F8DE21444B1C60A6
:10596000444B1C606FE0012000E00220C7B2019AA6
:105970007B1E82F8B03706F0D3FB06F077FC384682
:105980000CF0D6FFFFF7DDBABBF1000F02D07E2B83
:105990003FF4D5AA94F80131972B06D1334B4FF43D
:1059A000C872A3F80821FFF7CCBAA72B06D1324A58
:1059B000137843F004031370FFF7C3BA0022BB2B24
:1059C000079201D1022303E0B72B04D14FF6FE73F7
:1059D000ADF81E300AE0BE2B01D1022304E0BD2B3E
:1059E0007FF4AFAA4FF6FE73ADF81C30D9F8003043
:1059F000BDF81C10B3F858200A44A3F85820BDF88D
:105A00001E10B3F85A200A44A3F85A2006F000FEEC
:105A1000002384F80231FFF794BABAF800309B06ED
:105A20003FF5E3AE202006F039FB144B14481A680A
:105A30005B68011D4360026008F0D6FF0B4B012735
:105A400083F85071D1E609B0BDE8F08FB43500207D
:105A5000F21100206C2A002060320020C4130020C4
:105A60003014002070140020943200209810002080
:105A7000182600201C260020481400204C1400206A
:105A8000681400209148F0B50368914A9C8AA4B23A
:105A9000E1B211F0010F2ED0198821F40061090440
:105AA000090C1980198889B241F48061198000219C
:105AB0001170517899B1917811B9D178FF290ED12F
:105AC000012191701179022901BF198889B241F42D
:105AD00000611980517941F001011982E1E05179A9
:105AE00001F0FE011982D378FF2B00F0DA80784BA9
:105AF000FF211970D5E08E073AD5BFF35F8F147977
:105B0000E4B2012C13D1517889B1917879B1198817
:105B100021F480610904090C1980BFF35F8F198B90
:105B20001988947189B241F4007119801BE0198BB6
:105B3000BFF35F8F14796649022C0AD14C7844B1C7
:105B4000897831B1198821F480610904090C198020
:105B5000A1E014795E49032C05D14C781CB18978F9
:105B6000002940F09880998889B241F4806197E0DB
:105B70004D0756D5012191715178002937D0917880
:105B8000002934D011791C88022911781DD924F4F8
:105B900080642404240C1C801E8A9568CCB2F6B262
:105BA00049B26E54198889B241F4007119800168B4
:105BB000A31C13700B8A0134DBB264B22B558B88A3
:105BC0009BB243F480638B8026E0A4B244F400745B
:105BD0001C801D8A9668CCB2EDB249B275541B8AFE
:105BE000611C49B2DBB203347354147014E0917831
:105BF000374C09B9217B41B1198889B241F4007150
:105C0000198013780133137006E0198889B241F4C2
:105C1000807119800123A37001680B88DB05FCD417
:105C20003FE001F0400101F0FF05E1B114781F8A67
:105C30009668E5B2691C64B2FFB23755C9B21679ED
:105C4000117049B2CC1CA64201BF9C8824F4806428
:105C50002404240C08BF9C8013798B4221D11C4B57
:105C600002351D701DE027061BD511784CB2661C4D
:105C70000AD0156901312C5DC9B21C8214791170EA
:105C800049B28C420DD106E0D17815701982517855
:105C900009B9117929B9998821F480610904090C9D
:105CA0009980137992F9004001339C4208490CD144
:105CB00000238B708B7933B101688B8823F4407398
:105CC0001B041B0C8B8000231375F0BD00270020E4
:105CD000781200200A4B984205D10A4AD38A013330
:105CE0009BB2D38208E0084B984201BF054A138B50
:105CF00001339BB208BF13834FF0FF30704700BFE2
:105D00000030014078120020003800406B4B6C4A94
:105D10002DE9F04F5E89D4694FEA062AB4EB0A0AEE
:105D20009C884FF000054FEA04481C894FF0000B97
:105D3000A4FB0A6765EB0B0B04FB0B77F40944EA41
:105D4000476418EB04065C884FF000094FEAE7153A
:105D50004FEAC438DC8849EB050787B0CDE9046712
:105D6000A4FB0A6704FB0B77340A44EA076418EBC8
:105D700004064FEA27259C894FF0000949EB0507E7
:105D8000CDE90067AAFB046704FB0B77F40D44EA36
:105D9000472414F5FA664FEAE75545F10007B6F5D2
:105DA000FA6F77F10003CDE90267964666DADDE91E
:105DB0000489A4FB046704FB05F34FF0050C07EB13
:105DC0004307A6FB0C230CFB07335F104FEA320698
:105DD000B8EB06084FEA920646EA837669EB0709B4
:105DE0009F10DDE90023921B63EB0703CDE900233D
:105DF000DDE90267334A4FF0FF33964277EB030346
:105E0000CDE9048927DA40F6AC520023A4185D419D
:105E100004FB05F3A4FB04456FF0060205EB430504
:105E2000664202FB0566A4FB0223334418EB02061C
:105E300049EB0307CDE904670B26A4FB062306FB09
:105E40000533DDE900455B104FEA3202A41A65EB29
:105E50000305CDE90045DDE902450AFB0BF3AAFB8A
:105E60000AAB0BEB430B4FEADA7242EA4B02A41A7D
:105E70004FEAEB7365EB0305CDE90245DEF8204000
:105E8000009B019DA4FB032304FB05334FEA5258FA
:105E900048EAC3284FEA6359DDE90423B8EB02025C
:105EA00069EB03039946D30B43EA494300B103600E
:105EB00009B1029B0B6007B0BDE8F08F940500208C
:105EC0007812002024FAFFFF2DE9F04F87B06C4CC8
:105ED00002916C4922884E6A0546C2EB26135B4349
:105EE0005200C2EBE602B4F902601B135643B4F948
:105EF0000420B4F90A0053439B1303EBE62606EB98
:105F0000860380331B12B6F5FA384FEAE67704931E
:105F10008B6A47F1FF39A8FB08AB039308FB09F331
:105F2000B4F908200BEB430BE389A6610593D31763
:105F300008FB03F102FB0911A8FB02230B44C11764
:105F40001F030AFB01F300FB0B33AAFB000116033E
:105F5000194447EA1257020A42EA016292194FEACB
:105F60002123E6887B410032A2FB060143F5004372
:105F700006FB03114B100093CB170193DDE90023BF
:105F80001343B4F810E0B4F80CC06DD00FFA8EF0E3
:105F9000C1170AFB01F1AAFB002300FB0B11BDF99D
:105FA00014600B44F71708FB07F106FB0911A8FB67
:105FB00006670F4479047004801841EAD6315941CC
:105FC000039B0FFA8CF8C3F5801E7246D31700228C
:105FD00012184FEACE764FEAC3774FEAC8034B4117
:105FE00047EA5E07B61A67EB030740F63543A6FBA0
:105FF000030103FB0711DDE9002310F053FBB4F9A3
:1060000016204E1302FB06FE470B47EAC147D31783
:1060100007FB03EEA2FB07235643734407FB03660B
:10602000A2FB07233344560E46EAC3168219B4F97D
:1060300014604FEA636741EB07037143F71700FBF6
:106040000717A6FB00013944C60C46EA41369219EF
:106050004FEAE1474FEA1221B4F912207B4141EAAD
:10606000036113010B4400E000230DB11B0A2B60F8
:10607000029B13B11A46049B136007B0BDE8F08F72
:10608000D005002078120020704770472DE9F041BC
:10609000324C334D6289AB8DB4F904809A1A23894E
:1060A000B4F902E05A43B4F91230D613B4F914200B
:1060B000DB02324493FBF2F232440A26E261564399
:1060C000A2F57A6202FB02F3B4F90EC002FB0EFEE7
:1060D00002FB08F2B4F90C801B130CFB03FC03FB5E
:1060E00008F31B1403EB62320232E388921002F5CC
:1060F000004253434CF25032B4F920704FEAEE2E76
:10610000B4F900400EEBEC2C0CEB8404BC402D6B7E
:106110000234A5EBA4043A4162434FEAD3384EBFA0
:10612000B2FBF8F35400B4FBF8F340F6DE3448BF9A
:106130005B001A12524362430A4C08365C43241433
:1061400004EB224202F6CF62361103EB221300B1B8
:10615000036001B10E60BDE8F08100BFA80500201A
:106160007812002043E3FFFF064B93F8342002F03F
:10617000FF012AB101220270002283F83420704707
:10618000017070477812002037B5104B04465D68E7
:10619000187806216A46A847A8B19DF800209DF806
:1061A0000130012043EA022323809DF802209DF85C
:1061B000033043EA022363809DF804209DF80530F4
:1061C00043EA0223A38003B030BD00BF8405002052
:1061D00013B5104B04465B683B2006216A4698477E
:1061E000A8B19DF800209DF80130012043EA022368
:1061F00023809DF802209DF8033043EA0223638048
:106200009DF804209DF8053043EA0223A38002B0E4
:1062100010BD00BF8405002010B5224C2368998A68
:1062200089B211F4706F1EBF1F4A012082F8350039
:1062300011F4E06F2BD01A8B9A88890522F48062C2
:106240004FEA02424FEA12429A8020D41A889205FD
:106250001DD41A88D0050FD51A88D105FCD41A8808
:1062600092B242F400721A801A889205FCD40F4B45
:1062700018780CF0A3F80AE01A8892B242F400727F
:106280001A809A8822F440721204120C9A802268B2
:10629000938A23F470631B041B0C9382024B00222D
:1062A0001A7510BD00270020781200200427002056
:1062B000054A08B5138801339BB21380034B187845
:1062C0000CF07CF8002008BDBE130020042700203D
:1062D000F0B5334D85B095F83630002B5ED1314C9A
:1062E0002368002B5AD01A682F4E12B1B1690A43A5
:1062F000B2619A889868ADF8002002228DF80320D8
:10630000694604228DF802200BF000FFB369216872
:1063100043F00103B3610B7D0F2003F0030203F090
:10632000FC0303F1804303F580339F6892009040A3
:1063300027EA00000E7B9860986806FA02F2024392
:106340009A601A4B4A7D596819B100200CF008FB7D
:1063500002E017491A7059602368164A1B69012622
:106360005361029308230DEB030000278DF80D30D5
:106370008DF80C708DF80E600DF078FF236801A881
:106380005B7D8DF806708DF8043003238DF80530A1
:106390008DF807600DF04CFF85F8366005B0F0BD54
:1063A00078120020900500200010024008270020ED
:1063B000CD6300080004014008B5FFF789FF024BD8
:1063C0004FF480521A8008BD080000200C4B10B515
:1063D0001B681A690B4B1968586910420ED011429C
:1063E0000CD0094C5A61012384F834300CF010FAB7
:1063F000A36B064AC31AE3631380A06310BD00BFFA
:10640000900500200004014078120020B6140020FE
:1064100010B51E4C4000C0B2A36023611C4B6071DC
:10642000E1700120002121736070227120751868CD
:1064300084F8351040B383889B0515D40388D905AB
:106440000DD447F230530288920502D5013BFAD1B0
:1064500012E08BB103889BB243F48073038083887E
:106460009BB243F44073838047F23053227D12B1D4
:10647000013BFBD100E013B9BDE8104018E7034B26
:1064800093F8350080F0010010BD00BF78120020A5
:106490000027002007B5002101AB03227720FFF77A
:1064A000B7FF9DF805309DF804001B0243EA004346
:1064B0009DF80600184303B05DF804FB08B5FFF72C
:1064C000E9FF014B186208BD7812002008B5FFF7FC
:1064D000E1FF014BD86108BD7812002007B5F72114
:1064E0006B4606227620FFF793FF9DF800309DF85B
:1064F00001101B0343EA01139DF80210094A43EA05
:10650000111393629DF803309DF804101B0343EAB6
:1065100001139DF8051043EA1113536203B05DF8AF
:1065200004FB00BF7812002007B5F62101AB03225F
:106530007720FFF76DFF9DF805309DF804201B02C2
:1065400043EA02439DF806201343054AB2F920208E
:10655000C2F10802D340034A136303B05DF804FBA1
:10656000A80500207812002007B5F62101AB022211
:106570007720FFF74DFF9DF804209DF8053043EA92
:106580000223024A938503B05DF804FB78120020D1
:1065900030B505460C46134629462246BDE8304034
:1065A000682035E713B5204B400002ACC0B25871EB
:1065B00004F8012DD970012200211A7359701A7143
:1065C0001A751A4A1C6110689C6083F8351040B334
:1065D0008288920515D40288D4050DD447F2305232
:1065E0000188890502D5013AFAD112E08AB1028800
:1065F00092B242F480720280828892B242F4407277
:10660000828047F23052197D11B1013AFBD100E08E
:1066100012B9FFF74DFE04E0034B93F8350080F00C
:10662000010002B010BD00BF78120020002700203A
:10663000772048210122B5E7772058210122B1E7D0
:106640007620F4213122ADE7044B772093F8202007
:10665000F4219201343202F0FC02A3E7A8050020E5
:106660007720F4212E229DE703460A46682019462A
:1066700098E7FFF707BACFE5FFF704BACCE570B5A6
:1066800084894FF47A74FBB112B11578013207E0B6
:10669000FF2505E04FF6FF76013CA4B2B4420DD0D1
:1066A0000689B607F6D5ADB285810589ED070DD40B
:1066B0004FF6FF75013CA4B2AC42F6D1FFF70AFBDE
:1066C000003018BF012070BD012070BD8589ADB2BA
:1066D00009B10D700131013BD5E708B540F2E9334E
:1066E0000289920704D4013B9BB2002BF8D10AE047
:1066F00040F2E93389B281810289D20706D4013B95
:106700009BB2002BF8D1FFF7E5FA00E08089C0B218
:1067100008BD2DE9F04190460F46094C094E102561
:1067200040F0800165613046FFF7D7FF30464146B3
:1067300000223B46FFF7A3FF25610120BDE8F08161
:106740000008014000300140F8B503460F46074CF1
:10675000074E1025194665613046FFF7BEFF3046EB
:106760003946FFF7BAFF25610120F8BD0008014056
:1067700000300140F7B5574D0646FFF7A9FD95F8E3
:106780004070002F71D1544C802123886B2023F05E
:1067900040031B041B0C2380238823F038031B04B5
:1067A0001B0C43F03003238023889BB243F040034B
:1067B0002380FFF7C9FF96200CF051F803216820D1
:1067C000FFF7C2FF96200CF04AF803216B20FFF779
:1067D000BBFF0F200CF038F810216A20FFF7B4FF40
:1067E0000F200CF031F839466C20FFF7ADFF0F2079
:1067F0000CF02AF8394B19201978FFF7A5FF0F2064
:106800000CF022F818211B20FFF79EFF0F200CF040
:106810001BF810211C20FFF797FF0F200CF014F835
:1068200010213720FFF790FF0F200CF00DF8012109
:106830003820FFF789FF0F200CF006F8238801208D
:1068400023F040031B041B0C2380238823F0380310
:106850001B041B0C238023889BB243F0400323803E
:106860000BF0F2FF012385F84030FFF731FD1A4AA3
:106870000023EB821388314623F040031B041B0CDA
:10688000138013881A2023F038031B041B0C43F0D9
:106890003003138013889BB243F040031380FFF74B
:1068A00053FF01200BF0D0FF6846FFF76DFC9DF908
:1068B0000230013303D19DF90030013302D0EB8A5D
:1068C0009BB223B100230620EB820CF049F803B001
:1068D000F0BD00BF7812002000300140EC05002020
:1068E0002DE9F04FB04B8DB01C780093002C00F0D8
:1068F000AF80AE4F3B68002B01F0998038680CF0F8
:106900007BF8002801F09380A84BA94C18680CF084
:1069100070F8092801D03F2850D14FF000094D46AA
:10692000D4F80080A34EB8F1000F05D0A24831681A
:10693000424614F073F810B9B14605B935469F4B7D
:1069400008369E42EFD3C5B1D5F800E0D9F800C0B3
:1069500023681EF803601CF80300B0420DD15A1CD6
:10696000954938B92D2B05D8914E32602026CE544A
:10697000885402E0CE542260EAE723680BB14D450B
:1069800011D08F480DF0ECF84D4507D855F8080B9D
:106990000DF0E6F809200DF0DBF8F5E789480DF079
:1069A000DFF84FF0000823689845A7D2824B13F810
:1069B00008000DF0CDF808F10108F4E72368002B7A
:1069C00040F0A187042840F0FF877B4808F03EFF95
:1069D00001F02DB8DBF80000DFF800920CF00CF8A5
:1069E00028B3D9F800000CF004F8D8F8003082463B
:1069F00093F84820002A39D1242870D1012283F845
:106A00004820D8F80030DFF8D09193F848A0BAF1C8
:106A1000060FDFD193F8490001F00EF8002800F0CE
:106A200086800CF0E5FF2B68002283F84820664B37
:106A30001B794BB1305903F0A9F90CF065F905F059
:106A400045FB624A624BDA604C34982C00F0EF87C9
:106A5000604EA31993F84A20012AF5D15E4D5F4F8D
:106A60002B60A359A8463B60BB46B3E7012A04D17B
:106A70004D2814BF00220222C1E7022A04D13C287B
:106A800014BF00220322BAE7032A0AD140284FF09C
:106A900000029FBF1A71DA715871987198BF042271
:106AA000ADE7042A08D19A7983F8490080EA020AFE
:106AB00083F806A00522A2E7052AA2D159791A79FE
:106AC0009142997906D941409971511C1971134429
:106AD000187296E781420CBF062200228FE7404BD6
:106AE0001A7852078DD42328D9F8002012D10193A7
:106AF000009B012119702D493A480A6032490A6009
:106B00000DF02EF82F480DF02BF8019B1A7842F06B
:106B100002021A70344B1B681B78534501BF334A7D
:106B2000334B1A60294A04BF294BDA6069E7D9F868
:106B3000002092F849304C2B00F0C68400F2BB8054
:106B4000352B00F0AB8264D82B2B00F0958421D834
:106B5000252B00F0698404D8232B00F0658200F017
:106B6000CEBE272B00F06884292B40F0C8860CF09D
:106B70001DFF204FA7F880010CF018FFA7F8820135
:106B80000CF00AFF87F884010CF010FFA7F88601CB
:106B900000F0B0BE2F2B00F010852DD82D2B00F06B
:106BA000708400F0ACBE00BFBA3500202C29002054
:106BB000042300207CB70108D42200206CB801080F
:106BC00075D001087AD00108E41200200400FA050B
:106BD00000ED00E0D42900202429002028290020ED
:106BE000B8350020AAD001085C320020EFBEADDE2F
:106BF000F04F00206C2A0020312B00F0F184332B61
:106C000040F07D860CF0C8FEC84B83F8920100F07E
:106C100071BE412B00F0928419D8392B00F01A84F0
:106C200004D8372B00F0958400F069BE3C2B00F0AF
:106C3000DA803E2B40F063860CF0AEFEBB4F87F847
:106C4000E2010CF0A9FE87F8E10100F053BE442BED
:106C500000F0FB8427D8432B40F051860CF09CFEBB
:106C6000B24F0023BB6078710CF0AAFEBB681843DA
:106C7000B8600CF091FE87F890010CF097FEA7F831
:106C80005A010CF093FEA7F85C010CF08FFEA7F8F8
:106C90005E010CF08BFEA7F880010CF087FEA7F8D0
:106CA000820100F027BE482B00F05B834A2B00F0E6
:106CB000218600F024BED12B00F07A8320D8CC2B83
:106CC00000F014820FD8C82B60D004D84E2B00F0EF
:106CD000098400F014BEC92B00F04683CA2B00F0D3
:106CE0009A8000F00CBECE2B00F02C83C0F02083E5
:106CF000CF2B00F04582D02B00F0F78200F0FFBDD3
:106D0000D82B00F02B810AD8D32B39D024D3D42B05
:106D100000F07B82D62B40F0F28500276CE2F22B4C
:106D200000F0BA8210D8EF2B40F0E985804FD7F8F9
:106D300000800CF03BFEA8F85A003F680CF036FECD
:106D4000A7F8580000F0D6BDF32B00F09F84FA2B73
:106D500000F0028300F0D3BD764B1B7803F00403F0
:106D600003F0FF07002B40F0C5850CF015FE6F4BBC
:106D7000022883F8B00740F2BF8283F8B077BBE205
:106D80000CF014FE6C4B188000F0B4BD57797F08EE
:106D9000122F03D90DF070FC00F0ACBD4FF00008CD
:106DA000B84507D20CF002FE03AB23F8180008F137
:106DB0000108F5E73A460023BB4207DA03A931F898
:106DC00013005E4921F813000133F5E7122A05D0BC
:106DD0005A4B002123F812100132F7E7584B0122D9
:106DE0001A7000F087BD524FD7F800800CF0D4FD28
:106DF00018B10228A8BF022000E0012088F8000096
:106E00003B681B78022B18BF4E4A4F4B08BF4F4AB6
:106E10001A6000F06FBD464F4FF000083B681B78CA
:106E2000022B67D1D7F800900CF0B6FD0FF0D6F921
:106E300047490FF0DFFA08F1080A49F82A00D7F8A5
:106E400000900CF0A9FD08F10A0309EB83090FF08B
:106E5000C5F940490FF0CEFAC9F80400D7F8009000
:106E60000CF09AFD0FF0BAF93B490FF0C3FA08F1A4
:106E70000E0A08F10108B8F1030F49F82A00D1D130
:106E8000B8F1070FD7F800901AD10CF085FD0FF07C
:106E9000A5F92F490FF0AEFAC9F84400D7F80090D1
:106EA0000CF07AFD0FF09AF929490FF0A3FAC9F80E
:106EB0004800D7F800900CF06FFD89F84C0012E004
:106EC0000CF06AFDC14489F80100D7F800900CF07D
:106ED00063FDC14489F80B00D7F800900CF05CFD0D
:106EE000C14489F8150008F10108B8F10A0FC7D1AB
:106EF00000F000BDD7F800900CF04EFDC14489F8B9
:106F00000100D7F800900CF047FDC14489F80B0050
:106F1000D7F800900CF040FDC14408F10108B8F129
:106F20000A0F89F81500E5D100F0E4BC6C2A0020B6
:106F30000C140020B8350020E41100209434002007
:106F4000DD280020B147010894030020DD4A010834
:106F5000000020410000C84200007A440746DFF8E4
:106F6000BC8307F1080AD8F800900CF01FFD0FF061
:106F700035F9E4490FF03EFA49F82A00D8F80090B4
:106F80000CF014FD07F10A0309EB83090FF026F951
:106F9000DC490FF02FFAC9F80400D8F800900CF083
:106FA00005FD0FF01BF9D7490FF024FA07F10E0A7F
:106FB0000137032F49F82A00D1D1072FD8F80090C4
:106FC0001AD10CF0F3FC0FF009F9CE490FF012FAC8
:106FD000C9F84400D8F800900CF0E8FC0FF0FEF877
:106FE000C8490FF007FAC9F84800D8F800900CF02B
:106FF000DDFC89F84C0012E00CF0D8FCB94489F8AB
:107000000100D8F800900CF0D1FCB94489F80B00CD
:10701000D8F800900CF0CAFCB94489F81500013783
:107020000A2FCAD100F066BC0CF0B6FC1328074644
:107030003FF6B0AEDFF8E482D8F800900CF0ACFC7C
:107040000023B1490C2202FB0312117A814221D1A3
:10705000137809EB870787F879300CF09DFC87F8E7
:107060007A000CF099FC87F87B000CF095FCA74A9D
:10707000A74B87F87C001A60D8F80000A54B0021C8
:10708000186079300BF070FBA34B80F00100187092
:1070900000F030BC01331D2BD3D17BE60CF07CFC1F
:1070A0000B2807463FF676AE9C4BD3F800800CF0D9
:1070B00073FC03283FF66EAE0AFB078A8AF8CE00FF
:1070C0000CF06AFC8AF8C9000CF066FC8AF8CA0069
:1070D0000CF062FC8AF8CB000CF05EFC8AF8CC0065
:1070E0000CF05AFC8AF8CD0000F004BC5379092B4F
:1070F0007FF650AE8A4FD7F800800CF04DFC88F830
:107100000000D7F800800CF047FC88F801000CF074
:1071100043FC3B686428A8BF642018710CF03CFC59
:107120003B686428A8BF642058710CF035FC3B68AC
:10713000FF28A8BFFF2098710CF02EFCD7F8008024
:10714000642828BF642088F807000CF025FC88F824
:107150000200D7F800800CF01FFC88F80300D7F875
:1071600000800CF023FCD9F80030A8F80A005B7905
:107170000A2B40F2BF833F680CF00EFC3872B9E373
:107180000CF014FC6FF4AF67C3199BB2654FC62BAC
:1071900098BFA7F896010CF009FCA7F840010CF085
:1071A00005FCA7F842010CF001FCA7F844010CF023
:1071B000FDFBA7F8DA010CF0EFFB87F8EF010CF00C
:1071C000EBFB0CF0E9FB87F8F0010CF0E5FB87F82E
:1071D00085010CF0E1FB87F892010CF0DDFB4F4BD1
:1071E000D3F800800CF0E2FB00EB80004000A8F830
:1071F00056000CF0D1FB30E10CF0D8FB4A4B23F8E1
:1072000017000137082FF7D174E353790F2B7FF460
:10721000C1AD0CF0C1FB072807463FF6BBADDFF858
:10722000FC80D8F800900CF0C1FB0E235F43B944FA
:10723000A9F81901D8F800900CF0B8FBB944A9F8E6
:107240001B01D8F800900CF0B1FBB944A9F81D015E
:10725000D8F800900CF0A0FBB94489F81F01D8F8C9
:1072600000900CF099FBB94489F82001D8F80090FF
:107270000CF092FBB94489F82101D8F800900CF089
:107280008BFBB94489F82201D8F800800CF098FBF8
:107290004744C7F823012DE30CF07EFB0F28074677
:1072A0003FF678AD0CF078FB1E4BC7EBC7071F44C9
:1072B00087F8D0000CF070FB87F8D1000CF06CFB65
:1072C00087F8D2000CF068FB87F8D3000CF064FB61
:1072D00087F8D4000CF060FB87F8D5000CF05CFB5D
:1072E00087F8D6000BF050FD04E3104B1B785807CD
:1072F00000F100830AF004FA04F012FF04F0B6FF74
:10730000F8E200BF00007A4424AF0108AC2B002053
:10731000DC110020E0110020020000200C140020ED
:10732000441400206C2A00200A290020B8350020CF
:10733000C84B1B78590700F1DD82C74B4FF4C87268
:107340001A80D7E2C34B1B785A0700F1D382C34A95
:10735000137843F0040329E0BE4B1B785B07CBD5C1
:10736000CDE207F043FDC5E20CF016FBBB4B1A78EB
:1073700010B142F0020201E022F002021A700CF099
:107380000BFBB74BB74F18700CF01AFB38600CF0C2
:1073900017FB78600CF00AFBB34B18800CF006FB6F
:1073A000B24BB34A1880137843F002031370A1E282
:1073B0000CF0F2FA82460CF003FB81460CF000FB65
:1073C00080460CF0FDFA07460CF0F0FA0CF0EEFAED
:1073D0000CF0E2FABAF1000F12D1A64B1020C3F85C
:1073E0000090C3F8048004F049FE9C4A137843F0EF
:1073F00001031370002F00F07D829F4B1F6079E224
:10740000BAF1100F40F076829C4BC3F80090C3F89D
:1074100004800FB1984B1F609848994B0222011DC0
:107420001A7007F0E1FA65E2964FB8600CF0C8FAFE
:10743000BB681843B8605DE20CF0B8FA914FA7F84A
:107440005A010CF0B3FAA7F85C010CF0AFFAA7F8F8
:107450005E014FE20CF0A0FA8A4F87F87A010CF037
:107460009BFA87F87E010CF097FA87F87D010CF003
:1074700093FA87F87F013DE20CF08EFA814B587148
:1074800038E20CF089FA7F4F87F890010CF08EFA01
:10749000A7F89A010CF08AFAA7F896010CF086FA80
:1074A000A7F898010CF078FA2B6887F891015B79BE
:1074B000082B40F21F820CF079FAA7F89E010CF01D
:1074C00075FAA7F8A00115E20CF066FA6D4F87F87F
:1074D000D8010CF061FA87F8D9010CF067FAA7F827
:1074E000DA0107E257790323B7FBF3F7122F3FF6D0
:1074F00051ACDFF890814FF00009B94580F0FA8176
:107500000CF04AFA88F8A2010CF050FA40F2ED2390
:10751000984205DD40F6CA039842A8BF184601E02C
:1075200040F2EE20A0F2EE20192390FBF3F009F1D7
:10753000010988F8A30108F10208DEE707460CF00C
:107540002BFA504B3B440137082F83F88801F6D1C2
:10755000D0E153790727B3FBF7F7C7EBC7029B1AB4
:1075600013F0FF0F7FF416ACFFB2013FFFB2FF2F05
:1075700000F0C0810CF010FA5FFA80F94FFA89F040
:1075800002F00AFD804600283FF404AC80F8009029
:107590000CF00CFAA8F802000CF0FEF988F80400D0
:1075A0000CF0FAF988F805000CF0F6F988F80700F5
:1075B0000CF0F2F988F80600D7E7324F07F14008DF
:1075C0000CF0F4F9A7F8A8020CF0E6F987F8AA0283
:1075D0000CF0E2F9043787F8A7024745F0D189E1BA
:1075E0000CF0DAF91F2807463FF6D4AB2B685B791D
:1075F000082B7FF4CFAB0CF0D9F9DFF888908A37ED
:1076000009EB870800F03F00A8F802000CF0CEF963
:10761000B8F80230800100F4FE501843A8F80200C8
:107620000CF0BAF9000109F827000CF0B5F919F8C7
:10763000273000F00F00184309F827000CF0ACF9D0
:1076400088F8010006F014FA54E10F4B01221A7178
:1076500050E100BFB8350020A011002048140020E0
:10766000491400204C14002054140020561400200B
:107670005E140020601400207014002068140020A4
:10768000E81100206C2A0020E41200200CF084F99C
:10769000FF288146DFF8448366D1002708F10800FF
:1076A0003946602288F8057013F070F98DF80B7078
:1076B0009DF80B3098F86A20DFF820939A424AD957
:1076C0009DF80B3009EBC30393F86D30DF073BD512
:1076D0009DF80B3009EBC30393F86C20BD4B33F9D5
:1076E0001230002B30DD9DF80B3099F8057009EB56
:1076F000C3031B6F4FEAC70E58689DF80B3009EBA8
:107700000E0109EBC309D9F8703088601A89CA8163
:1077100092B2002101238B40134003D10131102983
:10772000F8D100E00B4608EB0E018B8148238DF861
:107730000E3003A901230137ADF80C208DF80F306E
:107740000AF0E4FC88F805709DF80B300133DBB2D9
:107750008DF80B30ACE701200CF06EF999F80500BC
:107760000CF037F9FFF75DB998F805309842BFF48F
:1077700011AB00200CF060F90CF03AF92B68186896
:1077800002F004FB38680CF0E7F80BF083F872B6EF
:10779000914F4FF400634FF4806A7B614FF0010B0F
:1077A000C7F814A03846ADF80C3003A948238DF86B
:1077B0000E308DF80FB04FEAC9090AF0A7FC10236C
:1077C000384603A98DF80E308DF80FB0ADF80CA037
:1077D0000AF09CFC08EB09018B89D1F808C0D80895
:1077E0000CEB8002C8F8CC205CF8202003F00703E3
:1077F000C8F8D0209B00C8F8D4200F229A40D2436A
:10780000D8F8D4E00BFA03FB02EA0E0EC8F8D4E075
:10781000D8F8D0E002EA0E02C8F8D020D8F8D42078
:107820004FF0080E0EFA03FE4EEA0202C8F8D4200A
:10783000D8F8D0204BEA0202C8F8D020D8F8D030CF
:10784000CA894CF820308B681A61C7F810A0BB6851
:107850001805FCD4614B4FF48067D3F8D010D3F8EF
:10786000CC209846116003EB090290685A49D289EE
:1078700042614F6108270F6140F60557DFF858A1B4
:10788000DAF80830190503D4002FF7D0013FF5E7E7
:107890004823026103A98DF80E300123ADF80C20B6
:1078A0008DF80F300AF032FC9FB14B4B9A681205ED
:1078B000D0D508EB09018A68C989926811424FF452
:1078C00080614FF0080215BF196159611A615A6150
:1078D000EBE74FF48063CAF810300823CAF8103081
:1078E00062B60A200AF0BBFF0CF099FD2B68F32268
:1078F00083F8492000200CF09FF8FFF792B80CF0B5
:10790000BBFEFFF78EB80C2803D135480CF028F9E0
:107910004CE00A2801D00D284AD1324D32480CF0F3
:107920001FF92846232113F064F808B1401B20609A
:1079300023688BB35A1EA95C202901D11346F8E7AE
:10794000284A00212360D154284B294DD3F80090B8
:10795000D5F800A0DFF88C80504613F057F80646A3
:1079600051463246404613F059F8224A28B918F8D1
:1079700006304B445B78590703D008359542E7D36E
:1079800006E0954204D2701C6B684044984702E0C0
:1079900019480CF0E5F8002312480021302223603A
:1079A00012F0F4FF009B1B78002B40D0134807E037
:1079B0007F2827D10B4A013B002111482360D15475
:1079C0000CF0CEF8FEF79ABF0C289ED07F281CD171
:1079D000FEF794BF10140020000C0140E4120020B8
:1079E0007FD00108D42200206CDB0108A403002012
:1079F0007CB701086CB801088AD001087AD0010868
:107A0000A6D001082F2B3EF679AFA0F12002D2B20A
:107A10005E2A3EF673AF13B920283EF46FAF5A1CAE
:107A20002260044AD0540CF093F8FEF767BF0DB003
:107A3000BDE8F08FD42200202DE9F04F4B28A1B0F3
:107A4000044600F0398600F2B480302800F0BE868B
:107A500051D8222800F0838423D8032800F06281C3
:107A600014D8012800F05281022840F01A8704201F
:107A70000BF0E2FF42200BF0ACFF54200BF0A9FF0B
:107A800046200BF0A6FF4C2000F04ABE042800F070
:107A90005481052840F005871A200BF0CDFF002403
:107AA0005DE1282800F0D68515D8242800F0BD8592
:107AB000262840F0F686B64C06200BF0BDFFB4F841
:107AC0005A010BF0BCFFB4F85C010BF0B8FFB4F83E
:107AD0005E0100F036BE2C2800F0CF852E2800F085
:107AE0004D862A2840F0DD8601200BF0A5FFA84B2B
:107AF000587900F015BE3D2800F0F8821ED83628CF
:107B000000F022860BD8322800F00486342840F09A
:107B1000C88648200BF090FF002500F042BC3A28B0
:107B200000F0BC823B2800F01384382840F0B9866E
:107B300004200BF081FF964C00F07DBD452800F03D
:107B40009D8627D8402800F0EE85422840F0A9867F
:107B50008F4C10200BF070FF60790BF03AFFA0689B
:107B60000BF076FF94F890010BF033FFB4F85A0154
:107B70000BF065FFB4F85C010BF061FFB4F85E0137
:107B80000BF05DFFB4F880010BF059FFB4F88201EF
:107B900000F0D7BD472800F04F86C0F03C8649284A
:107BA00040F07F8602200BF047FF7A4B188800F0E8
:107BB000C8BD702800F0E8825AD8692800F04982D0
:107BC0002AD8652800F0FA8015D84D2800F0838562
:107BD000642840F0668607200BF02EFFE7200BF0AC
:107BE000F8FE6B4B58790BF0F4FE00200BF0F1FE21
:107BF000042000F052BE672800F0AE8100F21C8223
:107C000012200BF019FF644B00251B88B3F5806F21
:107C10008CBF0826012681E16C2800F02D8217D840
:107C20006A2800F083846B2840F03B865B4C05207B
:107C30000BF002FFB4F89E000BF001FFB4F8A000B7
:107C40000BF0FDFE94F8A20000F0010000F068BD0A
:107C50006E28524C00F0268200F2668206200BF05D
:107C6000EBFE606F0BF0F4FEB4F8780000F069BD35
:107C7000782800F07E8119D8742800F0B3830BD8DF
:107C8000722800F01384732840F00B8608200BF054
:107C9000D3FE012400F043BC762800F0688400F293
:107CA000E5832F200BF0C8FE3D4C49E3A42800F0EB
:107CB000888414D87B2800F0E982A02840F0F18560
:107CC0000C200BF0B9FE374B18680BF0C1FE364B99
:107CD00018680BF0BDFE354B186800F0DEBDF128CA
:107CE00000F08381FE2800F09384F02840F0D985CD
:107CF0002A4C04200BF0A0FE236DB3F85A000BF0C1
:107D00009EFE236DB3F8580000F01BBD03200BF05E
:107D100093FE00200BF05DFE20460BF05AFE0D2076
:107D200000F0FEBC0BF088FE02200BF052FE204655
:107D30000BF04FFE052000F0F3BC06200BF07CFE9C
:107D400043200BF046FE43200BF043FE33200BF0A4
:107D500040FE44200BF03DFE002000F0F2BC144B2E
:107D6000185D01340BF035FE0B2CF8D10024114BBB
:107D7000185D01340BF02DFE082CF8D100240E4BB9
:107D8000185D01340BF025FE072CF8D100F087BDFB
:107D90006C2A00202035002008000020BC130020A1
:107DA000F3AE0108E8F7FF1FECF7FF1FF0F7FF1F26
:107DB000B7CE0108C3CE01089BCE0108D14C0B20E1
:107DC0000BF03AFE20880BF03AFE608880B20BF090
:107DD00036FE6368C3F3C000C3F38002800040EA4C
:107DE0004200C3F340021043C3F3401240EAC20012
:107DF00003F0100318430BF022FE2189E36801F021
:107E0000080203F4475A4AEA020A03F480424AEAA3
:107E1000020A03F400424AEA020A03F480324AEA00
:107E2000020A03F400324AEA020A03F480224AEA10
:107E3000020A03F400224AEA020A03F480124AEA20
:107E4000020AB14A03F0007B12784AEA0B0A03F0F7
:107E5000006311F0010FC2F380024AEA030314BF6A
:107E60004FF002094FF00009134311F0020F14BF45
:107E70004FF004084FF0000843EA090911F0040F1D
:107E800014BF4FF0100C4FF0000C49EA080811F035
:107E9000400F14BF4FF0200E4FF0000E48EA0C0CBC
:107EA00011F0100F14BF4FF4007700274CEA0E0EAC
:107EB00011F0200F14BF4FF4806600264EEA07072A
:107EC00011F4807F14BF4FF4006500253E4311F488
:107ED000007F14BF4FF400100020354311F4806F71
:107EE00040EA050014BF4FF08061002101430020EB
:107EF0000346247CA3420AD2844A9D5C012202FAF2
:107F000005F50D421CBF9A4010430133F2E70BF018
:107F10009FFD7F4B93F8B00700F002BC794C04F151
:107F20002E0333F91500013590FBF6F080B20BF00B
:107F300086FD032DF2D1A08E0BF081FDE08E0BF0BB
:107F40007EFD208F0BF07BFD608F0BF078FDA08F06
:107F50000BF075FDE08FF4E310200BF06DFD0024B5
:107F60006C4B185D01340BF034FD102CF8D100F08F
:107F700096BC70200BF060FD00260E247443614D0A
:107F800001362B6D2344B3F819010BF058FD2B6D0E
:107F90002344B3F81B010BF052FD2B6D2344B3F8BF
:107FA0001D010BF04CFD2B6D234493F81F010BF0CA
:107FB00010FD2B6D234493F820010BF00AFD2B6D6F
:107FC000234493F821010BF004FD2B6D234493F817
:107FD00022010BF0FEFC2B6D1C44D4F823010BF0A6
:107FE00037FD082EC9D100F05ABC70200BF024FDDB
:107FF000474C04F1700594F8D0000BF0EAFC94F8BB
:10800000D1000BF0E6FC94F8D2000BF0E2FC94F8FF
:10801000D3000BF0DEFC94F8D4000BF0DAFC94F8FB
:10802000D5000BF0D6FC073494F8CF000BF0D1FC50
:10803000AC42E0D100F033BC10200BF0FDFC00247A
:10804000354B185D01340BF0C4FC102CF8D100F056
:1080500026BC324D00242878400000F0FE000BF0D2
:10806000EBFC2B789C4280F01A842D4B33F81400E3
:108070000BF0E5FC0134F4E7224C06200BF0DCFCAD
:10808000B4F86C000BF0DBFCB4F86E000BF0D7FC1E
:10809000B4F970300A2093FBF0F025E004200BF0D7
:1080A000CBFCF9E307200BF0C7FC1E4B1888FF2818
:1080B000A8BFFF20C0B20BF08CFCE06F80F3100073
:1080C00080B20BF0BCFCB4F880000BF0B8FC104B95
:1080D000D4F8840093F8853123B10A23584380F300
:1080E000100001E000F30F0080B22AE3084C0220E8
:1080F0000BF0A2FC94F8E2010BF06BFC94F8E101A8
:108100000EE300BFBC130020B8350020CD130020C3
:108110006C2A0020FC130020101400205432002090
:1081200094320020F01700200B200BF085FCD4F8CF
:108130008830002618780BF04CFCD4F8883058783A
:108140000BF047FCD4F88830C34D3344187901361E
:108150000BF03FFC032EF5D1D5F88830D8790BF021
:1081600038FCD5F8883098780BF033FCD5F8883097
:10817000D8780BF02EFCD5F8883058890BF05FFCCE
:10818000D5F88830187ACBE2B34C1E200BF054FCA3
:10819000236D00251B78022B65D1236D05F10802A4
:1081A00053F82200AD490EF071F80FF007FA80F392
:1081B0000800C0B20BF00DFC236DA94903EB850349
:1081C000D86A0EF063F80FF0F9F980F30800C0B236
:1081D0000BF0FFFB236D05F10E0253F82200A149BD
:1081E0000EF054F80FF0EAF980F30800C0B2013540
:1081F0000BF0EFFB032DD0D1072D236D21D1586C4F
:1082000096490EF043F80FF0D9F980F30800C0B298
:108210000BF0DFFB236D9149986C0EF037F80FF0EF
:10822000CDF980F30800C0B20BF0D3FB236D93F8B7
:108230004C000DF0D3FF0FF0C1F980F30800C0B27D
:108240000BE02B4458780BF0C4FB236D2B44D87AF9
:108250000BF0BFFB236D2B44587D01350BF0B9FBB0
:108260000A2DC9D11BE3236D2B4458780BF0B1FBC9
:10827000236D2B44D87A0BF0ACFB236D2B44587D37
:1082800001350BF0A6FB0A2DEDD108E33C200BF0E5
:10829000D3FB0024704D04F108022B6D714953F893
:1082A00022000DF0F3FF0FF089F980B20BF0C7FB4D
:1082B0002B6D6C4903EB8403D86A0DF0E7FF0FF0D8
:1082C0007DF980B20BF0BBFB2B6D04F10E0253F86D
:1082D000220064490DF0DAFF0FF070F9013480B22A
:1082E0000BF0ADFB032CD5D1072C2B6D16D1586CA0
:1082F0005C490DF0CBFF0FF061F980B20BF09FFBF2
:108300002B6D5849986C0DF0C1FF0FF057F980B2F2
:108310000BF095FB2B6D93F84C000BE02344587841
:108320000BF08DFB2B6D2344D87A0BF088FB2B6D63
:108330002344587D01340BF082FB0A2CD4D1AEE2E9
:1083400014F8010F002800F0AA820BF042FBF7E7B7
:1083500001200BF071FB404B1B6D1878E0E15020C1
:108360000BF06AFB00253C4B0C211C6D3E4B04EBD3
:10837000850494F87920013501FB023393F8380025
:108380000BF027FB94F87A000BF023FB94F87B00AA
:108390000BF01FFB94F87C000BF01BFB142DE2D1BB
:1083A0007DE22D4B1C6D062303FB054494F8CE00A3
:1083B0000BF00FFB94F8C9000BF00BFB94F8CA000C
:1083C0000BF007FB94F8CB000BF003FB94F8CC0008
:1083D0000BF0FFFA013594F8CD000BF0FAFA0C2DF2
:1083E000DFD15CE24FF00008012600271A4B1A7C0F
:1083F000974227DA1133FA5C00240C2363431A4DA9
:1084000005F13001595C914207D12B44586B12F0B1
:10841000FDFA82462EB9B14605E001341D2CECD19F
:108420000EE080440CE0D1450ADA0C2303FB045330
:108430005B6B13F809000BF0CCFA09F10109F2E7C4
:108440000137D3E7002E00F02A825FFA88F00BF0A4
:10845000F3FA0026C9E700BFBC130020000020414A
:108460000000C84200007A44F4AE0108CE4D00245A
:10847000287C0BF0E1FA2B7C9C4280F01082CB4BE5
:108480000021E65C0C2202FB01F3C94800F1300731
:10849000DA5DB24205D1034493F838000BF099FA43
:1084A00002E001311D29EDD10134E4E7C14C162071
:1084B0000BF0C2FAB4F896010BF0C1FAB4F840011F
:1084C0000BF0BDFAB4F842010BF0B9FAB4F844016C
:1084D0000BF0B5FAB4F8DA010BF0B1FA94F8EF0149
:1084E0000BF077FA00200BF074FA94F8F0010BF01F
:1084F00070FA94F885010BF06CFA94F892010BF085
:1085000068FA00200BF065FAA74B0A201B6DB3F93F
:10851000563093FBF0F080B20BF091FA8BE0E0B2B2
:1085200001340BF056FA092CF9D1B8E19E4C102019
:108530000BF082FA94F88C0000F002000BF049FA7C
:1085400094F88D000BF045FAD4F890000BF080FA07
:10855000D4F894000BF07CFAB4F898000BF06FFAA2
:10856000B4F89A000BF06BFAB4F89C00E9E00BF059
:1085700013FA074612200BF05FFA8B4C27B9D4F898
:10858000A460D4F8A85007E0102F19BF00252E468C
:10859000D4F8AC60D4F8B05038460BF01AFA304634
:1085A0000BF056FA28460BF053FAD4F8B4000BF04F
:1085B0004FFA00200BF043FA00200BF040FA0020A5
:1085C000AEE0794D002495F8B8002E4680000130C9
:1085D000C0B20BF031FA95F8B8000BF0FAF996F842
:1085E000B8309C4280F05B81734D285D0BF0F1F94F
:1085F00005F11003185D0BF0ECF905F12003185D8F
:1086000030350BF0E6F9285D0BF0E3F90134E6E7CD
:1086100008200BF011FA0024684B33F814000134E1
:108620000BF00DFA042CF7D139E104200BF004FA19
:10863000604B986831E194F87A010BF0CAF994F82C
:108640007E010BF0C6F994F87D010BF0C2F994F8A5
:108650007F0165E0574C07200BF0EEF9B4F880017C
:108660000BF0EDF9B4F882010BF0E9F994F884010C
:108670000BF0AFF9B4F8860163E04E4C0C200BF020
:10868000DBF994F890010BF0A4F9B4F89A010BF01F
:10869000D6F9B4F896010BF0D2F9B4F898010BF0C2
:1086A000CEF994F891010BF094F9B4F89E010BF017
:1086B000C6F9B4F8A00144E03E4C04200BF0BCF92C
:1086C00094F8D8010BF085F994F8D9010BF081F9F1
:1086D000B4F8DA0135E03A4C3A4D2078002600EB48
:1086E0004000C0B20BF0A8F9237802359E4280F01A
:1086F000D68015F8020C0BF06CF915F8010C013658
:1087000000EB800000EB800000F2EE2080B20BF066
:1087100096F9E9E701200BF08FF9264B93F89201C7
:108720000BF057F9BBE008200BF086F90024214B31
:10873000234493F8880101340BF04BF9082CF6D14F
:10874000ADE00BF07CF9AAE0174B1A4C93F802014C
:1087500004F12005C0EBC000C0B20BF06DF994F835
:10876000F6010023184AD25C904200F09C800C3342
:10877000302BF7D10834AC42F1D190E040200BF01F
:108780005BF90C4C04F14005B4F8A8020BF057F962
:1087900094F8AA020BF01DF9043494F8A7020BF028
:1087A00018F9AC42F0D17AE0BC130020CD130020C0
:1087B000F4AE01086C2A002075140020B6140020C5
:1087C000543200200E2C002064320020E0200BF0F8
:1087D00033F9424C04F18005B4F82A02043400F065
:1087E0003F000BF02CF9B4F82602C0F386100BF012
:1087F00026F994F8240200090BF0EBF894F824020F
:1088000000F00F000BF0E5F894F825020BF0E1F80A
:10881000AC42E1D143E0324C0D200BF00DF909F0F0
:108820006BFD0BF0D6F8A0880BF012F920690BF065
:108830000FF906F0CDF930E00BF0C2F805468420C0
:108840000BF0FAF828460BF003F9254B1C6905F1EB
:108850008003A3428CBF641B802406F079FA28466B
:108860002246694609F080FD05460024AC4216DA2E
:108870001DF804000BF0ADF80134F7E713200BF0FE
:10888000DBF80024174B185D01340BF0A2F80B2C19
:10889000F8D100200BF0DCF800200BF0D9F8012013
:1088A00018E0002016E00BF094F8B4F8F8010BF093
:1088B000C6F894F8FA010BF08CF894F8FB010BF071
:1088C00088F894F8FD010BF084F894F8FC010BF0A3
:1088D00080F84FE721B0BDE8F08F00BF6C2A002080
:1088E00008000020B7CE01082DE9F34704F050FF3F
:1088F000724B1E78002E40F0B185714D2B685A05E1
:1089000040F1AC856F4B704CB3F84E712378DFF8B3
:10891000E481002B00F0FB81D8F800206368D31AB3
:108920007C2B40F2F481237A62600133237206F1DA
:108930002400C0B204F0E0FE644B33F916000DF0E1
:1089400051FC634B814618880DF04CFC01464846AB
:108950000DF050FD5F490DF099FC0DF05DFE013604
:1089600000B204F0B7FE032EE1D1302004F0C4FEC3
:10897000594BDFF85491B3F9000004F0ABFE04F05A
:10898000B3FE237A9B0732D141F28833D9F8042011
:108990009A4219D9102004F0AFFED9F80C006426D1
:1089A00090FBF6F000B204F095FE212004F0A4FE46
:1089B000D9F80C0090FBF6F306FB13000028B8BFB3
:1089C000404200B204F086FE142004F095FE434BB2
:1089D000B3F904000A2390FBF3F004F07BFE1C20A3
:1089E00004F08AFE002004F075FE04F07DFE237A78
:1089F0005E0740F06781022004F07EFE324B4FF0AC
:108A0000050918696423323090FBF3F000B204F0DA
:108A100061FE334B0320B3F9066004F06DFE96FB54
:108A2000F9F6304BB6B21B7858070BD52E483946AD
:108A300009F0ABFE20B92B6813F0100F18BF002609
:108A400030B205E0294B1B689889B0FBF9F000B201
:108A500004F040FE2B68990740F1A080DFF898A051
:108A6000234E9AF8003032884FF0640909FB023235
:108A70005B00B2FBF3F3A78A06203F01BFB247EACF
:108A80000327BFB2C3F303231F4304F035FE38B2FC
:108A900004F020FEA38A9AF8001001339BB293FBE6
:108AA000F1F201FB1233A382A3699B7B012B25D139
:108AB000392004F021FEB6F9000039E0BA35002073
:108AC000283500206C2A0020C0140020EA13002062
:108AD0000800002000007A443414002028140020EC
:108AE000B8320020B8350020F42B002044170020B5
:108AF000F0170020582900209F03002036886E239D
:108B00005E43152796FBF7F63A20B7B204F0F4FD62
:108B1000B7FBF9F630B209FB167604F0DBFD3B201B
:108B200004F0EAFDB0B2461D0A2096FBF0F000B258
:108B300004F0D0FD282004F0DFFDA14B0A201B68C3
:108B400093FBF0F000B204F0C5FD042004F0D4FD66
:108B50009C4B9D4A1B6810689E894FF6FF73984294
:108B6000A8BF1846AEB10028ACBF301A30460DF091
:108B700039FB96490DF08AFB074630460DF032FB73
:108B8000014638460DF036FC0DF046FD6428A8BFBE
:108B9000642020EAE07000B204F09CFD8C4B1B685E
:108BA0009A0640F185808B4F3B789B071FD5DFF8F5
:108BB0005C92112004F0A0FDB9F800004FF4F366B8
:108BC0007043854B90FBF3F000B204F083FD192055
:108BD00004F092FDB9F800004643642096FBF0F6DD
:108BE00096FBF0F300FB136000B204F073FD7B4BC7
:108BF00001201E883B7813F0020F08BF002604F006
:108C00007BFD30B204F066FD092004F075FD002004
:108C100004F060FD724B1E78724B1A88B2F5967F95
:108C200009D9237A03F00F03072B04D842F20F76F9
:108C3000964228BF1646052004F05EFDA3695B7BC3
:108C40000BB930B216E0A6F120000DF0CBFA664960
:108C50000DF0D0FB002106460DF0B6FC10B94FF028
:108C60007C5101E04FF03F4130460DF007FA0DF026
:108C7000D3FC00B204F02EFD3B789F0702D4237F83
:108C8000012B03D101232377584817E0584B59494A
:108C90009E6970680DF0FAFA0DF0BEFC554900901F
:108CA000B0680DF0F3FA0DF0B7FC0190684605E0EE
:108CB000514A92E803008DE80300684604F02CFD59
:108CC00004F012FD237A282B21D1494B0022D8F839
:108CD00000001A724FF47A73B0FBF3F74FF03C09BF
:108CE000172004F009FDB7FBF9F6B6FBF9F009FB14
:108CF0001060000200B204F0EDFC182004F0FCFC4F
:108D000009FB167000B204F0E5FC04F0EDFC637F93
:108D1000374E002B00F06F8109F07AFD336A374A35
:108D2000C31A9342074640F2EC80002386F82630AF
:108D300086F82830324B1B88DAB21B0A86F84220AC
:108D400086F8433086F8382086F83930326DD8F806
:108D500000309A1A736DD97B4FF47A734B439A4261
:108D60000DD3284B1B683365274B1B78013B012B28
:108D70009FBF102386F82630022386F82830104B38
:108D80000A201A68104B92FBF0F21B6884F840200E
:108D900093FBF0F3121284F8412084F844300D4A1A
:108DA0001B1284F845300E4B12781B789607104939
:108DB00084F872302CD42D2381F87330A0E000BFEA
:108DC0004014002044170020381400200000C8423E
:108DD000C013002048140020A08601005414002075
:108DE00049140020980300206666E63F4C140020DA
:108DF000C01400208096184B8CB001083F0D030072
:108E0000F017002058290020322900205614002095
:108E1000042B8CBF3323322381F87330CA48CB4BE9
:108E2000DFF85C8393E800449AFBF0F908FB09A2A1
:108E30004FF0060C0CFB02F2C54B9EFBF0F092FBD0
:108E4000F3F103FB1122642692FBF6F208FB00E823
:108E50000CFB08FC84F86420121284F865209CFB4B
:108E6000F3F203FB12C393FBF6F309EB890949B252
:108E700009EB890901EB890189B284F8621000EBE2
:108E80008000090A84F8631000EB800051B284F876
:108E900069301B1201EB800284F86A30AD4B92B24C
:108EA00084F867201B88120A84F868202422534320
:108EB00093FBF6F384F85F30C3F3072384F8603044
:108EC000A54B0A221B884FEADA7A84F86B301B0A1A
:108ED00084F86C30A14B4FEADE7E1B8884F861A0D9
:108EE000B3FBF2F303F5FA739BB284F86D301B0AFF
:108EF00084F86E309A4B84F866E01B8884F87430EE
:108F0000276294F88490974EB9F1000F0FD1D6F8EC
:108F10008C0009F071FD012809D90228DFF864826C
:108F200000F05E8202F098FC012388F80030D4F84B
:108F300090608C4B002E5ED093F884203AB140F6BE
:108F4000B731D3F89820BA1A8A4216D853E00122D2
:108F500083F88420D3F89C20D3F88C001278022A5E
:108F600004D80430022102F061FC02E0022109F081
:108F700037FD002384F8A0303BE093F89420AAB991
:108F8000C3F8902083F88420D3F89C20D3F88C0079
:108F90001278022A04D80430012102F047FC02E0D2
:108FA000012109F01DFD02F057FC22E0013AD2B286
:108FB00083F8942093F8A01093F8A10042B90130EF
:108FC0004A1C83F8A10083F8A020D3F88C000EE09F
:108FD000324612F801EB01300EEB0106714683F8C0
:108FE000A100D3F88C0083F8A060C3F8902009F0AA
:108FF00006FDC4F8987094F8A2305A4EDBB1D6F84A
:10900000A430C3B1D6F8A830ABB1574A13601A6880
:10901000564B1A60564AD6F8AC301344187AFEF70D
:109020000BFD0AF0E5FCD6F8AC300133092B88BF04
:109030000023C6F8AC304F4E94F8B0203768494B47
:10904000002A00F00B82D3F8B420002A00F0068238
:1090500093F8B830013B012B00F20082D4F8B40041
:10906000DFF8008109F0C8FCE0B1D8F8B40009F0DD
:10907000C0FC98F8B93081467E2BD6F800A00ED1FE
:1090800002231B2888F8B83009D1D8F8B40009F0B9
:10909000B3FC20B90123C8F8BCA088F8C03084F81C
:1090A000B990DBE7D8F8BC2033689B1A41F65832F8
:1090B00093421FD9032388F8B830CFE12E4A32F803
:1090C000130010B903464FF403600133B0F5C06FCD
:1090D000DBB200F0A3801ED9B0F5006F00F0A680CF
:1090E00052D9B0F5036F60D184F8C130234B1B68AF
:1090F000990661D494F8C01094F8C130002900F0AA
:109100006C813268D21B012AD8D984F8C13000237F
:1091100084F8C030A2E1B0F5007F63D007D8B0F585
:10912000807F6AD0B0F5887F00F0B280E6E7B0F5C6
:10913000806F00F0CE80B0F5826F00F00D81B0F549
:10914000047FDBD145E000BF809698004C140020DE
:1091500040420F00561400205A14002054140020DE
:109160005C140020C014002024290020282900209D
:109170008CB0010858290020CED10108C01300206E
:10918000806967FF1C000020B0F5E26F00F092805C
:10919000B0F5E46F00F09480B0F5E06FAED184F8E4
:1091A000C130B04BB3F900108FE0B0F5046F79D047
:1091B000B0F5026FA2D1F9E0AB4B1B789A0799D5B5
:1091C000AA4B198824234B436421123393FBF1F1FA
:1091D000FCE084F8C1302B689B078BD5A44B0A2197
:1091E0001B88F2E084F8C1302B68190582D5A14BA9
:1091F00019680A2391FBF3F1E8E084F8C1309E4B33
:10920000DFF888821B685A077FF574AFD8F80C1016
:1092100002F0D8FA002388F8C0306BE784F8C13038
:109220002B681B057FF566AF944B39E0924A84F8B2
:10923000C130126891067FF55DAF8B4A12789207B4
:109240007FF558AF13F0010F8D4B10D05B681922DA
:1092500083EAE371A1EBE37101EB5101B1FBF2F1A0
:10926000002BACBF41F0004141F040410DE01B68D4
:10927000192283EAE371A1EBE37101EB5101B1FB28
:10928000F2F1002BB8BF41F080414FF400607CE068
:1092900084F8C130784B1B685B077FF52BAF794BA7
:1092A000196893E084F8C130774B0A21B3F9043090
:1092B00059436AE084F8C1306A4BB3F9021004E004
:1092C00084F8C130674BB3F904102C2391FBF3F100
:1092D0005BE084F8C13094F8C2306C4A0133DBB2F1
:1092E000032B88BF012382F8C23042F2107394F836
:1092F000C2105943664B1B78D80748BF01319A0703
:1093000048BF02315807634B48BF04311B88DA0756
:1093100048BF0A31980748BF14311A0648BF2831A0
:10932000D80548BF28315A0748BF6431180748BFDD
:10933000C8319A0548BF01F5C871980648BF01F5C4
:109340007A71DA0648BF01F5FA61580648BF01F59F
:109350007A614FF4806039E084F8C130464B1B6875
:1093600013F0200817D0404B1A7812F0020F14BFE8
:109370004FF47A71002112F0010F474A14BF4FF4E5
:10938000FA6300230B441178194402F01BFA0023FE
:1093900084F8C030AEE62B6819067FF5ABAE4146C7
:1093A00002F010FA394B83F8C080A3E684F8C1308C
:1093B000314B1B689A067FF59DAE2B4B1B789B07A4
:1093C0007FF598AE354B64211B88594302F0FAF9BA
:1093D0002E4B002283F8C0208CE684F8C1303DE09B
:1093E00098F8003023B1C6F8887088F800909EE5A0
:1093F000D6F88830FB1AB3F57A6FFFF498AD0123E5
:10940000D6F88C0088F8003009F0F3FA8046D6F8D8
:109410008C0009F0EEFA18F07F0F7FF488AD8A28EF
:1094200002D08E280DD082E5134B1B6898067FF57D
:109430007EAD96F88430002B7FF479AD06F15803A9
:1094400006E096F88430002B7FF471AD06F124031A
:10945000C6F890302D2386F8943068E502B0BDE858
:10946000F08700BFEA1300204814002056140020A3
:10947000F017002040140020C013002038140020F2
:109480004C1400203414002028140020C0140020A4
:10949000B8350020C41300204914002054140020C3
:1094A000F8B504460E46174600252046202111F047
:1094B000A0FA0446D0B1013420460DF049FEB0F5C3
:1094C000617F05DB40F634039842A8BF184601E0EF
:1094D0004FF46170A0F56170192390FBF3F00DB9A2
:1094E000307000E070703B7801333B700DB901259E
:1094F000DBE72046F8BD30B505460C461346294645
:109500002246BDE83040014802F00FBDEED101080F
:109510007FB504780646E4B9354B1921186800EB8D
:10952000840090F87B5090F879204D4305F56175E3
:1095300090F87A30009590F87C00414301F5617114
:1095400001912C482146013402F0EFFC142CE3D1A8
:109550004BE00DF0FDFD1328054641DC244B701C4B
:109560001C68202100238DF80F3011F042FA1E35BF
:10957000064670B1013630460DF0EAFD1B289FBF4C
:1095800004EB850358709DF80F30013398BF8DF8B8
:109590000F303046202111F02CFA064670B101360A
:1095A00030460DF0D5FD0D289FBF04EB8503987064
:1095B0009DF80F30013398BF8DF80F3004EB850410
:1095C0003046E11C0DF10F02FFF76AFF9DF80F30E6
:1095D000042B0AD0601C0021042211F0D7F904E00A
:1095E000054800211322FFF786FF04B070BD00BFBD
:1095F0000C1400200DD2010822D2010801480AF003
:10960000AFBA00BF28D201082DE9F04304788FB02B
:109610000546002C59D17B4B0021142209A807AE26
:10962000D3F8008011F0B2F907223046002111F082
:10963000ADF900231A46A70005A8059308EB070516
:1096400083807149B5F802E031F813C01CEA0E0FAF
:109650000AD00E310DF1380C595C02F1010E624452
:1096600002F81C1C5FFA8EF20133072BE9D10021AE
:109670000B46664AB5F802E011F802C01CEA0E0F6C
:109680000AD006320DF1380C8A5C03F1010E6344F6
:1096900003F8242C5FFA8EF301310629E9D118F87A
:1096A00007308DE841006A785949029209A81A09E1
:1096B00003F00F030AF090FE2146564809AA013430
:1096C00002F033FC202CA6D198E00DF041FD1F28BC
:1096D000044600F3868028462021E4B211F089F97F
:1096E0001F2C02D9FFF78AFF88E0464B451C1B68F8
:1096F000002103EB84042046042211F047F90027DF
:10970000454B09AE304600210A2217F803905FFA54
:1097100087F811F03BF9002315F8012B32B10A2B21
:1097200004D04A4502D0F2540133F5E74A455ED1F0
:1097300008F1FF33032B09D8DFE803F01005023FDF
:109740000DF1230134E00DF123011EE030460DF050
:10975000FFFC2378C0B243EA001006E030460DF06B
:10976000F7FC237800F00F001843207031E001333C
:10977000062B0AD0244800F11B069E5D9642F6D1C6
:1097800003445A7D63881343638011F8012F02B3A9
:109790000023EFE70133072B0AD01B4800F10E0628
:1097A0009E5D9642F6D130F81320638813436380A0
:1097B00011F8012F6AB10023EFE730460DF0C8FC25
:1097C0000F2804DC30460DF0C3FC607001E000237C
:1097D00063700137052F93D1012404F049F96CB966
:1097E00080E70E4800211F22FFF785FE06E0204695
:1097F0000021042211F0CAF80024EEE70FB0BDE802
:10980000F08300BF84150020A0B00108B5B00108A6
:1098100036D2010845D20108C1B0010822D20108A0
:10982000F8B50478064674B9304D2146B5F8C6211E
:10983000B5F8C8312E48013402F077FB042C05F14D
:109840000405F2D1F8BD2B4911F0A8F8A8B9274BAF
:109850004FF47A714FF4FA62A3F8C611A3F8C82145
:10986000A3F8CA11A3F8CC21A3F8CE11A3F8D021F4
:10987000A3F8D211A3F8D421F8BD30460DF068FC4E
:10988000032805462BD83046202111F0B2F80446B3
:1098900030B1013420460DF05BFC0126074600E0A4
:1098A00006462046202111F0A4F810B9BDE8F84082
:1098B000A4E601300DF04CFC012EF7D140F2DC5350
:1098C000A7F2EE229A42F1D8A0F2EE229A42EDD807
:1098D000064B703503EB8503DF801881F8BD064821
:1098E00000210322BDE8F84005E600BF6C2A0020F5
:1098F00051D2010864D201087DDD01082DE9FF4144
:1099000004780546002C34D16E480AF029F96E4DD2
:10991000286900210CF04EFE002840F0D08021463E
:109920006A4802F002FB2869694602F099F901468B
:10993000674802F0FAFA6869694602F091F901464F
:10994000634802F0F2FAA869694602F089F9014613
:109950005F4802F0EAFAE869694602F081F90134E9
:1099600001465C4802F0E1FA0C2C05F11005CFD15C
:10997000A5E05949052211F051F838B9524B00229F
:1099800003441030C0281A61F8D198E028465349A2
:10999000042211F043F804462846002C41D120212E
:1099A00011F027F8002800F08A80451C284611F0A5
:1099B0002DF807464A4B53F824601EB949480AF06F
:1099C000CFF87CE028463146FAB211F027F801348E
:1099D0000028EFD13C4B0021C2181030C028116183
:1099E0009E46F7D1404BE4001A19D2F82CC0984695
:1099F000BCF1000F04D131463C4802F096FA55E024
:109A0000002708EB040393F828309F42F3DA3B0168
:109A10000EEB0305103563440FCB013785E80F00CB
:109A2000EFE70DF095FB0B28064643DC2846202186
:109A300010F0DFFF054648B10135284602F07AF8FC
:109A4000214B012403EB0613186100E0044628466D
:109A5000202110F0CEFF054640B10135284602F026
:109A600069F8194B013403EB06135861284620218D
:109A700010F0BFFF054640B10135284602F05AF804
:109A8000114B013403EB061398612846202110F096
:109A9000B0FF10B9FFF7B2FD11E0013002F04AF853
:109AA000094B032C03EB0616F061F3D11048FFF7C6
:109AB00025FF04E00F4801210C22FFF71CFD04B034
:109AC000BDE8F0816AD201086C2A002085D2010825
:109AD0008BD2010898DA010864D201088FD20108FC
:109AE0006CB8010894D20108A0B00108A3D2010803
:109AF000A9D0010822D20108F0B5047887B0064643
:109B000014BB514B19201968062303FB041191F86B
:109B1000CA5091F8CE20454305F5617591F8C930DA
:109B2000009591F8CB50C831684300F56170019001
:109B3000087902904979454803912146013402F0A1
:109B4000F4F90C2CDDD17CE00DF002FB0B2804466F
:109B500072DC3D4B701C1D68202100238DF81730EE
:109B600010F047FF064680B1013630460DF0F0FA9E
:109B700003289FBF062303FB045383F8CE009DF800
:109B800017309CBF01338DF817303046202110F07C
:109B900030FF074680B1013738460DF0D9FA0D285D
:109BA0009FBF062303FB045383F8C9009DF81730B9
:109BB0009CBF01338DF8173006266643A919384635
:109BC000CA310DF11702FFF76BFC202110F011FFD5
:109BD000074670B1013738460DF0BAFA14289FBF16
:109BE0009DF817307619013386F8CC0098BF8DF8B0
:109BF00017303846202110F0FCFE78B101300DF00E
:109C0000A7FA0D289FBF062303FB045383F8CD005A
:109C10009DF817309CBF01338DF817309DF8173031
:109C2000062B0ED0062202FB04500021C93010F092
:109C3000ADFEFFF7E3FC04E0054800210B22FFF72F
:109C40005AFC07B0F0BD00BF0C140020AFD20108D1
:109C500022D201082DE9F347047807464CB9204683
:109C600001A90AF069FC0134FFF7F4FF122CF6D1C8
:109C70007FE00DF06DFAC5B2112D75D83E4C05F19F
:109C8000D00604EB4603781C202193F8028010F0E4
:109C9000B0FE3A4F034630B9A8F10202D2F10008F3
:109CA00048EB020848E007F5807800F1010A59788E
:109CB000404610F09EFE68B1032D8CBF03230023A5
:109CC000C8EB0000C0B23B44184490F80491B9F1CD
:109CD000030F02D1FFF792FC4BE0A9F10203D3F18D
:109CE000000850464FF0200148EB030810F081FEB9
:109CF000D8B1B8F1000FEDD001300DF029FA40F2E3
:109D0000ED2380B2984205DD40F6CA039842A8BF11
:109D1000184601E040F2EE20A0F2EE20192290FB5E
:109D2000F2F004EB4603D87002E0B8F1000FD1D195
:109D300004EB460383F8029004EB4604A3781F4427
:109D400097F80021B8F1000F09D0E17819234B43AF
:109D50000B48294603F2EE2302F0E7F809E0294612
:109D6000084802F0E2F804E0074800211122FFF75A
:109D7000C2FB02B0BDE8F0876C2A0020A0B0010849
:109D8000CFD20108E1D201087DDD010810B50446FB
:109D9000204608F028FE18B90A2008F060FDF7E711
:109DA00010BD002207490C2303FB021359688142AE
:109DB00004D10022C2621A725A6070470132042A2A
:109DC000F0D17047643200202DE9F04F064687B08D
:109DD00088469DF8407011461A469DF8443000258B
:109DE0000C206843594C00EB040E0057A146B042CA
:109DF00005D19EF808A0BAF1000F04D0A2E0013509
:109E0000042DEDD19EE0022E00F08C8005DC002EAA
:109E100040F0988000934E4886E0142E0AD01E2E03
:109E200040F09080504603F095F93946044608F01A
:109E3000D7FD7DE0474F484CBB69032243F0040344
:109E4000BB614FF4805B204605A98DF81620039274
:109E5000ADF814B08DF8176000F0ECFBC4F814B046
:109E6000C82008F0FCFCC4F810B0BB69039A43F0AA
:109E70000403BB614FF4C053204605A9ADF814306C
:109E80001C23364C8DF816208DF8173000F0D2FBCD
:109E9000334A4FF4802353614FF0010BE36404F124
:109EA0004C00082384F8513084F852B00AF0DEF9EF
:109EB0002C4B2D4AC3F800A0FB6905A843F400030E
:109EC000FB612A4BDA6002238DF815308DF814609F
:109ED0008DF816A08DF817B00AF0AAF92A238DF88C
:109EE00014309DF817308DF815B08DF816A01BB101
:109EF00005A80AF09DF904E01D4B4FF48062C3F8F9
:109F000084201C4B1C4A1D49136002221A721C4BF0
:109F10001C4A13601C4A1B68116098471B4B636006
:109F20001B4C06E01B4800933B4605F0BFF9044676
:109F300044B10C2303FB05952671204685F8088063
:109F40006C6000E0002007B0BDE8F08F64320020B4
:109F50000038014000100240000801408415002034
:109F600000040140D80042420005FA0500ED00E07F
:109F700000E100E068290020642900202000002082
:109F800064030020CC240020C8240020ACB10108C8
:109F9000881500200048004010B5084B00221968C1
:109FA00001EBC20393F90240844201D1981C10BD19
:109FB0000132042AF4D1002010BD00BF5C32002021
:109FC000F0B5027887B08AB94A4C04F1200694F8BB
:109FD000F6210023484950B2595681426ED00C33C5
:109FE000302BF7D10834B442F1D181E00022049241
:109FF0000592451C0DF0ACF8C4B260B2FFF7CCFF7F
:10A00000074618B18DF81040012400E004462846A8
:10A01000202110F0EEFC054638B1013528460DF040
:10A0200097F80134ADF81200E4B20026284620214A
:10A0300010F0DFFCB0B3451C28460DF089F8002273
:10A040002E495FFA82FE51F82230834204D0013259
:10A05000082AF5D1002300E0734651F823208242FC
:10A0600020D1022E0FD0032E12D05A1E012ED2B2B2
:10A0700004D0042A13D88DF814300EE0042A0ED828
:10A080008DF8153009E0052B09D88DF8173004E05C
:10A090009A1E052A03D88DF816300134E4B2013631
:10A0A000042EC3D1052C04D807B0BDE8F040FFF75B
:10A0B000A5BA04AB03CB3860796019E094F8FB01D2
:10A0C0000E4B94F8FA5153F82000B4F8F8210090A0
:10A0D00094F8FD0153F82000019094F8FC0153F826
:10A0E000200053F825300290054801F01EFF79E763
:10A0F00007B0F0BD6C2A002064320020ECCC0108CF
:10A10000F0D2010838B1438811EA030003D08B4232
:10A110000CBF01200220704710B5204A18B91368FF
:10A1200002221A8210BD1E48146800230380217881
:10A13000024611F07F010DD1637A990644BF0221D6
:10A14000017013F0400F037814BF43F0010323F0B4
:10A15000010314E0012920D002291DD1617901F009
:10A160000F039B0003F1804303F5B84311F0800F08
:10A170001B6806D003F03003102B07D101231370A6
:10A1800004E003F44053B3F5805FF6E7054B1B682A
:10A190001B699847024810BD184610BD642900206D
:10A1A000D8150020C824002010B5064C18B9236823
:10A1B00001221A8210BD044B1B689B6898472068D7
:10A1C0000C3010BD64290020C824002010B5064CB6
:10A1D00018B9236801221A8210BD044B1B681B6842
:10A1E000984720680A3010BD64290020C824002048
:10A1F000084BDA68D10709D4DA68520708D4DB685B
:10A2000013F0100F14BF0320042070470120704783
:10A210000220704700200240024B03EB8101888836
:10A22000704700BFD815002003788B4283BF034BD3
:10A2300003EB4101888C0020704700BFD815002037
:10A240000022134670B5264914180C4494F83C407B
:10A2500083EA0423082413F4004F4FEA430318BF92
:10A2600083F4815304F1FF3418BF83F0010314F029
:10A27000FF049BB2EFD10132192AE4D100F1190297
:10A2800000F11A050A440D4492F83C6095F83C2010
:10A2900002EB062292B29A4221D1114B93F85D5003
:10A2A000E2B2AA4218D2431C03EB4203DBB2CA1843
:10A2B00001330B4492F83C2093F83C3003EB02232B
:10A2C0009BB24FF4AF625343064A1B1303F5487326
:10A2D00022F814300134E3E7012381F85E3070BDC9
:10A2E000D8150020FC15002003788B420BD9074BB2
:10A2F00089001A78064B1944086E02B1400800F52F
:10A30000777080B270470020704700BF583200203D
:10A31000D815002007299DBF034B03EB8101B1F83D
:10A3200090000020704700BFD8150020034B03EBBE
:10A330004101B1F8B000C008704700BFD815002037
:10A3400010B5044608F064FA40F6B8310E4BD3F865
:10A35000D020C3F8D000821A8A4284BF002283F83A
:10A36000D42093F8D4200AB9202C0CD113441F2AEE
:10A37000054983F8D54003D1012381F8F53010BD9C
:10A38000013281F8D42010BDD815002070B50546E3
:10A3900008F03EFA334CD4F8F830C4F8F800C31A89
:10A3A000B3F5FA5FC4F8FC3082BF002384F80031B3
:10A3B00084F8013194F800312BB9A12D02BF294A4C
:10A3C000012182F8011194F80111264A31B1D11806
:10A3D000EDB2013381F83C5082F8003194F800511D
:10A3E00094F80231AB423CD11E4B93F80331052B5C
:10A3F00002D0062B03D02FE00020FFF721FF94F8B6
:10A400003D301E2B28D100200246C1B26B1E99425E
:10A410001ADA214491F83C300821DBB283EA0206C3
:10A42000F60744BF83F01803C3F3460301F1FF317D
:10A4300054BF5B0843F0800311F0FF01C2F34702F1
:10A44000ECD101301A46E0E7234493F83C309A42BD
:10A4500002D10320FFF7F4FE002384F8013184F8D1
:10A46000003170BDD815002010B5044608F0D0F9B1
:10A4700041F28831104BD3F80421C3F80401821A49
:10A480008A42C3F8082184BF002283F80C2193F884
:10A490000C31094A0F2B0DD8591CC9B2134410298D
:10A4A000E4B283F80D4114BF0023012382F80C119C
:10A4B00082F81D3110BD00BFD815002010B504462C
:10A4C00008F0A6F941F288310E4BD3F82021C3F8E9
:10A4D0002001821A8A42C3F8242184BF002283F813
:10A4E000282193F828210749142A134418BF013260
:10A4F00083F8294112BF81F82821012381F83E31D8
:10A5000010BD00BFD815002008B50C4B002093F8F3
:10A510002C1006F089F80A4B1B68187A082801BF2E
:10A52000084B4FF480521A80074B04BF10221A8048
:10A53000A0F109035842584108BD00BF6403002040
:10A5400064290020C4240020C62400202DE9F843FB
:10A55000324F3D682A8A2E7AB2B9042E14D1304C7B
:10A5600030482378012B0BD12F4B19682F4B89B220
:10A570000B445B0019681A6030230380227048E0A6
:10A5800010230380072644E0AC8AAB69A24294BF43
:10A5900004260226944228BF14461FFA84F8404637
:10A5A0009847214A04F1010E13684FEA6E0E9BB2E0
:10A5B00003F1005303F540535B001B6800219BB27D
:10A5C00003F1005303F540535B00714500F10200B5
:10A5D00009D010F8019C10F802CC4CEA092C23F8A1
:10A5E00021C00131F1E71268104B92B213445B00B5
:10A5F0001A681C602B8A3022C8EB03032B826B8AFB
:10A600009844084BA5F812801A80094B4FF4405229
:10A610001A803B681E72BDE8F88300BF64290020E1
:10A62000BB350020C6240020505C004002300020D2
:10A63000C4240020CA78F0B5D40648BF8C780D88B1
:10A6400002F00F0348BF234315F0FF0F1DD0016830
:10A6500000240126A64006EA0507B74211D14FEAB9
:10A66000840E0F2606FA0EF621EA0601282A03FABE
:10A670000EF641EA060101D1476102E0482A08BF0F
:10A6800007610134082CE4D10160FF2D1FD9416816
:10A69000002404F108070126BE4006EA0507B74278
:10A6A00011D14FEA840E0F2606FA0EF621EA0601B2
:10A6B000282A03FA0EF641EA060101D1476102E0B9
:10A6C000482A08BF07610134082CE2D14160F0BD7F
:10A6D0000A88F0B54B888E88B1F808E0CC88002A4B
:10A6E0003AD1028C43F0010322F001021204120C51
:10A6F0000284058B078CADB225F0F30545EA0E11F7
:10A7000089B241EA06027B49BFB2884212D001F504
:10A71000006188420ED0B0F1804F0BD0A1F5983186
:10A72000884207D001F58061884203D001F580613D
:10A73000884202D127F0020701E027F00A071F43F1
:10A7400002830784038B23F00C031B041B0C03837D
:10A75000038B9BB21C4344E0042A44D1028C22F0B8
:10A7600010021204120C0284018B058C21F4407239
:10A770001205120D42EA0E325E4992B242EA0622F8
:10A780008842ADB292B212D001F5006188420ED07B
:10A79000B0F1804F0BD0A1F59831884207D001F578
:10A7A0008061884203D001F58061884207D125F09D
:10A7B000200141EA03139BB243F0100304E025F0AB
:10A7C000A00143F010030B4302830384038B23F4A3
:10A7D00040631B041B0C0383038B9BB243EA0424DA
:10A7E000A4B20483F0BD082A028C3ED122F4807208
:10A7F0001204120C0284828B3E4D92B222F0F307B7
:10A80000018C47EA0E1292B2A84289B242EA0602CD
:10A8100012D005F50065A8420ED0B0F1804F0BD0E4
:10A82000A5F59835A84207D005F58065A84203D064
:10A8300005F58065A84207D121F4007141EA0323A0
:10A840009BB243F4807304E021F4206143F48073ED
:10A850000B4382830384838B23F00C031B041B0CA8
:10A860008383838B9BB21C4341E022F48052120409
:10A87000120C0284858B018C25F440752D052D0D5D
:10A8800045EA062545EA0E321A4D89B2A84292B22F
:10A8900012D005F50065A8420ED0B0F1804F0BD064
:10A8A000A5F59835A84207D005F58065A84203D0E4
:10A8B00005F58065A84207D121F4005141EA033330
:10A8C0009BB243F4805305E047F6FF5543F48053B1
:10A8D0000D402B4382830384838B23F440631B044A
:10A8E0001B0C8383838B9BB243EA0424A4B284832E
:10A8F000F0BD00BF002C014010B50446FFF778FC06
:10A90000012806D11CB1FFF773FC013CF8E70520D4
:10A9100010BD002C08BF052010BD1F4A10B553689C
:10A9200003F00C03042B03D0082B04D01B4B14E0C2
:10A930001B4B1B6811E053685168C3F38343C90381
:10A9400003F1020301D4174906E0516811F4003FF6
:10A950001349096818BF49084B43036053681249FB
:10A96000C3F30313CC5C0368E34043605468C4F34F
:10A9700002240C5D23FA04F484605468C4F3C224F6
:10A980000C5DE340C3605268C2F381320A44127C1A
:10A99000B3FBF2F3036110BD0010024000127A0015
:10A9A0004400002000093D00D0B6010800230360E8
:10A9B00043608360C360036143618361C361036279
:10A9C0004362836270478A6810B50C6A0368144357
:10A9D0000A6923F4FF4314434A6923F070031443C4
:10A9E0008A691443CA6914434A6A14438A6A22432F
:10A9F00013430360CB6843600B6883604B68C3609C
:10AA000010BD4FF6FE73026813400360002303601D
:10AA100043608360C360294B984201D1284A27E0F4
:10AA2000284B984201D1264A2AE0274B984201D16F
:10AA3000234A2DE0254B984201D1214A30E0244B96
:10AA4000984201D11E4A33E0224B984204D11C4A5D
:10AA5000536843F470032EE01F4B984204D1184A08
:10AA6000536843F0706326E01C4B984204D11C4AA3
:10AA7000536843F00F031EE01A4B984204D1184A62
:10AA8000536843F0F00316E0174B984204D1144A80
:10AA9000536843F470630EE0144B984204D1104A9B
:10AAA000536843F4704306E0114B984204D10C4ABA
:10AAB000536843F470235360704700BF080002409E
:10AAC000000002401C0002403000024044000240EE
:10AAD000580002406C00024080000240080402401E
:10AAE000000402401C0402403004024044040240BE
:10AAF000580402400F4B1A6842F001021A6059686C
:10AB00000D4A0A405A601A6822F0847222F4803298
:10AB10001A601A6822F480221A605A6822F4FE022F
:10AB20005A604FF41F029A60044B4FF000629A6023
:10AB3000704700BF001002400000FFF800ED00E089
:10AB40002DE9F8435B4C0368023AC4F8403183882E
:10AB50000D46A4F84431062A05D8DFE802F00A10B1
:10AB60001822292F3500B4F840310B80B4F8423157
:10AB700013E0B4F842310B80B4F8403105E0B4F88A
:10AB800040315B420B80B4F842315B4205E0B4F8DF
:10AB900042315B420B80B4F840316B80B4F84431F1
:10ABA0001DE0B4F840315B420B80B4F8423112E052
:10ABB000B4F842310B80B4F840310CE0B4F84031C5
:10ABC0000B80B4F8423105E0B4F842315B420B80AF
:10ABD000B4F840315B426B80B4F844315B42AB80E7
:10ABE000354B1B79002B62D1B5F900000BF0FAFA56
:10ABF0008046B5F902000BF0F5FA0746B5F90400F6
:10AC00000BF0F0FAD4F84811064640460BF03EFB34
:10AC1000D4F85411814638460BF038FB01464846BB
:10AC20000BF02CFAD4F86011814630460BF02EFB65
:10AC3000014648460BF022FA0CF0C0FCD4F84C1147
:10AC4000288040460BF022FBD4F858118146384644
:10AC50000BF01CFB014648460BF010FAD4F86411C7
:10AC6000814630460BF012FB014648460BF006FACF
:10AC70000CF0A4FCD4F85011688040460BF006FBA1
:10AC8000D4F85C11804638460BF000FB0146404684
:10AC90000BF0F4F9D4F86811074630460BF0F6FAD9
:10ACA000014638460BF0EAF90CF088FCA880BDE8B4
:10ACB000F88300BFD81500204400002044F6FB7143
:10ACC000084BD3F86C21137803EB431300FB0313F9
:10ACD0005078C0EB0030B3FBF0F39078B3FBF0F0AA
:10ACE00080B27047D815002010B50A4C0A2294F89B
:10ACF000713104F5C87004EB4303B3F8801189B2D5
:10AD0000A4F8881107F07EFE80B2FFF7D7FFA4F801
:10AD1000180210BDD8150020334B344A1B68126846
:10AD200010B51A60324A116859605168926899608A
:10AD3000DA60304A116819615168926859619A6104
:10AD40002D4A1168D9615168926819625A622B4A7A
:10AD500011881985518859859188D2889985DA8515
:10AD6000274A118819865188598692889A86254AD9
:10AD70001188D9865188928819875A87224A118862
:10AD800099875188D9879188D288A3F840101946AD
:10AD900021F8422F1D4A10780022824206DA1C4C0C
:10ADA00034F81240013221F8024FF6E7194A1288AE
:10ADB000A3F86C20184A1288A3F86E20174A11884D
:10ADC000A3F8741051889288A3F87610A3F878201D
:10ADD000134A12681A67134A1288A3F87A20124A93
:10ADE0005289A3F8662010BD28230020DC2500200E
:10ADF000B4330020C0330020CC330020B832002010
:10AE0000F0130020EA130020B61400208027002051
:10AE10001014002060170020F0280020F6130020F6
:10AE2000CC1400203C140020FC130020A0F17D0372
:10AE3000012B70B504460D460A4E05D830687D21B9
:10AE400007F0DDFD84F020043068214607F0D7FDCF
:10AE500035B12B881C4404EB142404F0FF042C802F
:10AE600070BD00BF741500202DE9F84305460E465D
:10AE70000D4B002493E88003B44213DA7B1933F9B5
:10AE8000140008EB050333F9142009EB050333F92B
:10AE9000143001341344022293FBF2F3C01A06F07B
:10AEA00075FFE9E7BDE8F8832823002010B5104BB3
:10AEB000014693F8D837012B12D10E4A0E4C107868
:10AEC000431CDBB213701B0644BF002313702154D4
:10AED00003F07CFF3F2809D9BDE8104003F054BFC0
:10AEE000064BBDE81040186807F089BD10BD00BFD3
:10AEF0006C2A00206C2600206E2600206C1000209A
:10AF000070B54720FFF7D2FF174B1B681B0307D50F
:10AF1000164B174A5B6810681B68C01A06F026FFBC
:10AF2000144E154C154D307806F020FF2368286824
:10AF3000C01A06F02BFF63686868C01A06F026FF87
:10AF40000F4B188806F012FF0E4B188806F00EFF04
:10AF50000D4B188806F00AFF337823742B68A36022
:10AF60006B68E36070BD00BF8010002028230020C4
:10AF7000DC25002049140020142300204C1400205C
:10AF80005414002056140020581400207FB5264C7D
:10AF9000264E274D2749284A284B20B128480088AB
:10AFA000B0F5805F31D2308891F820101278ADF87A
:10AFB000040028781C4D1B788DF806008DF80710CA
:10AFC0008DF8082001A8294606228DF809300FF0D7
:10AFD000C5FC30B30198BDF808302860AB80532021
:10AFE000FFF764FF208806F0C1FEA07806F0BEFEE1
:10AFF000E37801A80193237902936379039306F020
:10B0000025FE0F4B00221A800BE0308891F82010AB
:10B010002080127828781B78A070E170227163710B
:10B02000DDE704B070BD00BFF8170020C413002096
:10B030004814002034350020AC1800206E11002088
:10B04000861000200A4A138801331380094A1368C6
:10B0500001331360084A138801339BB2202B01BFD0
:10B0600000231380054A138808BF013313807047FB
:10B07000861000208C10002088100020A8240020BA
:10B0800038B5294B05461B780C46083B012B4AD89E
:10B090004520FFF70BFF2846FFF708FF0E2D33D0A2
:10B0A00003D83DB10D2D07D038BD142D20D0FF2D74
:10B0B00032D038BD20682BE0637820788BB180F0E7
:10B0C0008000FFF7F3FEA468E0B2FFF7EFFEC4F3E1
:10B0D0000720FFF7EBFEC4F30740FFF7E7FE200E63
:10B0E0001EE0FFF7E3FE6068BDE8384006F04EBEA4
:10B0F0002078FFF7DBFE606806F048FE2489E0B2A6
:10B10000FFF7D4FE200A0BE0206806F02FFE6068EF
:10B11000BDE8384006F02ABE044806F048FE00208C
:10B12000BDE83840C2E638BD691000200FD30108E1
:10B130002DE9F04FBC4B8BB01A880193BB4F002A0E
:10B1400040F0AC8042F20103B7F8D607B84EC21AFD
:10B1500050425041FFF71AFFFFF7DEFD34684920E7
:10B160002546FFF7A3FEB34B04F11C09186806F04F
:10B17000FDFD55F8040B06F0F9FD284609F042F9EB
:10B1800004F1100009F03EF94FF01008AA4D012318
:10B190002A6803FA08F3134203D0D9F8000006F036
:10B1A000F5FD08F10108B8F1130F09F10409EDD11B
:10B1B00004F12800032106F0EDFDB7F84031B4F9A1
:10B1C0002E00C01A06F0D2FD2B68DB0408D59B4B7D
:10B1D000B4F86C001B88181AC0F30D0006F0C6FD09
:10B1E0002B68980403D5B4F86E0006F0BFFD2B68F9
:10B1F000590504D504F17400032106F0CBFD2B683A
:10B200001A0502D5206F06F0C1FD2B681B0403D57B
:10B21000B4F87A0006F0AAFDA04604F1300003213C
:10B2200006F0B8FD04F13600032106F0B3FD04F189
:10B230003C00042106F0AEFDB7F8403138F9440F68
:10B240000127C01A06F092FD7D4B1B789F4208DA59
:10B2500038F9020FB4F944300137C01A06F096FDF0
:10B26000F2E72B68980505D5B4F96600A0F2DC502A
:10B2700006F08CFD326873487260B260121A911049
:10B28000714A4A43531C032293FBF2F202EB42023F
:10B290009A1A7C2303FB02033360CEE16B4B6C4AAA
:10B2A0001B6811688B4206D00AA941F8203D002096
:10B2B0001360FFF7E5FE019B97F8D6171B8897F8F8
:10B2C000D7070B44013BB3FBF0F200FB12338B4278
:10B2D00080F07E81564C0120FFF758FEFFF71CFDE1
:10B2E000502026686568FFF7E1FDA26823681068B2
:10B2F0001B68626803441068A046A3EB400006F098
:10B3000045FD6A68736802A89B1A0293AA68B3682D
:10B3100006F11C099B1A0393EA68F36805F11C0BFC
:10B320009B1A049309F06EF82A69336902A89B1AE4
:10B3300002936A69736910279B1A0393B369AA6918
:10B340009B1A049306F082FC3B4801210368B94034
:10B350001942824606D0D9F80000DBF80030C01A46
:10B3600006F014FD0137132F09F104090BF1040B4A
:10B37000EAD106F1260005F12601002331F9024F3A
:10B3800030F9022F121B02AC44F823200133042BA6
:10B39000F4D10322002702AB53F82230BF00FFB2E2
:10B3A0006BB103F108010F2902D847F0010706E04D
:10B3B0008033FF2B94BF47F0020747F0030712F1D9
:10B3C000FF32E8D238460024FFF770FDA3460DF1A6
:10B3D000080907F00302022A10D0032A17D0012A15
:10B3E0004BD1BBF1000F42D0D9F800004FF0000B59
:10B3F00000F00F002043FFF759FD3EE0BBF1000FC6
:10B400000CD0D9F80000C0F3031020432DE0BBF1AD
:10B41000000F1FD199F80100FFF748FD99F80000CF
:10B42000FFF744FD29E000BF881000206C2A0020AF
:10B43000282300208C100020801000208410002081
:10B440008027002034230020DF7BEFBD002900206F
:10B45000AC240020D9F80000C0F303302043FFF7EC
:10B4600025FDD9F80000C0F30710FFF71FFDD9F83C
:10B4700000404FF0010B2401E4B209F1040906ABCE
:10B4800099454FEA9707A4D1BBF1010F02D120469D
:10B49000FFF70CFDDAF8003013F480541FBFB6F844
:10B4A0006C20B5F86C100124521A18BF029299044E
:10B4B0000AD50AAA02EB8401B5F86E00B6F86E2030
:10B4C0000134121A41F8202C5A0513D502AA02EBB6
:10B4D000840E06F1720705F17200002237F9021F8F
:10B4E00030F902CFCCEB01014EF822100132032AD1
:10B4F000F4D103341F0508D50AAA02EB8400296F92
:10B50000326F0134521A40F8202C18040BD50AABC4
:10B5100003EB8402B5F87A10B6F87A3001345B1A7E
:10B5200042F8203C00E0F4B1012C03D1029806F06F
:10B530002DFC18E0631E002002AA52F823204000D0
:10B54000C0B20AB140F0010013F1FF33F4D2FFF7AB
:10B55000ADFC002702AB53F8270008B106F016FC3B
:10B560000137A742F6DB30200321FFF77DFC3620B0
:10B570000321FFF779FC3C200421FFF775FC314BD8
:10B5800044201978FFF770FCDAF80030990506D5E9
:10B59000B6F96600B5F96630C01A06F0F7FBD8F8C0
:10B5A00000202948D8F80430C8F80420121A911055
:10B5B000264AC8F808304A43531C032293FBF2F290
:10B5C00002EB42029A1A7C2303FB0203C8F8003004
:10B5D0001F4B1B681A0630D51E4C1F4D22682B6866
:10B5E0009A420BD162686B689A4207D1019B1B8813
:10B5F000102B11D1194B1B885B060DD14820FFF78A
:10B6000055FC206806F0C2FB606806F0BFFB2368AB
:10B610002B6063686B600EE0114A0F4B11782A7C37
:10B62000914208D10F4A99681068884203D1526844
:10B63000DB689A4201D0FFF763FC06F0F5FA0BB025
:10B64000BDE8F08F8027002034230020DF7BEFBD92
:10B65000283500206014002014230020A824002096
:10B66000491400204C1400202DE9F74F0E9FC2EB27
:10B67000030B4C4C0D9B002914BF4FF006094FF0F3
:10B680000409FF1A636882460133164634D12268E2
:10B690004A4580F08280DFF82881019158F8220025
:10B6A0000FF0B4F90B3006F05FFA0199054608B1C6
:10B6B000012073E022683C48032A98BF514658F89D
:10B6C000222006F0DFFB394A1368181A63681060FD
:10B6D00001336360364B9D710EE00D9A92B103FB0E
:10B6E00007F20D99895C01228A40324909680A42B1
:10B6F00008D163680133636063680C9A294D9342F3
:10B70000EBDB32E003FB0BF5236806EB050A2BB9F4
:10B7100070590FF07BF900F1050801E04FF00308C4
:10B72000404606F021FA0028C2D1204A204B10687A
:10B73000C8EB000010609A791AB12C20FFF7B6FB15
:10B7400001E001229A71236843B9705906F02FFB7A
:10B750009AF904104B1CCCD0174803E09A441748C0
:10B760009AF8041006F08EFBC3E710D1012006F012
:10B77000FBF960B90D4A0A201368013B1360FFF71B
:10B7800095FB2B6801332B604FF0FF336B60206813
:10B7900048452CBF0020012000E0002003B0BDE898
:10B7A000F08F00BF781000201AD30108701000201D
:10B7B000F81700208010002029D30108B0DA010812
:10B7C000E4B6010830B585B004AC002524F8025D6C
:10B7D0000091ADF8060021461020FFF727FB9DF8E9
:10B7E00006002146FFF722FB9DF807002146FFF7E0
:10B7F0001DFB9DF800002146FFF718FB9DF8010096
:10B800002146FFF713FB9DF802002146FFF70EFBD0
:10B810009DF803002146FFF709FB9DF80E0029461D
:10B82000C043C0B2FFF702FB05B030BD73B50D4693
:10B830000646084C2068FEF7B4FA002296F900008C
:10B840000095019208214FF49643FEF7BDFA20605F
:10B8500002B070BD4C15002010B5054C206807F0F3
:10B86000CBF818B1206807F0C4F8F6E710BD00BFA8
:10B870004C150020144810B5046854B113496422D3
:10B880000B685343B3FBF4F3114A138000230360A6
:10B890000B60002213460F491144087D062803D08F
:10B8A000496A8B4238BF0B463432B2F5297FF2D158
:10B8B000092B05DDB3F5967FA8BF4FF4967300E022
:10B8C0000A23054A136010BDB8240020BC240020C0
:10B8D0003029002064000020B4240020F0B50124A9
:10B8E000B0FBF4F58D4201D34C43F9E70026D4B107
:10B8F000B0FBF4F504FB1500B4FBF1F41EB9002D08
:10B9000001DC002CF3D1092D03F1010EEFB204DDAF
:10B91000002A14BF3725572500E030253D441D700F
:10B9200001367346E3E71C70F0BDF0B50124B0FBAF
:10B93000F4F58D4201D34C43F9E70026D4B1B0FBB6
:10B94000F4F504FB1500B4FBF1F41EB9002D01DC85
:10B95000002CF3D1092D03F1010EEFB204DD002A12
:10B9600014BF3725572500E030253D441D700136B2
:10B970007346E3E71C70F0BD03685A1C026019703F
:10B9800070472DE9F843089E002B07468846144669
:10B99000334614BF4FF030094FF0200913F8012B44
:10B9A0000AB9254603E0002CFBDD013CF6E7002D3B
:10B9B00004DD38464946C047013DF8E7354624EAEC
:10B9C000E474A01B284415F8011B11B13846C04788
:10B9D000F7E7BDE8F883024B186807F010B800BF1E
:10B9E000E41200202DE9F0410C464E69CD6909684A
:10B9F00007460AF04BFC6168804630460AF046FC78
:10BA0000014640460AF03AFBA1698046A0680AF068
:10BA10003DFC014640460AF031FBE168804628467D
:10BA20000AF034FC014640460AF026FB216A8046B3
:10BA300020690AF02BFC014640460AF01DFBA66176
:10BA400067612562E061BDE8F0812DE9F8430646B3
:10BA50000C461046002115460AF0ACFD60B1314B92
:10BA600018680AF0BBFB30490AF010FC01464FF0A1
:10BA70007E500AF0BFFC054630460AF0AFFB2B496A
:10BA80000AF004FC29460AF0B5FC06460BF0D4FD8A
:10BA9000054630460BF05CFD2549074630460AF066
:10BAA000F5FB29460AF0A6FC0BF0C6FD0146284628
:10BAB0000AF0ECFB394606464FF07E500AF0DCFAFD
:10BAC0004FF07E51814630460AF0D8FA05464FF0D5
:10BAD0007C5148460AF0DAFB29460AF08BFC2946DD
:10BAE0008046206048460AF085FC4FF04041606087
:10BAF000C4F8088038460AF0C9FB29460AF07AFCE7
:10BB00003146E0604FF07E500AF0B6FA29460AF05E
:10BB100071FC00232061A36163612362E361BDE8DE
:10BB2000F88300BF20350020BD378635DB0FC940C4
:10BB3000CA92283F2DE9F04102780346202A00F1FD
:10BB40000100F9D0092AF7D02D2A02D10346414D30
:10BB500004E02B2A08BF03464FF07E551C46002602
:10BB6000234614F8012BA2F13007F9B209290DD8A8
:10BB7000394930460AF08AFB064638460AF032FB5D
:10BB8000014630460AF07AFA0646E9E72E2A17D12E
:10BB9000314F234614F8010B3038C2B2092A0FD8AE
:10BBA0000AF020FB39460AF025FC014630460AF02F
:10BBB00065FA2949064638460AF068FB0746E8E771
:10BBC0001A7802F0DF02452A39D15A782D2A02D19B
:10BBD0000233012704E02B2A14BF0133023300276C
:10BBE000013B002413F8012F303AD1B2092903D8C0
:10BBF0000A2101FB0424F5E7B4F59A7F28BF4FF42E
:10BC00009A74A0464FF07E53B8F1070F07D9184633
:10BC100012490AF03BFBA8F108080346F4E704F0D8
:10BC2000070434B118460C490AF030FB013C0346C6
:10BC3000F7E719462FB130460AF0DCFB04E04FF07D
:10BC40007E5130460AF022FB014628460AF01EFBD0
:10BC5000BDE8F081000080BF0000204120BCBE4C48
:10BC600030B5054687B00C4603A800210C220EF023
:10BC70008DFE284600210AF0C5FC20B1284628493F
:10BC80000AF0FCF903E0284625490AF0F5F92549B0
:10BC90000AF0FCFA0AF0C0FC054680EAE07069464A
:10BCA000A0EBE57008F048FC002DACBF20232D234D
:10BCB00068468DF80C300EF0A9FE012807D130231C
:10BCC0008DF80D308DF80E308DF80F300CE0022815
:10BCD00005D130238DF80D308DF80E3004E00328A7
:10BCE00004BF30238DF80D30694603A80EF074FEB2
:10BCF00003A80EF08BFE0338C5B22A4603A92046DE
:10BD00000EF0AEFE00236355204607490EF064FE98
:10BD100003AB204659190EF05FFE204607B030BD38
:10BD20006F12033A00007A444DD3010870B50646FD
:10BD3000B6FBF2F40846154614B12046FFF7F6FFAD
:10BD400005FB1464024B1B5D00F8013B70BD00BF96
:10BD50004FD301082DE9F04F81468A4616461C460E
:10BD600089B000253178002900F0DB80252902D038
:10BD70000136484674E072784FF00008302A0CBF54
:10BD8000B278B71CA2F1300312BF4FF0000BF71CC2
:10BD90004FF0010B092B19D8A2F13003D9B20929B0
:10BDA00005D80A2202FB083817F8012BF4E7A2F1A4
:10BDB0006103052B02D8A2F1570305E0A2F141036C
:10BDC000052B03D8A2F137030A2BEADD6C2A30D108
:10BDD0003A787E1C642A00F083800BD8252A3DD057
:10BDE00003D8002A00F09D80BCE7582A0CD0632AB3
:10BDF00019D0B7E7732A22D002D86E2A37D0B1E71C
:10BE0000752A5CD0782AADD1271D2068A2F158048C
:10BE100062424FF01001624155E02CD9582A32D0CD
:10BE2000632A2AD13E4648462178271DD04701354E
:10BE30000FE0642A63D00ED9732A14D13E462368DA
:10BE400048460093514642460023FFF79AFD271DBE
:10BE500005443C4686E7252ADFD13E464846252153
:10BE6000D04701357EE70AD86E2A06D13E462368C0
:10BE700004341D6076E7002A53D03E4672E7752AE7
:10BE800026D0782AF9D1A2F1580304F1040C5A42C1
:10BE90002068CDF80CC04FF010015A4105ABFFF7F8
:10BEA0001DFDDDF80CC03E46644605AB00934846D8
:10BEB000514642465B46FFF764FD054452E7206861
:10BEC000271D0A21002205ABFFF72FFD3C46ECE7BA
:10BED00004F1040CCDF80CC020680A210022DDE733
:10BEE0002068271D002808DA2D238DF814304042E1
:10BEF0000DF115030A210022E6E705ABFAE72068F9
:10BF000004F1040C00280ADA2D238DF81430404285
:10BF10000DF11503CDF80CC00A210022BFE705ABD7
:10BF2000F8E7284609B0BDE8F08F0FB413B50B4908
:10BF300004AB08680A4953F8042B09680193FFF71A
:10BF400009FF0446074B186806F04DFD0028F9D09C
:10BF5000204602B0BDE8104004B070471404002031
:10BF600010040020E412002080EAE073A3EBE073E9
:10BF70008B4206DB002801DD401A704702D00844DE
:10BF800070470020704770B504460AF045FB20302A
:10BF9000402857D820462C490AF034FB28B12046C7
:10BFA0002A490AF069F80446F4E7204628490AF0CD
:10BFB0000BFB28B1204625490AF060F80446F4E757
:10BFC000204624490AF01EFB30B1224920460AF0DF
:10BFD00053F801461F480AE020461F490AF0F4FAC8
:10BFE00040B11C4920460AF049F801461A480AF0B7
:10BFF00043F80446214620460AF048F90546204603
:10C0000029460AF043F90021064628460AF03EF97F
:10C0100012490AF031F8014628460AF037F910496A
:10C020000AF02CF8014628460AF030F90D490AF0CA
:10C0300023F8014630460AF029F9014620460AF065
:10C040001DF870BD002070BDDB0F4940DB0FC940FB
:10C05000DB0F49C0DB0FC93FDB0FC9BF92E7413996
:10C060009730083C15A82A3E08B503490AF006F89F
:10C07000BDE8084087E700BFDB0FC93F064B10B59E
:10C080001A881C4622EA00009042188002D0012043
:10C0900006F04EFC208810BDC4130020064B10B5DE
:10C0A0001A881C4610439042188002D0012006F0E6
:10C0B0003FFC208810BD00BFC4130020024A9368D3
:10C0C00023EA0000906070476C2A002008B5104BEE
:10C0D0001A780023D9B2914207D20E49002051F8B4
:10C0E0002310013309680880F4E7322006F0B7FB1B
:10C0F000094B1B685A0309D5084B9B685B0305D4A1
:10C10000BDE8084040F2DC5006F0A9BB08BD00BF06
:10C110008027002050270020283500206C2A00208E
:10C120002DE9F34109F0A0F94B4A7723137040F24F
:10C13000E4735380BE231371EF2382F8E0370023AA
:10C140001946164682F8E137F25C0133514040F25D
:10C15000E4729342F8D1404B404A83F8E117404BD8
:10C1600004275A6002F188325A600020013F17F01C
:10C17000FF075ED03A4B34223A4CDA6004F178483B
:10C18000A8F5FC38C8F3090353B100234FF400505D
:10C1900056F808800193FEF7AFFB0428E6D11CE0B7
:10C1A0004FF43020FEF7A8FB0428DFD12C4D4FF4CC
:10C1B00030202B6943F002032B616C612B6943F043
:10C1C00040032B61FEF798FB41F6FD732A690428B2
:10C1D00003EA02032B61D8D0C8E7214D4FF4005089
:10C1E0002B6943F001032B611FFA88F32380FEF7CC
:10C1F00083FB042813D1A31C0193019B4FEA184829
:10C20000A3F800804FF40050FEF776FB41F6FE7372
:10C210002A69042803EA02032B6106D0A6E741F647
:10C22000FE732A6913402B61A0E70F4B04349C4234
:10C23000A4D10B4A0428136943F08003136102D18F
:10C2400005F03CFA10B9052006F08AFB09F0F6F873
:10C2500002B0BDE8F08100BF6C2A002023016745D1
:10C260000020024000F80108E4FF01082DE9F04138
:10C2700005F024FA10B9042006F072FBB94C09F05D
:10C28000F3F8B94940F2E47220460EF076FB94F8D8
:10C29000B0374FF4CC71022B84BF002384F8B03741
:10C2A00094F8B027B14D01FB02F303F53A70204436
:10C2B0002344286093F83C0301FB0242022803F563
:10C2C0004E7384BF0020187192F83C33A84A137053
:10C2D0000C2202FB0343A74A03F2B273136046F237
:10C2E0000902A3681A401AB99E4A43F400539360A6
:10C2F000A368DE0703D54FF40050FFF7DFFEA36805
:10C30000580409D50820FFF7D9FE4FF40050FFF775
:10C31000D5FE0120FFF7D2FEA368190706D54FF41A
:10C320000050FFF7CBFE0120FFF7C8FEA3689A0478
:10C3300013D54FF40040FFF7C1FE8A4B93F88431C8
:10C34000012B03D14FF40060FFF7B8FE4FF48030AB
:10C35000FFF7B4FE4020FFF7B1FEA3685B0603D5EC
:10C360004FF48030FFF7AAFE4FF0000C6746824E74
:10C37000824B1E6004EB0C03B3F8F8E14FEA5E0158
:10C3800001F077314FEA9E0303F03333C1EB0E0027
:10C39000C11A4FEADE0303F01133CB1A03EB231368
:10C3A00003F00F32FF2392FBF3F31EF00108C3EBFF
:10C3B000032318BF0137A2EB030318BFFFB2012B01
:10C3C0000ADD022B40F0CA80B8F1000F00F0C680F1
:10C3D0001EF0BC0F00F0C2800CF1080CBCF1200F65
:10C3E000C8D1013F012F00F2B98005F044F9302295
:10C3F000002163480EF0CAFADFF81082614B2F6803
:10C40000C3F80080604B002107F179001F6006F03F
:10C41000ABF95E4B80F0010018705D4B08F128010C
:10C42000196097F850205B4B1A705B4B08F1D802EB
:10C430001A603B781BB1022BA8BF022300E0012346
:10C44000DBB2022B14BF554A554A3B70554B384658
:10C450001A60554B07F5C5721A6002F00BFB94F891
:10C46000D801642242435149514BC8321960514BA3
:10C470002D685A6000229A60DA601A615A619A61E6
:10C48000DA6183F8202083F821204B4BA1F16A0266
:10C490001A604A4B05F219121A60494B05F28912CB
:10C4A0001A60484BA1F190021A60474B01F10C024F
:10C4B000C3F80080454B464F1A60464B16311E604C
:10C4C0003960B4F8640109F08DFE434909F092FF28
:10C4D000F860B4F8660109F085FE3F4909F08AFF6B
:10C4E00095F85C303A1D3B7195F87830B8607B71F7
:10C4F00094F8E331286E3B74384B7D611A60384BF9
:10C5000005F164021A60374909F0C0FE01464FF098
:10C510007C5009F06FFFB5F81641334B1860204688
:10C5200009F060FE0146314809F064FF304909F026
:10C53000ADFE304A304B1560304A186005F1680393
:10C5400013602F4A05F2111515602E4AC2F80080BB
:10C550002D4ABDE8F041136008F070BF07F0A0FF5E
:10C5600043E700BF6C2A002000F801080C140020EB
:10C570000829002044140020F42B0020243500203A
:10C58000A8110020DC110020E01100200200002092
:10C59000DC090020690900203C090020B14701089E
:10C5A000DD4A010894030020EC110020442C0020F7
:10C5B0004434002034350020683500200C2300204E
:10C5C000240C00202428002028280020300B0020E4
:10C5D00000180020FC0B002000401C46340A0020FC
:10C5E000CC0A0020DB0F4940C80A0020000061444B
:10C5F0004C3D0F44142600202C0B00200826002060
:10C60000200B0020280B002000250020AC2B002050
:10C6100008B5FFF785FDFFF729FEBDE808400120BA
:10C6200006F086B92DE9F04FB34B85B01A68039335
:10C6300012F4803F00F0DC82B04C2378002B00F035
:10C64000D782AF4B1A7802F0FF03002A40F0D08265
:10C65000AC4ADFF8F892126812F4804F0ED099F8C5
:10C66000002072B1A84A1168A84A42F82310013389
:10C67000202BF7D105F06CFC002300E0012389F8A2
:10C68000003099F80030002B00F0B28206F0C0F8BC
:10C69000D4F88460D4F88850D4F88C70861BF643A4
:10C6A000451BC71BED43FF43F60F8046ED0FFF0F01
:10C6B0002EB93FB9002D00F09B82BA462DE04FF015
:10C6C000000A2AE0B24628E00B684FEA8B021344C6
:10C6D000598808050FD411F4805F884918BF58782D
:10C6E0000A4415BF8A4988490968096818BF51F882
:10C6F0002010C2F802105A88D10516D493050AD525
:10C70000844B04EB8B0B1B78580754BF824B834B35
:10C710001B68CBF802300AF1010A94F890005FFA26
:10C720008AFB83457E49CFD329E019467D4A584686
:10C73000019301F02DF97C4A019B128812F0400F01
:10C7400003D058461946794A16E0510703D5584692
:10C750001946774A10E0100703D558461946754A1E
:10C760000AE0910703D558461946734A04E0D207F8
:10C77000D1D558461946714A01F00AF9CBE70B6842
:10C78000782201936E4BB3F90630A3F57A735343C5
:10C790004FF47A7293FBF2F303F22B13029300220D
:10C7A0005FFA82FE864517D2019B03EB820EBEF82C
:10C7B00002E01EF4806F0DD040F2671BDFF84CA141
:10C7C000029B3AF822E09E449EFBFBFC0BFB1CEE16
:10C7D0002AF822E00132E3E785B308F5C333A0333A
:10C7E000C4F8883094F89130444A3BBB82F89230C8
:10C7F000039B1B6813F0020F0AD0DFF854E19EF888
:10C8000000E0BEF1000F03D04FF0010E82F892E07D
:10C81000DA0508D54B4BDB782BB194F8923043F016
:10C82000020384F892303B4B1B7813F0050F02BFD4
:10C8300094F8923043F0040384F8923094F892E034
:10C84000BEF1000F05D12D4B93F89130002B00F075
:10C85000838094F891C01CF0010FACF10C031DD142
:10C86000BCF1030F07D8DFF8A0A01EF0040F2A4A7E
:10C8700008BF524600E0244AACF1040CBCF1070F9B
:10C8800005D8DFF8D0C01EF0010F18BF6246DBB23A
:10C89000032B0ED81EF0020F2B4B06E0DBB2032B4E
:10C8A00006D81E4B184A1EF0020F18BF1A4600E0A9
:10C8B000154A4FF0000C5FFA8CF383420DD20B68DF
:10C8C00003EB8C035B881B0642BFD2F800A00F4B22
:10C8D00043F82CA00CF1010CEDE7002D44D0BEF183
:10C8E000000F3AD094F89130044A0133DBB2142B94
:10C8F00038D1002336E000BF28350020181800206A
:10C90000B9350020C813002074D301081A1800207C
:10C9100008230020B8350020FCB6010808B701083C
:10C92000841500200CB70108C413002012B70108B9
:10C9300018B701081EB7010824B701082AB7010873
:10C94000943200203435002004B701084C00002048
:10C950003229002000B7010835B194F89130002B3E
:10C96000C0D101E082F8913036B3A34A3223B2F944
:10C970000250B2F90020002DB8BF6D42002AB8BFA6
:10C98000524295FBF3F592FBF3F2EDB2D3B2AB4218
:10C9900038BF2B46994A13B192FBF3F300E01346DC
:10C9A0004344C4F8843094F89330954A0BB901237A
:10C9B00000E0002382F8933094F89450904B94F860
:10C9C0009320ADB9002F00F00E818E4B94F890604B
:10C9D0001A788D4B02F00402D3F800E00B680021B6
:10C9E000D2B299F801C0894D03EB86060F46B1E03B
:10C9F00022B9874AC3F89820002508E0854AF9E75C
:10CA00000A68AB00D6187688760604D40135EBB2F6
:10CA10008342F5D3D6E7784EB6F90060192E23DDB0
:10CA200012F803C094F89CA00CF00F0BD345744E81
:10CA3000D4F898E009DC96F89DA0BAEB1C1FDEBF85
:10CA4000DEF800C0023643F806C012F803C094F8BE
:10CA50009EA00CF00F0BD345694E2FDB96F89DA0DE
:10CA6000BAEB1C1F2ADC24E0193627DA12F803C0BF
:10CA700094F89CA00CF00F0BD345614ED4F898E0CD
:10CA800009DC96F89FA0BAEB1C1FA2BFDEF800C01D
:10CA9000023643F806C012F803C094F89EA00CF0CA
:10CAA0000F0BD345564E09DB96F89FA0BAEB1C1F1F
:10CAB00004DBDEF800E0023643F806E04E4EB6F93D
:10CAC0000260192E1ADD12F803A094F89CC00AF037
:10CAD0000F0BE3454A4ED4F898E009DC96F89DB078
:10CAE000BBEB1A1FDEBFDEF800A0023643F806A03B
:10CAF000D25C02F00F0666451DDD87E7193685DA40
:10CB000012F803A094F89EC00AF00F0BE3453C4EC8
:10CB1000D4F898E009DB96F89DB0BBEB1A1FDEBF96
:10CB2000DEF800A0023643F806A0D25C02F00F0641
:10CB30006645FFF66BAF94F89F60B6EB121FA2BF7D
:10CB4000DEF80060344A9E5060E75888000504D43F
:10CB500004330435B342F8D122E04AB101EB0C0BA7
:10CB600006209BFBF0FA00FB1AB001280DDC01E067
:10CB700057B9012793F801A00EEB8A003EF82AB0BE
:10CB800090F802A0C07803E0174600208246834652
:10CB9000013125F802BC85F800A06870C9B2D7E75A
:10CBA00099F801301D4A013B13F0FF0308BF06232B
:10CBB0005370144B1B785B0743BF194B4FF47A72C9
:10CBC000B3F90630012342BFA3F57A7303EBC30325
:10CBD00093FBF2F3094A44BF0133DBB292FBF3F358
:10CBE0004344C4F88C3005B0BDE8F04F05F0B0B94F
:10CBF00005B0BDE8F08F00BFB8320020400D030043
:10CC000018180020B8350020082300201C18002028
:10CC100030B7010874D301081A1800204C00002016
:10CC200094320020426A806A131A58425841704771
:10CC30004171704743799B070AD5436A8269D15491
:10CC4000436A01690133B3FBF1F201FB1233436222
:10CC50007047427902F0020202F0FF0342B1036919
:10CC6000426A806A013BDBB2101A23EA0000704777
:10CC700018467047437913F001031FBFC36803F1DF
:10CC8000FF32C369006A1DBF181A1040C0B21846AF
:10CC90007047437910B513F0010304460DD0FFF738
:10CCA000E9FF58B1236A6269E168D05C0133B3FBE4
:10CCB000F1F201FB1233236210BD184610BD90F84B
:10CCC0003B3210B57BB990F83A3290F83942A34222
:10CCD00009D2B0F8401201229A400A430133A0F869
:10CCE0004022DBB2F3E710BD8379DB0748BFB1FA1E
:10CCF00081F1D0F8343148BF49095A681B8909B11C
:10CD0000136170475361704710F80A3C0133DBB27E
:10CD10000A2B84BF10F8131C044A00F80A3C82BF97
:10CD2000002322F8113000F80A3C7047B834002084
:10CD3000354A70B5136C90681944344B1B78D94050
:10CD400040F68C23081A98429160D06051601346D7
:10CD50003BD9127893F9451010468A420BD1111F26
:10CD6000082908D893F84610182901D8013103E0A2
:10CD700083F8442002E0002183F8461093F94440F0
:10CD80002149A24219D191F84740B4B10C31002495
:10CD9000944206DA51F8046F1D4D25F814600134F1
:10CDA000F6E70C2805D01A49002421F8104001307C
:10CDB000F7E7184801780131017083F84520002217
:10CDC00001211A7083F8471070BD92F84710C9B15D
:10CDD00040F2DA51A0F2EF248C4208D811780B29E6
:10CDE00005D80B1D0131117042F8230070BD0022DF
:10CDF00083F84720084B03F13002002143F8041F59
:10CE00009342FAD170BD00BF3804002035040020E1
:10CE1000B8340020DE28002044040020024A136CAD
:10CE2000013319441164704738040020024B53F851
:10CE300020301B681980704750270020074BA1F550
:10CE40007A7153F820301A681B8959434FF47A736A
:10CE500091FBF3F189B21180704700BF5027002089
:10CE60001FB50123ADF80830ADF80410002301A967
:10CE7000ADF80A30ADF80C30ADF80620FDF728FC0F
:10CE800005B05DF804FB38B5A0F513746379A57996
:10CE9000DB0745D594F8383205F00105F3B1226B74
:10CEA0001068838DC3F34E03838494F83C3223B11E
:10CEB000B4F842320133A4F84232917A6A00FFF7A3
:10CEC000CFFF012384F83B32002384F8393284F801
:10CED0003A3284F83832A4F8403238BD94F83B3204
:10CEE0002046012B04BF94F8393284F83A32FFF718
:10CEF000E6FE94F83B22236B3AB9012284F83B22E8
:10CF00001868997A05FA02F207E0002284F83B22B9
:10CF100095421868997A08BF0222BDE838409FE719
:10CF200038BD10B5A0F5127494F83C22BAB9A36AC2
:10CF3000616A994228D0591CA069A162C35C20692A
:10CF4000DBB25B0043F400738142A4F83E324FF041
:10CF50000A0384F83D3228BFA262012312E094F94B
:10CF60003D327BB1B4F83E1220464B08A4F83E3265
:10CF700001F00101FFF7B8FE94F83D32013B84F85F
:10CF80003D3201E084F83C3294F83832002B4ED127
:10CF900094F839320133DBB2092B84F8393203D1EA
:10CFA0002046BDE810408AE60A2B40D194F83B3277
:10CFB0002BB9B4F8403243F00103A4F8403263794E
:10CFC000D9071CD5B4F84002820501D4C30705D4A3
:10CFD000B4F844320133A4F8443210E0E36AC0F3F9
:10CFE00047000BB198470AE0E3696269D054E369EE
:10CFF000E1680133B3FBF1F201FB1233E36101227B
:10D0000084F8382294F83B220023012A84F839322C
:10D010000DD1A27984F83B32236B12F0010F18680E
:10D02000997A0CBF02220022BDE8104018E710BD1B
:10D03000F0B5046D8279A389467923F4005312F088
:10D04000020F4FEA03434FEA13430CBF00214FF492
:10D05000005112F0040FA38114BF4FF4806E4FF003
:10D06000000E16F0010F8768054614BF042000204B
:10D07000B307238A48BF40F008029BB223F4405311
:10D0800043EA01032382A18948BF90B289B221F407
:10D09000B05121F00C014EEA010140EA0102A281E7
:10D0A000A38A87B023F440731B041B0CA38201A83E
:10D0B000FDF733FC039B049E254A944218BF1E468D
:10D0C000A389192272431BB2002BB4BF7E00BE009D
:10D0D000B2FBF6F66427B6FBF7F00001010907FB87
:10D0E0001163A28912B2002AB7BFD9001A013231E6
:10D0F000B1FBF7F2A7BF3232B2FBF7F302F007023F
:10D100001043A8BF03F00F03AA79A8BF184380B249
:10D1100012F0010F20812B6D06D00D498B4202BF0A
:10D120000420A1F53051086112F0080F9A8A0BBF54
:10D1300022F0080292B2120442F0080208BF120C58
:10D140009A829A8992B242F400529A8107B0F0BD55
:10D15000003801402DE9F04F4E4C4FF4147585B066
:10D16000804691461E4605FB0045274620B94A4B9E
:10D170002B63103BC5F834314FF4147303FB08F3F1
:10D18000464AFC18FA5003226271224603F59C734A
:10D190003B44E162A36100214FF48070D4F8343144
:10D1A00034324FF0010B62612162E161A162616280
:10D1B00084F83C1284F83912A4F84212A4F84412FC
:10D1C000C4F80890A671E060206184F838B284F851
:10D1D000468258681B890222ADF80C3003A910233F
:10D1E0008DF80E308DF80F20019204F08FFF236B25
:10D1F000019A597B58681B898DF80E1003A9ADF868
:10D200000C308DF80F2004F081FF28465946FFF7B7
:10D210006BFD322005F023FB214BD4F834A11B68B1
:10D220001A46B2FBF9F1B1F5803F03D3012AF8D9D0
:10D230005208F6E71B4A5046B3FBF2F289B2D2B26B
:10D2400001F06EFF4FF4147000FB08F0164B07EB73
:10D25000000800F512703C180022C8F84832504609
:10D26000214601F0A5FFD8F8307016F0010F0CBF71
:10D27000022200223868B97AFFF7F2FD0B4B3846DC
:10D28000C8F84C32211D002201F092FF284605B05B
:10D29000BDE8F08FB8180020CCCD010834B70108E4
:10D2A000A003002040420F0023CF000887CE0008D3
:10D2B00003460A4690F84602D96A9B794AE71FB5A9
:10D2C0000123ADF808300023ADF80C30ADF80A307A
:10D2D000084BADF804101B7801A9012B08BF0323EC
:10D2E000ADF8062008BFADF80C30FDF7F1F905B038
:10D2F0005DF804FB3404002038B510F80E2C044609
:10D3000050F8043C52B9012200F80E2C20F80C1CF5
:10D31000997A18680222BDE83840D0E730F80C2C22
:10D3200020F80A1C891A89B220F8081C074A10F84C
:10D330000F0C002522F8101004F80E5C1868997A7A
:10D340002A46FFF7BCFF04F8065C38BDB83400205D
:10D35000044B53F820301BB107289CBF1B68198071
:10D36000704700BF600500202DE9F7438E46054653
:10D37000DFF8A092114699F8504200681646984688
:10D380007246631C89F8503201F076FE2B8901A9A0
:10D39000ADF8043018238DF80630686802238DF844
:10D3A000073004F0B3FEAB7A09F515772401274462
:10D3B0002A6849460C2B00F2F680DFE813F00D00D6
:10D3C000F400F400F4005100F400F400F4008A00CA
:10D3D000F400F400F400C200138CDFF83CC223F028
:10D3E00001031B041B0C1384138CB2F804E0108B94
:10D3F000624520F073004FEA00404FEA10409BB2B4
:10D400001FFA8EFE40F0700014D00CF5006C6245DF
:10D4100010D00CF5406C62450CD00CF5806C624568
:10D4200008D00CF5806C624504D023F0020343F071
:10D43000030307E023F00E032EF4407E43F00303C2
:10D440004EF4807EA2F804E01083A2F834801384A6
:10D45000138B23F008031B041B0C43F0080336E076
:10D46000138CDFF8B4C123F010031B041B0C1384CE
:10D47000138CB2F804E0108B624520F4E6404FEACA
:10D4800000404FEA10409BB21FFA8EFE40F4E0408D
:10D4900008D00CF5006C624504D023F0200343F063
:10D4A000300307E023F0E0032EF4406E43F0300336
:10D4B0004EF4806EA2F804E01083A2F83880138442
:10D4C000138B23F400631B041B0C43F400631383CE
:10D4D00069E0138CDFF840C123F480731B041B0C3C
:10D4E0001384138CB2F804E0908B624520F0730033
:10D4F0004FEA00404FEA10409BB21FFA8EFE40F008
:10D50000700008D00CF5006C624504D023F4007361
:10D5100043F4407307E023F460632EF4405E43F469
:10D5200040734EF4805EA2F804E09083A2F83C8041
:10D530001384938B23F008031B041B0C43F0080394
:10D5400030E0138CDFF8D0C023F480531B041B0C95
:10D550001384108CB2F804E0938B20F4005023F471
:10D56000E6431B0400041B0C000C62451FFA8EFEF0
:10D5700043F4E04340F4405003D00CF5006C6245A6
:10D5800003D12EF4804E4EF4804EA2F804E0938333
:10D59000A2F840801084938B23F400631B041B0CBF
:10D5A00043F4006393832B7B43B1B2F844306FEABA
:10D5B00043436FEA53439BB2A2F8443013889BB2B3
:10D5C00043F001031380AB7A0C2B19D8DFE803F08A
:10D5D000071818180B1818180F18181813000B191B
:10D5E00002F134000AE00B1902F1380006E00B19D1
:10D5F00002F13C0002E00B1902F14000C3F85402B2
:10D6000038460C44A4F85C62C4F8582203B0BDE864
:10D61000F08300BFB8180020002C01400028114AF8
:10D62000B8BF404290FBF2F330B50F4C3C2504FBF1
:10D63000030068430D4D90FBF2F22D682D7B25B958
:10D6400003EB830303EB830301E0C3EB031302EB60
:10D65000830304FB02020B804FF47A7392FBF3F214
:10D660004A8030BD80969800806967FFD8140020FA
:10D67000022803D0431E584258417047064B1B688E
:10D680001B7823B1054B1868C0F3C0407047044BAA
:10D690001878C0F3800070473C090020C8130020B0
:10D6A000B835002010B50A4C5E280146206805D127
:10D6B0005D2105F0A4F920683E2105E05D2903D134
:10D6C00005F09DF920683D21BDE8104005F097B9AF
:10D6D000CC1B002010B50446C0B2FFF7E3FFC4F333
:10D6E0000720BDE81040DDE7024B5E21186805F019
:10D6F00086B900BFCC1B002038B50546054C5E211D
:10D70000206805F07CF920682946BDE8384005F01E
:10D7100076B900BFCC1B002013B5044601A90068F0
:10D72000FFF77CFF1320FFF7E7FFBDF90400FFF7C9
:10D73000D1FF1B20FFF7E0FFBDF90600FFF7CAFF8E
:10D740002320FFF7D9FF2368002BB4BF53204E20BE
:10D75000FFF7C0FF01A96068FFF760FF1220FFF725
:10D76000CBFFBDF90400FFF7B5FF1A20FFF7C4FF98
:10D77000BDF90600FFF7AEFF2220FFF7BDFF63688B
:10D78000002BB4BF57204520FFF7A4FF02B010BD07
:10D79000674B73B51878FFF76BFF664D04462B781F
:10D7A000834220D0C8B1644B1B68E3B193F90000F9
:10D7B00002230093614B04211B6800225B78003335
:10D7C00018BF012301934FF41653FCF7FDFA5C4B8D
:10D7D000186040B101232B7005E0594E3068FCF70A
:10D7E000E0FA34602C70574B574D1878FFF740FF24
:10D7F0002B780446834218D088B1544B1B68A3B1E0
:10D800000022012493F9000008214FF4964300946C
:10D810000192FCF7D9FA4E4B186028B905E04C4E3E
:10D820003068FCF7BEFA34602C704A4B4A4D1878C9
:10D83000FFF71EFF2B78044683422E4643D0002874
:10D8400038D0464B1A68002A3DD0D37992F90000AF
:10D85000002B4FF00202424C08BF0223009200222C
:10D8600054F8233001921021FCF7AEFA3D4B0546E7
:10D87000186040B33C4C94F84A30022B0BD094F81B
:10D880009620022A01D14C3405E023B1002A04F18C
:10D890004C0418BF0024354B1C6044B120460021C5
:10D8A0004C220DF073F80223256084F84A300123DE
:10D8B000337008E02B4E306806F04EF83068FCF705
:10D8C00070FA34602C702A4B2A4D1878FFF7D0FE7E
:10D8D0002B780446834229D000B3274B1B682BB317
:10D8E000264A93F900001268032352782021002A67
:10D8F0000CBF08220922009301924FF461430022D9
:10D90000FCF762FA1E4B186080B11E4A01231370A7
:10D910002B701D4B1A681D4B1A6007E0184E3068BB
:10D92000FCF73FFA174B34601C702C7002B070BDCE
:10D9300044090020C014002040090020D814002011
:10D94000CC1B002045090020DD1400205C150020C0
:10D950004C15002050090020621500204C090020C1
:10D96000ECCC010864150020D429002068150020A3
:10D970005C0900207015002058090020540900207F
:10D980007415002078150020582900207C150020EF
:10D9900010B54B88DC0641BF2F4B14791B6853F838
:10D9A000244044BF2D4B43F820404B889B0641BF89
:10D9B000294B54791B6853F8244044BF274B43F844
:10D9C00020404B881C070ED5254B0C781B78B3EBF9
:10D9D000141FA1BF204BD4781B6853F82440A4BF68
:10D9E0001E4B43F820404B889B070ED51D4B0C78EF
:10D9F0001B78B3EB141FDFBF174B54781B6853F829
:10DA00002440DCBF154B43F820404B88DC070FD582
:10DA1000154C0B78247803F00F03A342DFBF0E4BA5
:10DA200014781B6853F82440DCBF0C4B43F82040AB
:10DA30004B885B070FD50B780C4903F00F0309786F
:10DA40008B42A1BF044B92781B6853F82220A4BFDD
:10DA5000024B43F8202010BD082300201A18002094
:10DA6000B7180020B5180020B4180020B618002000
:10DA7000254A0023F0B514681D461A462348244958
:10DA800003700B71661976884EB9675D3FB90370F4
:10DA900000230A714B7107781D461A460CE03605C3
:10DAA00048BF013205F1040503F1010348BFD2B2BA
:10DAB000802DDBB2E6D1EAE7E8B2B8420CD214F826
:10DAC0002500013506099E4200F00F00A8BF731C17
:10DAD0009042A8BF421CEFE74B718A71C2F3470125
:10DAE00002F001020A444C1E0A490B480A70C3F3B3
:10DAF000470203F00103134404700849501E084A0A
:10DB000008701370F0BD00BF84150020A818002015
:10DB1000CC1B0020B6180020B4180020B718002035
:10DB2000B5180020924B2DE9F04FDA68914D1A613B
:10DB30002A6891B0DA60904A0295136843F0200396
:10DB400013608E4B1A78012A0CBF002201221A7032
:10DB50008B4B1A78910740F14D838A490978042943
:10DB600040F248838849097801F0040101F0FF0080
:10DB700011B922F001021A701B78DB0702D408B138
:10DB800000F0C8FF8149CA79531C052293FBF2F2C9
:10DB900002EB82029A1A7E4BCA711F789200002310
:10DBA000DFF81082DFF8109258F82310794C91FBBF
:10DBB000F9FE04F1080040F823E0774844F8231008
:10DBC00000FB0E1142F2107091FBF0F004F1100610
:10DBD00080B226F813004FF0140C04F114060CFB6D
:10DBE000036C04F13C0A5AF823605CF802504CF8CC
:10DBF0000210761B314405264AF8231091FBF6F1FA
:10DC000009FB0E114434012F44F823104FEA830B13
:10DC1000444605D10238B0F5797F98BF4BF808101B
:10DC20000BB90123BCE7594E029BB2461868736DCD
:10DC3000C01A08F0D3FA594908F0DCFB029B4FF0F8
:10DC40007E511B680746736508F0BEFC08B94FF0AB
:10DC50007E574B4BCAF858701B78514E13F0010396
:10DC6000504D12D00DAA00924F4B0EAA01920CCB30
:10DC700094E8030000F0EAFD0D9A6421B2FBF1F292
:10DC80000E9B328093FBF1F300E033802B809AF8F7
:10DC90005C303E4D002B35D0A96D4FF07E5008F022
:10DCA000A9FB07462B6E2068C01A08F09BFA39467C
:10DCB00008F0ECFA08F0B0FC6B6E86B2606836B221
:10DCC000C01A08F08FFA394B196808F0DFFA3946A4
:10DCD00008F0DCFA08F0A0FCB5F96A2000B281185F
:10DCE000B5F968200220B31891FBF0F193FBF0F333
:10DCF00089B29BB2A5F86E10A5F86C30A5F86A1031
:10DD0000A5F8683001238AF85C30294B61681B88CC
:10DD1000206803F030031D4E264DCAF86410CAF87F
:10DD20006000002B00F0668206F17803009306F194
:10DD30007C030193326F736F00F088FD6B68706F26
:10DD4000C01A08F04FFA194B196808F09FFA08F04A
:10DD500063FC336F2A68C6F884009B1AC6F88030CB
:10DD60000B4B1B78012B29D0022B00F0E58041E200
:10DD70004426002058290020C01300205E140020F3
:10DD80004814002049140020B8350020CC1B002086
:10DD9000E8110020D41B0020806967FF00007A444E
:10DDA0005A1400205C140020601400205000002051
:10DDB000C41300204C14002080969800D6F88830B8
:10DDC000D6F8A4400293D6F8983004F100400393AB
:10DDD000D6F89C30B76D059308F01EFC81462046AE
:10DDE00008F01AFCD6F8A030BB4C0493BB4B06904D
:10DDF0001B684FF0000B0793B94E4FEA4B0356F8E0
:10DE00002B80A6F11402404632F81B50089308F00C
:10DE1000E9F9029908F03AFA08F0FEFB401B1FFAF4
:10DE200080FA283626F81BA00FFA8AFA504608F026
:10DE3000D9F9039908F02AFA08F0EEFB86B20AEB4A
:10DE4000080008F0CFF9059908F020FA394608F0E3
:10DE50001DFA216808F012F908F0DEFB484504DBE2
:10DE6000069B9842A8BF184600E0484608F0BAF959
:10DE7000206008F0D1FB079B304486B2987808F008
:10DE8000ADF9984908F002FA01464FF07E5008F0CB
:10DE9000B1FA394608F0F2F80146384608F0AAFA15
:10DEA00009906068D4F808A0C0EB080008F09AF95F
:10DEB000394608F09FFA514608F0DEF8099A014603
:10DEC000104608F0E3F90146504608F0D7F831351E
:10DED000ADB2622D01462061C4F80480A0600ED965
:10DEE000049808F0D3F908F097FB7F4AB0F5FA6F71
:10DEF000A8BF4FF4FA609042B8BF104600E000207F
:10DF000040F6B832064436B29642A8BF1646774A63
:10DF1000089B9642B8BF1646754A54F8140B9E5299
:10DF2000142202FB0BF273495050BBF1000F40F07A
:10DF300061814FF0010B5FE7684BB6F8AC401F689A
:10DF4000B36F3D8902935B089D4228BF1D4623B2F3
:10DF50009D4202DC1FFA85F90AE06749B06D08F0BE
:10DF600095F908F059FB20441FFA80F9A6F8AC9007
:10DF7000DAF87C60DAF8B040341B204600F022FD6D
:10DF800041F293130028D8BF40429842CCBF0020F2
:10DF9000012078B3204608F025F9584908F076F9B1
:10DFA000FDF7F1FF0446029808F018F901462046F3
:10DFB00008F06CF908F030FB40F6B83380B2AAF8EC
:10DFC000B40000B29842A8BF1846484B9842ACBF74
:10DFD0003018F01848F6A043984203DDA0F50C4035
:10DFE000A03804E00028BCBF00F50C40A030CAF8FF
:10DFF000B80001E0CAF8B860DAF8B8300026C3F516
:10E000000C502830039308F0EDF83C4908F03EF935
:10E010000446FEF729F80F902046FDF7B4FFDAF822
:10E02000BC30DAF8C8400593DAF8C0300E9004F13D
:10E030000040089308F0F0FA0490204608F0ECFA4B
:10E04000DAF8C430DAF858802A4C09900793730044
:10E0500048460A9308F0C6F80EAB53F8261008F0AD
:10E0600015F9DFF8A0A005463AF9160008F0BAF84D
:10E070000146284608F000F808F0CEFA05B2204B19
:10E08000B5F57A7FA8BF4FF47A759D42B8BF1D469B
:10E090000AF13C0AA8B22AF8160000B208F0A2F869
:10E0A0000599824608F0F2F808F0B6FA089983B2AA
:10E0B0005046069308F0EAF8414608F0E7F8216870
:10E0C00007F0DCFF08F0A8FA049B98421CDB099BD0
:10E0D0009842A8BF184618E024120020EC11002036
:10E0E0004C1C0020DB0FC94030F8FFFF48F4FFFF55
:10E0F000F61100204C1200200000C842D30237392C
:10E1000018FCFFFF381C0020049808F06BF8206012
:10E110008346B87808F062F8384908F0B7F8014645
:10E120004FF07E5008F066F9414607F0A7FF014620
:10E13000404608F05FF90B906068D4F808A0281AF0
:10E1400008F050F8414608F055F9514607F094FFA1
:10E15000DDF82CC00146604608F098F801465046AC
:10E1600007F08CFF656001462061A060079808F009
:10E170008DF808F051FA069B1434034458469A4629
:10E1800008F04AFA40F6B832504400B29042A8BFB4
:10E1900010461B4A0A9B9042B8BF1046194A1A49BA
:10E1A00098521422724342F801B00EB901264EE78C
:10E1B0003B792BB1039A642392FBF3F3134A138048
:10E1C0003B88029A124C9A420DD9D4F8B030E06FD5
:10E1D000C01A00F0F7FB42F2107380EAE072A2EB83
:10E1E000E0729A4206DD0B4B01221A70B4F8CC2083
:10E1F000064B1A8011B0BDE8F08F00BFDB0FC9409D
:10E2000048F4FFFFF611002024120020E411002042
:10E21000CC1B0020E811002010B507F0E3FF00211F
:10E22000044608F0EFF908B1204601E004F100408F
:10E23000054908F0DFF8054908F028F8FDF714FF54
:10E24000034B186010BD00BF8096184B35FA8E3C0A
:10E2500050000020F8B59A4B05461B68187818B195
:10E26000012800F06281D6E2242D964C0CD006D80D
:10E270000A2D00F0D7800D2D00F0D48040E12A2D2A
:10E2800006D02C2D04D03BE120706070A07048E1D6
:10E290008D4B6178277800208A4A58542FBB197813
:10E2A000D770472921D1597850291ED1997847290B
:10E2B00007D1D978472904D11979412901D1012100
:10E2C000D1709978804A522903D1D1784D2900F034
:10E2D000A48299787C4A472907D1D178532904D15F
:10E2E0001279562A04BF0322E270E278754E022AA0
:10E2F00038D0032A4BD0012A40F08380BA1E072A67
:10E300007FD8DFE802F004080F131A257E2A05F0F3
:10E31000DDFF606075E01B78532B72D163685B4250
:10E3200063606EE005F0D2FFA0606AE01B78572BB7
:10E3300067D1A3685B42A36063E01B78302B634B1B
:10E340001A788CBF42F0020222F002021A7058E0E2
:10E35000002006F01BF8207353E0002006F016F8AA
:10E36000E0814EE0072F06D0082F4AD1012006F0A9
:10E370000DF8708245E0012006F008F841F21843DC
:10E3800058434FF47A73B0FBF3F0308239E0022F38
:10E3900007D0032F0AD1002005F0F8FF4C4B18706E
:10E3A0002FE0002005F0F2FF30752AE029D93A1F4E
:10E3B0009210337D0132D2B2013B02EB8303DBB218
:10E3C000102B1ED8F91EC2F1010201EB8202D2B25B
:10E3D000012A0BD0042A11D100205E1E05F0D6FFC1
:10E3E0003C4B002298553C4B9A5507E03B4A5E1E39
:10E3F0000020935505F0CAFF394B9855A3690133A6
:10E40000A361304B2A2D18BF9A7807F101074FF00E
:10E4100000000CBF01225540277060700CBF1A77B6
:10E420009D707EE0207F002847D02E4B13F8012DF1
:10E430002D495A708B42F9D1234A224D13785278D4
:10E44000402B85BF373B1B011B01DBB298BF03F09C
:10E45000F003402A8CBF373A303AD2B21344A27844
:10E46000DBB29A4226D121230B70E8782B6A01286F
:10E4700003F101031C4A2B620AD002281CD172232B
:10E4800013702A8A194B1A806A8A194B1A8013E072
:10E49000672313700D4B1B789F070ED5154B6A68C9
:10E4A0001A60AA685A602A7B134B1A70EA89134BC8
:10E4B0001A8002E03F230B7000200023237730E016
:10E4C000642600209C1C0020C52900204814002040
:10E4D00074140020A5140020951400207514002049
:10E4E0008514002010060020FC0500205614002092
:10E4F000581400204C14002049140020541400200B
:10E500006378207F0E2B9FBFA84A591C5170A84AE0
:10E5100098BFD554A54A18B993785D40957000E02E
:10E520000020003018BF0120F8BDA04B002293F856
:10E530002410082900F26F81DFE801F0050C101AA1
:10E540002B3B5E788500B52D40F0658183F8252052
:10E5500001224EE0622D08BF02224AE0032283F826
:10E56000242083F8265083F8275083F8285052E15E
:10E57000042283F8242093F8272093F828102A44B3
:10E58000D2B283F827200A4483F8282083F8295040
:10E5900041E1052283F8242093F8272093F82810DE
:10E5A0002A44D2B283F827200A4483F828205D85C4
:10E5B00031E1062283F8242093F8272093F82810CD
:10E5C0002A44D2B283F827200A4483F828205A8D9F
:10E5D00002EB0525ADB2B5F5AC7F82BF734A0121D0
:10E5E00082F8251000225D859A85002D40F0138168
:10E5F000072283F824200EE193F8272093F82810AF
:10E600002A44D2B283F827200A4483F828209A8D1E
:10E61000B2F5AC7F3EBF6549891881F830500132B0
:10E62000598D92B291429A85E2D9F4E0082283F89A
:10E63000242093F82730AB4200F0ED805B4B0122A1
:10E6400083F825200FE05B4C83F8242014F8012D7B
:10E650006270594A9442F9D193F82810534AA9425A
:10E6600006D03F232370554A536801335360D2E0EC
:10E67000116A92F825000131116210B13E23237016
:10E68000C9E02121217092F82910062941D004D82F
:10E69000022907D0032923D0F8BD122959D03029E7
:10E6A00067D0F8BD502121704549546B4C60946B84
:10E6B0000C60116C4FF47A7491FBF4F1414C2180A1
:10E6C00092F88811404A19B1117841F0020102E034
:10E6D000117821F002011170012283F889218CE068
:10E6E0005321217092F83510CE0705D592F83420C9
:10E6F000D51E6A426A4100E0024602F0010183F839
:10E700008811002A79D130490A7822F002020A7071
:10E7100073E04F21217092F83B10CC0705D592F899
:10E720003A20D11E4A424A4100E0024602F001016D
:10E7300083F8881122B924490A7822F002020A706B
:10E7400093F85F10214A1170B3F85C10204A1180D1
:10E7500053E056212170546C1E490C8042F2107413
:10E76000916C91FBF4F11C4C2180012182F88A11FB
:10E7700043E04921217092F83410184A102988BFCB
:10E7800010211170164914780022A24232D20E7A5A
:10E79000144D56554E7A144D5655CE7A134D565546
:10E7A00011F80C6F124D56550132EEE79C1C0020FB
:10E7B000C529002010060020FC050020442600206A
:10E7C0004C14002054140020481400204914002048
:10E7D00098030020561400205814002074140020C0
:10E7E000CC1C0020751400208514002095140020F6
:10E7F000A51400209A6901329A6193F889310B4A75
:10E8000093B192F88A317BB1002182F8891182F8A4
:10E810008A111846F8BD0020F8BD1279432A7FF40A
:10E8200058AD0222E27054E5F8BD00BF9C1C0020E8
:10E830000449054B0968002218705A6199611A77DA
:10E84000704700BF58290020442600202DE9F047DA
:10E85000101A0E461F4607F0C5FC0446B81B07F009
:10E86000C1FC4B4B099D196807F010FD21468046FD
:10E87000204607F00BFD41460646404607F006FDE0
:10E880000146304607F0FAFB09F0EEF8414907F07F
:10E89000FDFC07F0E7FE04F10046089B28F0004766
:10E8A00026F0004918604946384607F0ABFE08B923
:10E8B0004C4600E03C462046002107F07BFE60B954
:10E8C0003846494607F080FE08B9484600E0384619
:10E8D000214607F08FFD044600E0002420462E4923
:10E8E00007F0D4FC2D4907F0C7FB214607F0CEFC0A
:10E8F0002B4907F0C1FB214607F0C8FC294907F066
:10E90000BBFB214607F0C2FC274907F0B5FB2749AE
:10E9100000F1004A204607F0B9FC254907F0AEFB9C
:10E92000214607F0B3FC4FF07E5107F0A7FB0146EC
:10E93000504607F05FFD39460446484607F062FE40
:10E9400020B121461B4807F097FB044640460021B2
:10E9500007F03AFE20B12146174807F08DFB044628
:10E960003046002107F030FE08B104F1004413499D
:10E97000204607F08BFC124907F080FB07F04CFEA5
:10E980000028BCBF00F50C40A0302860BDE8F0872F
:10E99000500000202C7D8E3F39094E3DE3B59E3E50
:10E9A00088FA163E45FE7F3FA7DFA83499FB243F37
:10E9B00069A2163EDB0FC93FDB0F4940A00CB345EF
:10E9C00000A00C4644F25063984203DDA0F50C40D1
:10E9D000A0387047034B9842BCBF00F50C40A030F4
:10E9E000704700BFB0B9FFFFF7B50368174C184D6B
:10E9F00023600B68174E63600068FFF70DFC95E815
:10EA00000300154B0196009394E80C00FFF71EFFDE
:10EA10003668124B60681E606B68114FC01A07F0B1
:10EA2000E1FB104B196807F031FC07F0F5FD2A688F
:10EA3000236878609B1A3B600B4B1E600B4B1B6876
:10EA4000DA880B4B1A8003B0F0BD00BF3C1C0020DD
:10EA50004C140020481C0020441C0020841C002072
:10EA60004C1C0020500000207C1C0020EC110020D9
:10EA7000781C002070B50446407907F0AFFB1E49B2
:10EA800007F0B8FC1D4D1E4E2860E07B07F0A6FB8A
:10EA9000194907F0AFFCEE606860A07907F09EFBB3
:10EAA000184907F0A7FC184D2860207C07F096FB5A
:10EAB000114907F09FFC6860A07E07F08FFB1349A7
:10EAC00007F098FCEE60A860E07907F087FB0D493D
:10EAD00007F090FC0E4D2860607C07F07FFB064934
:10EAE00007F088FC6860E07E07F078FB074907F0D4
:10EAF00081FCEE60A86070BD0000C842541C00207C
:10EB00000000FA4400002041641C002000007A4408
:10EB1000881C002010B50E4C23789B0717D50D4B91
:10EB20001B78042B13D90C4A0C4B106852681860E0
:10EB30005A60FFF771FB0A4B0A22B3F9043093FBCA
:10EB4000F2F3084A1380237843F00103237010BDC9
:10EB500048140020491400204C14002060140020A8
:10EB600028140020981C0020094A137818441346E2
:10EB7000C0B210F0800F18BF80381070054A1978A5
:10EB80001378994201BF00231370014A1370704734
:10EB90006D2600206C26002010B50A4B0A4A1B780F
:10EBA00042609C18094A046012789A4225BFD31A21
:10EBB0000B60C3F1800300232EBF4B600B604A60E3
:10EBC00010BD00BF6D2600206E2600206C260020A0
:10EBD0001FB5684602A9FFF7DFFF044B02981B68C8
:10EBE00003440398184405B05DF804FB6009002055
:10EBF0002DE9F04F814689B00293002303910492DE
:10EC00000193049A934207DA039A019952F8232058
:10EC1000013311440191F4E7029B019D002B57D170
:10EC200003F06AFB002853D102987FE00222414E94
:10EC30008DF81C201A0C4FF480578DF81D200620EB
:10EC40001A0A8DF81E208DF81F3003F07DFB7761C6
:10EC500006213948F7F741FD384B01223761C84694
:10EC60001A70776126463448002107AA0423F7F773
:10EC700006FD039F4FF0000A049B9A451DDABC462F
:10EC800057F8043B4FEA8A0B002B48D0B34235D3E8
:10EC900033462948002159F80B20CDF814C0F7F766
:10ECA000EEFC59F80B30DDF814C0334449F80B3052
:10ECB000DCF800309E1BCCF800601E4B4FF48052F5
:10ECC0001A611F4A2D1B13681C44029B14605BB31E
:10ECD00055B31B4B1B68DCB22A19B2F5807F194A69
:10ECE00088BFC4F58074D26898BF2C4693429DD3E8
:10ECF000154A00231370154A137015E0D8F8002048
:10ED00000D480021F7F7BBFC57F8043CD8F8002069
:10ED1000F61A1344C8F80030002347F8043C0AF1FF
:10ED2000010A08F10408A7E7019B581B09B0BDE8D8
:10ED3000F08F00BF000C0140003800405D0900204A
:10ED4000600900200C0000206C2600206D260020A9
:10ED500030B50B4C0B4D22782B7885B09A420CD0F5
:10ED6000684602A9FFF718FF0123684602A902229C
:10ED7000FFF73EFF00232B70237005B030BD00BFAE
:10ED80006D2600206C26002030B50E4D0E4C2A78E2
:10ED9000237885B09A4211D0684602A9FFF7FCFE9D
:10EDA000002302A902226846FFF722FFFFF7DCFEDC
:10EDB00020782B781B1A5842584100E0012005B0FA
:10EDC00030BD00BF6D2600206C260020054A064B92
:10EDD00010781B7883422EBF181AC0F18000C0182B
:10EDE000704700BF6D2600206C26002070B50F4CC8
:10EDF0000F4E4FF4805545F2082003F0A5FA062186
:10EE000065613046F7F769FC0A4B012225613046FF
:10EE10001A70C7216561F7F760FC074A0023256176
:10EE20001370064A1370064A136070BD000C01404F
:10EE3000003800405D0900206C2600206D2600206F
:10EE4000600900200148024900F0D2B800080040E3
:10EE5000FC2700200148024900F0CAB80004004025
:10EE6000D42700204FF08040014900F0C1B800BF16
:10EE7000AC2700200148024900F0BAB8002C01403C
:10EE8000842700200148024900F0B2B8002C01405C
:10EE900084270020026D70B515880446ADB2A9061E
:10EEA00013D5036B8BB9C36A1BB1908880B29847A6
:10EEB0000BE0E169928840694E1CD2B2E66142548F
:10EEC000E169E268914228BFE3612B0613D5636ACA
:10EED000A26A9A42236D0AD0511CA069A162825C89
:10EEE0009A802369994206D30023A36270BDDA6831
:10EEF00022F08002DA6070BD026B0346C16810B573
:10EF0000406942B11A6C8C1A013A08BF0A46005D8A
:10EF10001A64C0B210BD1A6A805C01328A4228BFEE
:10EF20000022C0B21A6210BD436B13B190F84400C6
:10EF30007047836A406A1B1A584258417047426AB8
:10EF4000816A03698A4238BFD218521A416B21B1D3
:10EF500049680A44591E8A4203D2013B981AC0B23A
:10EF6000704700207047036B13B15B68016C01E0D0
:10EF7000C369016A8B423CBFC2689B18581AC0B271
:10EF80007047836A8169426B1944D160416A994232
:10EF900097BF0169CB1ACB1A536096BF0023536009
:10EFA00083624FF0000380F84430136888BF8162A9
:10EFB00043F0010313607047436A8269D154436A86
:10EFC00002690133934228BF00234362436B1BB1A4
:10EFD0001B68DB0705D4D4E7026DD36843F08003D8
:10EFE000D36070474171FEF723B88160FEF720B807
:10EFF0002DE9F04105460E46078A83899BB21F40E2
:10F00000002F37D0B7FA87F24FF00043D340DB43ED
:10F0100099B21F40A2F11B032982042BF0D8DFE82C
:10F0200003F0221F1C190300746A24B1013C002361
:10F03000A4B2736201E0AC8DA4B2D6F82080B8F11E
:10F04000000FDDD0D8F80030404621469847D8F868
:10F050000480F4E73068A98E08E07068298F05E025
:10F06000B068A98F02E0F068B5F84010036889B273
:10F070009847C5E7BDE8F081254B10B55A43254BAD
:10F08000254C1B680139B3FBF2F20388013AA04218
:10F0900089B292B29BB212D004F50064A0420ED0A5
:10F0A000B0F1804F0BD0A4F59834A04207D004F5FE
:10F0B0008064A04203D004F58064A04202D123F012
:10F0C00070039BB2154CA04206D004F58064A042A8
:10F0D0001CBF23F440739BB203800F4B8185984281
:10F0E00002850FD003F5006398420BD003F540630F
:10F0F000984207D003F58063984203D003F58063FC
:10F10000984201D1002303860123838210BD00BFF2
:10F1100040420F00A0030020002C014000100040DE
:10F1200073B505460068FFF7A7FF2A680124138816
:10F1300000269BB243F001031380EB7A01A88DF8FF
:10F1400004308DF805408DF806608DF8074005F015
:10F150006FF8EB7A1B2B0BD1192301A88DF8043023
:10F160008DF805408DF806608DF8074005F060F8D1
:10F1700002B070BD0C4B800A98420CD004D8B0F598
:10F18000801F0CD101207047084B984205D04933AD
:10F19000984206D003E00220704703207047FE200B
:10F1A00070470020704700BF0100100002001000EF
:10F1B0002DE9F84304680746204688469146FFF744
:10F1C000D9FF03284BD8BA7A9108B8F1000F06D1BD
:10F1D000A589AEB202258D4026EA0505A5810A2340
:10F1E00003FB00131F4A42F82380043342F82390A4
:10F1F000B8F1000F07D0BD7AA189AD080223AB405A
:10F200000B439BB2A3812823434303F12001114404
:10F21000EFF31286502585F3128803F10C051C3399
:10F220001544134455F8047F17B10F602968043161
:10F230009D42F7D100230B60F3B283F3118828239A
:10F2400003FB0020036A23B1A3899BB243F00103AF
:10F2500004E0A38923F001031B041B0CA381BDE878
:10F26000F88300BF84270020004813E6281E0020F2
:10F2700000480FE67C1E00200A4B4FF400525A60F3
:10F280004FF6FE730848D0F8882011680B401360D1
:10F29000826FC36F9A4201D0543072E6012380F826
:10F2A0009830704700000240281E00202DE9F043EE
:10F2B0001E46A04B8DB09842894690469DF85070EE
:10F2C0005ED19D4B9D4AC3F85C805A6503F1A8024C
:10F2D0009A6603F5D472DA664FF480721A665A663B
:10F2E000974AC3F8A400C3F88820A2F54842403AE0
:10F2F000C3F89C20934B9A6942F480429A615A6900
:10F3000042F001025A6102238DF803303A074FF4AC
:10F310000073ADF8003001D51C230FE0B30706D50C
:10F320001823894869468DF8023002F0EFFEF50790
:10F330000AD54FF48063ADF800304823824869460F
:10F340008DF8023002F0E2FE01240E23002501A810
:10F350008DF804308DF805408DF807408DF8065083
:10F3600004F066FF252301A88DF805408DF80740BD
:10F370008DF804308DF80650744C04F059FF50E0BD
:10F38000734B984240F0D1806B4B6C4AC3F80880B5
:10F390001A6003F52A725A6103F56A729A614FF492
:10F3A0008072DA601A616B4A18659A64DA64654B98
:10F3B0003C07DA6942F48022DA619A6942F0080275
:10F3C0009A614FF002038DF803304FF48063ADF87B
:10F3D000003001D51C230FE0B00706D518235E4886
:10F3E00069468DF8023002F091FEF1070AD54FF41C
:10F3F0000063ADF800304823574869468DF8023065
:10F4000002F084FE27238DF804300022012301A896
:10F410008DF805308DF806208DF8073004F008FFD0
:10F42000454C0025012384F844302562E561A5623E
:10F430006562C4F82C906671C4F80880A7712046F4
:10F44000FDF7F6FDF20735D5236B002B2AD001A876
:10F45000FBF7ACFAE36C206B01934FF480530A93F3
:10F4600080230693E3680B95049320230993636933
:10F4700005950293079508950395FBF7C2FA01A934
:10F48000206BFBF7A0FA226B216D136843F0010398
:10F4900013608B8A9BB243F040038B8253689BB20C
:10F4A000236407E04FF6DF72236D1A80DA6842F0BA
:10F4B0002002DA60B30730D5636B002B28D001A897
:10F4C000FBF774FAA36C002501934FF480530A9361
:10F4D000802306932369606B0493102303930B9599
:10F4E0000595079508950995FBF78BFA606B01A9BF
:10F4F000FBF769FA636B1A6842F002021A60226D28
:10F500005D605D60938A9BB243F08003938204E068
:10F51000226DD36843F08003D360226D2046938927
:10F520009BB243F40053938100E000200DB0BDE88E
:10F53000F08300BF00380140281E002058B70108A2
:10F540004400024000100240000801407C1E0020E0
:10F550000048004004480040000C014010B5002461
:10F56000054B53F8340004F0FBFA0134034804F06F
:10F57000F7FA1E2CF4D110BD7CB701086CDB010832
:10F5800070B5054628460BF041FA064658B91A4BA5
:10F590001A485A791A4BBDE8704003EB8203D3F83E
:10F5A000EC10FCF7C2BC2846164932460BF036FA7E
:10F5B00060B9154804F0D4FA144C54F8041F19B17A
:10F5C0001348FCF7B2FCF8E7124805E00024124BA0
:10F5D00053F8241021B91148BDE8704004F0C0BAB6
:10F5E000284632460BF01AFA01340028EFD1024BBC
:10F5F0000B4D5C71C6E700BF6C2A002078D3010870
:10F600007CB7010884D3010889D3010868B80108D0
:10F610009CD301086CDB01086CB8010894D2010886
:10F62000A9D00108F0B585B004460BF0EFF9082821
:10F6300026D1621EE01D1F4912F8013F09681944D6
:10F64000497801F00301022908BF203B8242137070
:10F65000F1D1254604F1080715F8016B164831462B
:10F660000BF0C7F920B1284631460BF0C2F910B1B2
:10F67000F9F7C4FF1CE0BD42EED1204604F03EFF86
:10F680000E4804F06DFA00230D4A04A91A4492F8BA
:10F6900088210A440849595C0133082B02F80C1CE4
:10F6A000F2D10023074801A98DF80C30FCF73DFC8E
:10F6B00005B0F0BDA40300202DE70108A0D3010888
:10F6C0006C2A002098DA01081C4B1D4C1D6880B57F
:10F6D0002068FAF75BFB2846FAF758FB2068417967
:10F6E0008B0703D441F0020103F07AF9154B08228D
:10F6F0001A61206803F080F990B1124E08237361FB
:10F700000F4B186803F075F90746FEF7A3FD08B123
:10F71000FEF708FA2846394603F071F908233361E9
:10F72000284603F069F90028E3D02846266803F04C
:10F7300060F90146304603F062F9DAE72C2900202F
:10F74000D0220020000C01402DE9F04705460BF0C7
:10F750005DF9314E0446D6F8088090B92F4804F080
:10F76000FFF92F4B53F8241049B10123A34013EAAA
:10F77000080F02D02B48FCF7D8FB0134F1E72A48E8
:10F7800022E02846294922460BF048F958B9284872
:10F7900004F0E6F9274C54F8041F0029EFD0214863
:10F7A000FCF7C3FBF7E72B784FF000092D2B03BFC5
:10F7B000013504F1FF344FF0010A4FF0000A184BF5
:10F7C00053F8297027B91C48BDE8F04704F0C8B9C0
:10F7D0002846394622460BF021F9C8B9012000FA23
:10F7E00009F0830501D51548EEE7BAF1000F03D003
:10F7F000FCF764FC124803E040EA0800B0601148DE
:10F8000004F0AEF93946BDE8F0470F48FCF78DBB70
:10F8100009F10109D3E700BF6C2A0020A6D3010833
:10F82000D8B801089CD301086CDB010884D3010817
:10F83000B0D30108D4B8010894D20108BCD30108A0
:10F84000CAD30108D3D3010897DA010810B50848D4
:10F8500004F086F9074B00241C715C63064B1C7096
:10F8600003F076FA04F042FB044B1C6010BD00BFAD
:10F87000DBD30108D0220020BA3500202C2900203B
:10F8800070B5064600240C4AA5182B7903F0300306
:10F89000B3420AD1A1580948FCF747FB284600218A
:10F8A00004F0DFF8064804F05BF940F6BC4314347A
:10F8B0009C42E8D170BD00BF2CBF010807D40108ED
:10F8C0006CDB010808B50848FCF72FFBFFF78EFA40
:10F8D00002F012FD18B9642002F0C1FFF8E70348F6
:10F8E000BDE80840FCF721BB11D401081ED4010873
:10F8F0002DE9FF410A48068885684488B0F80480ED
:10F90000C768FFF765F9CDF800800290019731468E
:10F910002A4623460348FCF708FB04B0BDE8F08103
:10F920000C00002026D40108F0B504788BB0054601
:10F930000CB1002436E04B4B19680E2303FB041175
:10F94000B1F91D51B1F91921B1F91B31009591F8A7
:10F95000205101F58C70019591F8215101F59071BC
:10F96000029590F90700039091F902103E48049126
:10F9700021460134FCF7D9FA082CDCD170E02D2B9C
:10F9800014D1072C1BDC284607F0E2FB0AAB661CEF
:10F9900003EB440424F8100C15F8013F303B092B0D
:10F9A000FAD934462B78002BE9D104E0A3F13002D8
:10F9B000092A09D8E5E7082CBDF8182009D00BB0B2
:10F9C000BDE8F040F9F71ABE202BF8D101352646E4
:10F9D000E7E7072AF3D840F2DC55BDF81A00214BBF
:10F9E000A0F2EE2189B2A9421B68E8D8BDF81C102C
:10F9F000A1F2EE24A4B2AC42E1D8BDF81E6004B27C
:10FA000037B2A742DBDB0DB2AF42D8DCA542D6DB72
:10FA1000BDF8247007F16404A4B2C82CCFD8BDF897
:10FA200026E00FFA8EF4112CC9DCBDF82050B42D5D
:10FA3000C5D8BDF82240B42CC1D812B24FF00E0C7C
:10FA40000CFB0233A3F81901A3F81B11A3F81D61E5
:10FA500083F8205183F8214183F81F7183F822E154
:10FA60000BB0F0BD0C14002083D40108F0B504469F
:10FA70008FB020460AF0CAFFC5B21DBBAE4804F0E5
:10FA80006FF8AE4C94F8D21009B9AD4853E049B2C2
:10FA900094F8D02094F8D130009194F8D310A9486C
:10FAA000019194F9D4100734029194F9CE10039186
:10FAB00094F8CF10049129460135FCF736FA102D41
:10FAC000E0D1E2E72046A04905220AF0A7FF05465B
:10FAD000B8B929469D4870220AF058FF28469C4B29
:10FAE00019680E2303FB001301300022082883F855
:10FAF000232183F8242183F8252183F82621F0D1BE
:10FB000018E12046934904220AF088FF0546204662
:10FB1000002D4AD120210AF06CFF002800F00A8154
:10FB2000461C30460AF072FF2C4607468A4B53F8B3
:10FB300024502DB989480FB0BDE8F040FCF7F5B965
:10FB400030462946FAB20AF069FF01340028EDD1A7
:10FB50007A4A164602F17001002382F8D63082F804
:10FB6000D23082F8D13082F8D03007328A42F3D1D5
:10FB70007B4901EBC40191F8B421934210DAD1F82A
:10FB8000B871C3EBC302B0183A44176800F1D00152
:10FB9000C0F8D07090880133888092798A71E7E745
:10FBA00029467048FCF7C1F995E06F4907220AF031
:10FBB00035FF05462046002D49D120210AF019FFC6
:10FBC00006460AF023FFC4B26CBB6848FCF7ADF9E7
:10FBD000214667480134FCF7A8F90E2CF8D15848A3
:10FBE000FCF7A3F9002463482146FCF79EF90025A1
:10FBF000574A012311680E2202FB0412D2F8232176
:10FC0000AB4013425C4B5D495D4808BF1946013566
:10FC1000FCF78BF90E2DEBD149480134FCF785F93F
:10FC2000082CE0D186E03046564907F095FA2C467C
:10FC3000002852D0022C55D007F08AFA06AB43F8C0
:10FC400024005049002007F087FA0134F0E74D49BD
:10FC500007F082FA002460B1082C3ED007F078FA51
:10FC600006AB43F824004749002007F075FA013439
:10FC7000F1E7082C31D1069B0F2B2ED8DDF81CE0C4
:10FC8000BEF1070F29D8089F0D2F26D8099E06F12F
:10FC90006402C82A21D80A9DFF2D1ED80B9864281B
:10FCA0001BD80C99642918D8884216DA0D9C032CAD
:10FCB00013D8224AC3EBC303134483F8D0E083F87C
:10FCC000D17083F8D26083F8D35083F8D40083F8DE
:10FCD000D51083F8D6402C4CCBE60FB0BDE8F040F1
:10FCE000F9F78CBC069B072B20D807990D291DD846
:10FCF0000278722A0DD06E2A18D1154A0E20126889
:10FD000000FB032301228A40D3F8231121EA0202D7
:10FD100009E00F4A0E20126800FB032301228A40EB
:10FD2000D3F823110A43C3F8232101E0F9F766FC55
:10FD30000D4C9EE60FB0F0BDABD401086C2A00203C
:10FD40006CDB0108D6D4010864D201083C2B0020EA
:10FD50000C1400208FD201086CB8010894D201085D
:10FD60007CB70108A3D20108A3D40108B5CE0108CD
:10FD7000F2D40108B0DA0108B1DF0108F7DE0108AA
:10FD8000F7D40108FBD40108A9D001082DE9F743F5
:10FD9000047805468CB9324D95F8AB12B5F8A82217
:10FDA00095F8AA322F48009121460134FCF7BDF89E
:10FDB000102C05F10405EFD14EE007F0C9F90F282A
:10FDC000044636DC284620210AF013FE264EE4B213
:10FDD000D6F83880451CA4000027284607F0B8F95B
:10FDE0005FFA87F9B9F1010F83B208D0B9F1020FB8
:10FDF0000BD0B3F5B47F24D2B26B13530AE0FF2BC0
:10FE00001FD8B36B2344987004E0FF2B19D8B36B51
:10FE10002344D87028462C210AF0EBFD054608B192
:10FE2000013502E0B9F1020F0BD10137032FD4D114
:10FE300012E00E4800210F2203B0BDE8F043F9F7AD
:10FE40005ABB08EB0400002104220AF09FFD03B016
:10FE5000BDE8F043F9F7D2BB03B0BDE8F08300BFC3
:10FE60006C2A0020FDD40108D022002022D20108F3
:10FE70002DE9F04FAB498BB004460AF08FFDAA493B
:10FE8000002820460CBF012507250AF087FDA74959
:10FE90000028204608BF02250AF080FD002808BF80
:10FEA0000425E90740F1E780A14803F059FE00204E
:10FEB00003F02CFC9F4CA04803F052FE9F4803F037
:10FEC0004FFE62799E4B9F4803EB8203D3F8EC1000
:10FED000FCF72BF89C48FCF728F826460027D6F8B4
:10FEE00010800021404606F065FB20B19748FCF7E2
:10FEF0001CF8002669E039469548D6F814B0D6F8C3
:10FF000018A0D6F81C90FCF710F84046002106F027
:10FF10005BFB10B1202003F01BFE06A94046FBF757
:10FF20009FFE01468B48FCF700F85846002106F07A
:10FF30004BFB10B1202003F00BFE06A95846FBF73F
:10FF40008FFE01468348FBF7F0FF5046002106F084
:10FF50003BFB10B1202003F0FBFD06A95046FBF748
:10FF60007FFE01467B48FBF7E0FF4846002106F094
:10FF70002BFB10B1202003F0EBFD06A94846FBF750
:10FF80006FFE013701467448FBF7CFFF0C2F06F1D7
:10FF90001006A4D1AAE749B294F8D02094F8D13041
:10FFA000009194F8D3106D48019194F9D41007345E
:10FFB000029194F9CE10039194F8CF100491314638
:10FFC0000136FBF7B2FF102E03D094F8D2100029AF
:10FFD000E1D1634803F0C4FD564B624C9F6854F86E
:10FFE000041F19B16048FBF7A0FFF8E70E465F4B0E
:10FFF00053F826404CB10123B3403B4203D05C4848
:020000040801F1
:100000002146FBF792FF0136F1E75A4803F0A8FDBD
:100010002146484B0AAA0B4493F888311344564AA8
:100020008A5C0131082903F8102CF2D106A90024BA
:1000300052488DF82040FBF778FF514803F090FDBF
:100040005048F9F7BDFF504803F08AFD4D48F9F7D5
:10005000DBFA4E4803F084FD4A48FFF797FE4C4810
:10006000FBF763FF2046FFF70BFC4A4803F078FDDF
:100070004448F9F7EFFDAA0739D5474803F070FD6A
:10008000464803F06DFD3F4803F0A4FB444803F0ED
:1000900067FD3C48F9F73CFA424803F061FD3948F6
:1000A000F9F72AFD4048FBF740FF3648F9F7B8FB5F
:1000B0003E4803F055FD3348FFF736FC00260E2777
:1000C000774300243A4A0123D26BA3403A44D2F842
:1000D0000A2013421DD101340E2CF3D10136082E13
:1000E000EDD12B48FBF721FF1020FFF7C9FB6B0771
:1000F00015D5304803F034FD2F4803F031FD214879
:1001000003F042FB2248FBF710FF2020FFF7B8FB6B
:1001100005E0314622462948FBF707FFDBE70BB035
:10012000BDE8F08F11D50108E1E2010818D50108FA
:100130001ED501086C2A00202CD501083ED50108E7
:100140007CB701084AD5010855D5010862D50108D8
:100150006FD50108B4CE010898DA010887D50108E7
:1001600077D50108D4B80108A6D50108D8B8010888
:10017000B4D50108C1D501082DE70108CDD5010886
:10018000D6D50108A9D00108E5D50108F1D50108A7
:100190006CDB0108FFD501080CD601081FD6010849
:1001A0002DD6010837D6010846D6010854D60108D5
:1001B000D022002060D6010871D6010883D601083C
:1001C0002DE9F04F9E498BB00B7813F0010F03F02F
:1001D000040200F09A81002A40F0A4819948066840
:1001E00016F0806640F09E81980700F18E8143F002
:1001F00004030B70944B0A22B3F90430934F93FB22
:10020000F2F3934A13803B681B0340F15F81914BEB
:1002100080201E7004F0E2F908B103F09DFB8E4BC4
:100220001D789846012D40F051818C4C94F8D627CA
:1002300022B194F8D7370BB19A4203D3012384F843
:10024000D6370FE01846114630B191FBF0FE00FBA7
:100250001E1E01467046F7E792FBF1F293FBF1F3A5
:1002600084F8D62784F8D73794F8D837012B82BF83
:100270007A4B002283F8D82794F8D897B9F1000F69
:1002800003D0B9F1010F32D03BE0802002F0CCF96D
:100290008246002835D08021F9F734FF704B9AF858
:1002A000062018706F4B022153F822309AF9000093
:1002B000B3F5613F0CBF022200228DE806004A46DA
:1002C0008021F9F781FD684B4FF4FA721860674B93
:1002D0001B6803EB4303B3FBF2F31BB1402BA8BF36
:1002E000402300E00123624A137070B909E0614BBA
:1002F000DB6833B101F068FC18B95D4B40221A701D
:1003000003E0002388F80030E0E0DFF854810021AA
:1003100008F1040014220AF039FB08F12403C8F89C
:10032000183008F1A003C8F81C3008F58E73C8F81F
:100330002030514B94F892111A88504B00291A80A2
:100340003B6894F88411C3F3C03218BF01220692AF
:10035000C3F3400803F40062494B05911B68494808
:10036000C3F3800CC3F3C00963790078A3F11907C4
:1003700079427941012B14BF0B46012394F8D6171B
:10038000049394F8D737039099423F4928BF00233C
:100390008A46D1F800B038BF01236F1EFFB2791E24
:1003A000132944D8DFE801F00C0C0C0C0C0C0C0CDD
:1003B0000AB8BA3234463E12121240460499AEE0F0
:1003C0000399B942B4BF002401242FE09BF8001028
:1003D000022914D1B91E5BF8210000210992CDF841
:1003E00020C0079306F0E6F84FF00104079BDDF804
:1003F00020C0099A08B14FF00004E4B216E00BEBFC
:1004000007014C79003418BF01240FE0414686E013
:1004100022B10599481E4142414100E0114601F0D8
:1004200001017CE006997AE0194678E014B10121D7
:10043000B9400E43142D29D80135EDB2ADE700BF08
:10044000B8350020C81300202814002028350020CB
:10045000E611002060320020691000206C2A002084
:1004600010230020ECCC01086C1000202035002067
:10047000741000200C000020601700208410002061
:10048000C0130020802700200C140020DAF80000A0
:10049000264B192179301E6002F066F9244B254A5B
:1004A0001870002313602449244A09681380244AE1
:1004B000A2F89831C2F89C11224A1360224A1360B4
:1004C000224B1B685360224B02221A701F4B214A99
:1004D0001B6892F8E2214FF47A7101FB02331E4A45
:1004E00013601E4B1B681A0609D51D4B1B789B0712
:1004F00005D51C4B1B78042B01D9062000E00520F4
:100500000BB0BDE8F04F02F0DBB95AB901200BB0D7
:10051000BDE8F04F02F00CBA494600E06146002900
:1005200085D189E70BB0BDE8F08F00BF80100020B7
:10053000901000208C10002000290020881000203E
:10054000102300207010002078100020582900206F
:10055000691000206C2A002094110020283500200A
:10056000481400204914002010B5154A1378590783
:1005700025D523F004031370124B1B681B0319D5F8
:10058000114C2378A3F10802012A0BD8FF20002187
:10059000FAF776FD0D4B1A680D4B5A6001F044FBDB
:1005A0000A2306E0012B05D90A2B03D001F022FB18
:1005B000012323700420BDE8104002F081B910BD72
:1005C000B835002028350020691000205829002067
:1005D0007810002008B5054B93F8A03103F005030F
:1005E000052B01D102F090FBFEE700BF1023002095
:1005F0007047704770477047FEE7FEE7FEE77047B9
:1006000030B50024E3B293420DD2030F092B94BFFF
:100610003033373301F81430002501EB4403000177
:100620005D700134EEE730BD0E4B0F4A1B683E296A
:100630009BB203EBC00002444FEA420209D94B09C6
:10064000C80604BF03F1FF339BB29B0243F400438F
:1006500004E04B08C90748BF01339B0211681360CF
:10066000704700BF505C00400630002030B50022CB
:1006700040F60F7102F1805303F5B8539B001D68DB
:1006800042F4004444F08004294001322143042A0A
:100690001960EDD1024B40F08000186030BD00BF02
:1006A0004C5C00402DE9F347884D894C2B68894EFE
:1006B0009BB22380228831880A40970507D54FF6E0
:1006C000FF53854A2B6013780133DBB21370238804
:1006D0000B40180440F100830023ADF802302B6872
:1006E0007B4F9AB21804228040F1F6823B8803F0D7
:1006F0000F03BB70002B40F0C182784A13689BB295
:10070000BB80BB8803F03003FB80BB8803F44053FD
:10071000BB804BF6BF7311680B4083F4005383F02A
:10072000200343F4004343F0800313603B88D90661
:1007300021D448F60F7311680B40694913600B68A8
:1007400088461A7A022A01D0042A02D1F9F7FEFE5D
:1007500059E2062A40F06B825A78052A08D11A78A5
:10076000520605D1D878FFF781FFBB681B6A98470E
:10077000E3689B685AE213689BB2ADF80230BDF89B
:1007800002301F0540F1CF8140F68F731168544F3E
:100790000B40544913600A68534B92B213445B00F8
:1007A0001A683B688846187A092817D092B2520016
:1007B00002F1804202F5C0421178197051785970E7
:1007C0009188C8B2090A41EA002159801189C8B24A
:1007D000090A41EA002199809289DA8001221A727D
:1007E000DA8893F80190002A40F0DC801A7812F041
:1007F0007F024AD1B9F1090F0FD1DA78012A00F24C
:10080000B8809978002940F0B4809988002940F098
:10081000B0809A72A3685B68A9E0B9F1050F10D1A6
:1008200093F90320002A01DA0823B9E09A78002A14
:10083000FAD19A88002AF7D19B7A002B00F0A28087
:10084000F2E7B9F1030F0ED1DA78012A40F0918076
:100850009A88002A40F08D805A7A42F020025A721B
:10086000A368DB6983E0B9F1010F40F08280DA7898
:10087000012A7ED19A88002A7BD15B7A980678D5A6
:1008800006F098FA00287DD073E0012A2ED1B9F144
:100890000B0F6ED1E26858799269D97890473B681E
:1008A0009A7A002A65D0002863D11A79002A60D18B
:1008B0009B78002B5DD1064B9B68DB689847084B03
:1008C0001B685A79DA72DA781A735BE0445C00408C
:1008D000C024002048340020BC350020005C0040CB
:1008E00064290020505C004004300020022A40D1DE
:1008F000B9F1010FC4D0B9F1030F3AD1587920F002
:10090000800E4FEA8E0202F1804101F5B84109687C
:1009100010F0800F14BF01F0300101F44051BEF11E
:10092000030F26D8B3F802E0BEF1000F21D101B3C6
:100930009B7AF3B102F1804202F5B84213680106D6
:100940004BBF23F4E04323F4804323F0400323F020
:1009500070034BBF9BB29BB283F0100383F48053B0
:1009600043F4004343F080031360A3689B699847F6
:1009700008E0E36848465B69984703280FD00028E1
:100980007FF452AFD8F80020A14B92B213445B0021
:100990001A6800221A603023E380062300E009234E
:1009A0003A6847E1B9F1060F12D11A78520677D1A9
:1009B0009B78012B02D1E368DB6966E0022B02D150
:1009C000E3681B6A61E0032B6AD1E3685B6A5CE061
:1009D000B9F1000F37D15988002961D15A6822F442
:1009E0007F42B2F5003F5BD11A7812F07F0204D14A
:1009F0009B88002B00F0D58152E0012A08D1E268E3
:100A000058799269904700284AD13B689B7A16E052
:100A1000022A45D15A7902F00F018B0003F180437D
:100A200003F5B8431B6812F0800F14BF03F03003C6
:100A300003F44053032933D812F0700F30D1002B48
:100A400040F0AF812CE0B9F1080F04D11B785B06B0
:100A500000F0A98124E0B9F10A0F21D11A7802F03F
:100A60007F02012A1CD19A7AD2B15988C1B95A6839
:100A700022F47F42B2F5803F12D1E2685879926940
:100A80009047002800F091810AE04BB13A684FF09E
:100A90000008A2F8128093614046984740460BE058
:100AA000E3683A681B6950789847032804D1594B8A
:100AB00009221B681A72BEE04FF6FF713A68138A6A
:100AC0008B4201D10923B5E0022800D00BB90823DD
:100AD000B0E092F9001000291FDAD1880191019845
:100AE000834202D9019B138210E08B420ED2E1684F
:100AF00091F82C00834201D2002105E093FBF0F134
:100B000000FB113313B90121434B1970E36893F8CB
:100B10002C309382F9F71AFD8DE0032313724FF402
:100B20004053A38087E0BDF802301BB2002BBFF614
:100B3000D6AD40F68F7311680B401360354A1768C5
:100B400090463B7A022B72D0042B70D0032B01D03D
:100B5000052B67D1BB693A8A8BB9398A00293BD00A
:100B60004FF44053A3802D4B1A68294B92B2134483
:100B70005B001A6800221A603023E3802CE0002A10
:100B8000EBD0B7F81490914528BF91461FFA89FA27
:100B9000504698473B8A4FF0000ECAEB03033B8256
:100BA0007B8A53447B821D4B1A681D4B92B21344BF
:100BB0005B001B6809F101029BB203F1005303F5CE
:100BC000405352105B009645C7D053F82E1020F8C2
:100BD0001E100EF1010EF6E7BB8A8B42D8F80030EA
:100BE00001D8032201E011B105221A720BE006229E
:100BF0001A720A4B1A68064B92B213445B001A68C9
:100C000019603023E380D8F800301B7A10E000BF71
:100C10000230002064290020BB350020505C0040D9
:100C200004300020072B02D1E368DB6898470823D3
:100C3000D8F800201372F9F767FC5E4B1A684BF680
:100C4000BF731340A288D704A28848BF83F480539F
:100C50009004E28848BF83F40053D106E28848BF7D
:100C600083F01003920648BF83F0200343F400434F
:100C700043F080034F4A9BB213602DE09A0002F1CB
:100C8000804202F5B842116889B2ADF80210BDF891
:100C9000021009B2002909DA40F68F711068013B91
:100CA00001401160444A52F823309847BDF80230A1
:100CB0001F067FF514AD48F60F72A1788B0003F183
:100CC000804303F5B843186802401A603A4B03EBBF
:100CD00081039B69984702E52288338813405905B0
:100CE00005D54FF6FF332B60344B5B68984722885D
:100CF00031880A40920444BF4DF6FF732B6023886D
:100D00002F4A0B40DB0452D54EF6FF732B600023B5
:100D10001374137C052B41D8DFE803F0030D14187E
:100D2000222D6369264D1BB903F0AAFC062300E0BF
:100D300005232B743BE003F0A3FC0423237401235D
:100D4000636134E002236374032328E0637C013B86
:100D5000DBB26374637C53BB194B04221A7426E024
:100D6000184A13689BB243F01003136005232374E1
:100D70000A2363741BE0637C114A013BDBB263749A
:100D8000637C03F0FF0093B94FF6EF730D490C68D5
:100D900023400B6006231374506108E0062323747C
:100DA00005E0094B72E6094B70E6094B6EE602B0AE
:100DB000BDE8F087005C0040C8BA01086403002069
:100DC000C0240020405C004019A10008CDA100080B
:100DD000A9A10008F8B5304B1B685B075BD52F4D08
:100DE0002F782C46012F07D0EB6898472B6998473E
:100DF00001232B70EA8842E06B699847AB689847FB
:100E0000AB6905F11C0026499847A96A6A6A097806
:100E1000501C8842296B08BF85F82C70EB692E6A3C
:100E200001F1010508BF0020032D02BF1B4D012762
:100E300085F8347004EB81018B6394F8341008BF9B
:100E40000025164F256369B1BD6BF96B3B6C8D4274
:100E5000DEBF0F4629463D46AB42A8BF2B468B421C
:100E6000B8BF0B4604EB8202536404EB8002526C61
:100E70006062B21A13442362A28800232370094BD4
:100E80001B780C2B07D80849342000FB0313642A75
:100E900038BF64221A61F8BDC0130020D824002096
:100EA000D01400209A030020640000202DE9F04FA8
:100EB000C14B87B01B685B0740F1E181BF4B93F8E2
:100EC0002C209846002A00F0DA81D3F80811D3F8D4
:100ED0000421531A46F2A7118B42019340F2CF81AD
:100EE000B74DC8F808212C886CB3D8F82820D8F85A
:100EF0000C111278013C501ED8F82020B2FBF0F201
:100F0000082091FBF0F6891B0A44C8F80C2192FBDB
:100F1000F0F005F067F9AB4905F06CFAAA4906F064
:100F20001BFC01464FF07E5005F0A6F8A74905F0DE
:100F3000ADF905F071FB0022C8F810012C80C8F84B
:100F40001421C8F81821D8F82840D8F820002278B1
:100F5000013AB0FBF2F005F041F99A4905F04AFA7E
:100F6000994906F0F9FB01464FF07E5005F084F8F0
:100F7000964905F08BF906F021FB6668944C814692
:100F8000206805F02FF9314605F080F90746D8F8BA
:100F90001001C0EB090005F025F9314681464FF0FC
:100FA0007E5005F069F80146484605F06FF90146A4
:100FB000384605F063F806F001FB864E20600746D0
:100FC000306805F00BF98449814605F05FF9D8F8DF
:100FD0001C418346039674B1784AD2F8280105F083
:100FE00001F90646204605F0FDF80146304605F0B9
:100FF00001FA064600E00026D8F82C11304605F02C
:1010000045F9494605F042F9D8F830314FF07C51A6
:10101000D3F80CA00293059005F038F9594605F075
:1010200035F9D8F8149159460490484605F02EF940
:10103000049A0146104605F021F8D8F8181105F079
:101040001DF8514605F022F98346384605F0CAF8E6
:10105000514604904FF07E5005F00EF8049A014678
:10106000104605F013F90146584605F007F8DDF87B
:1010700014C0C8F8180182466146484604F0FEFFD5
:10108000039BB5F800B000224C4C8146C8F814010F
:10109000C8F82021C8F82421C8F82821C8F81C2144
:1010A0001A60BBF1000F40F0EA80504605F0B4FA38
:1010B0004A4D2860D4F83401381A05F093F84849AD
:1010C00005F0E4F88246019805F088F8014650469C
:1010D00005F090F905F0A0FA40F2DC529042A8BF6A
:1010E0001046A2F6B8329042B8BF10460A21C4F8A2
:1010F0003471FAF739FF029B82469F6848463946A9
:1011000005F0C4F80190504605F06CF83946814668
:101110004FF07E5004F0B0FF0146484605F0B6F8A7
:10112000019B0146184604F0A9FFC4F8140106F01B
:1011300045FA05218146FAF717FF40F23E61294A38
:10114000D4F8387110602848028802F21F3292B237
:101150008A4205D8428802F21F3292B28A4205D9E9
:101160005B46C8F84431C8F8386188E094F84821F3
:10117000002A3FD11D4A286812680A21121AB2F5C6
:10118000FA7F1B48A8BF4FF4FA729042B8BF1046CE
:10119000FAF7EAFED4F83C2112795043802290FB02
:1011A000F2F0B0F5967FA2F5D672A8BF4FF4967014
:1011B0009042B8BF10461FE0C0130020D824002082
:1011C000B235002080E6C547B1DC423ED048874AB0
:1011D000CC14002094350020BD3786353014002013
:1011E00000247449341400202814002070140020B6
:1011F0000CFEFFFF234A1068D8F83C31C9EB000011
:101200009C7A2025444394FBF5F5197DD8F84021BC
:10121000B5F5967F00FB0122A8BF4FF496751A49D9
:10122000B2F5C81FA8BF4FF4C8128A42B8BF0A4619
:101230004FF40054C8F8402192FBF4F2134C987F0D
:10124000A542ACBF5419141904F0CCFF3946054629
:10125000304604F013FF0146284605F017F84FF01A
:101260006C5105F013F805F0D7F99628A8BF962021
:101270006FF095029042ACBF231AA31A71E707B032
:10128000BDE8F08F983500200000E7FFD4FEFFFF97
:10129000464B70B51B681B0740F18680444CD4F860
:1012A0000431D4F84C219A1A002A7DDB03F5C333AC
:1012B000A033C4F84C313F48D4F8543198473E4BE2
:1012C0003C481A780146F9F73BFC3C4B19781A4622
:1012D00011F0040F15D0D4F84C31C4F85831002364
:1012E000374800251844A0F8745132481D5A354833
:1012F0001D5206301D520233062BF1D121F004019C
:10130000117094F8683183B12A4B2D491A88B1F8CD
:101310007401121A1A80B1F876015A88B1F878115E
:10132000121A5A809A88521A9A80D4F85811204A70
:10133000002939D0D2F84C3102F5AE745B1A22493B
:1013400002F5B1708B421AD8204AD36883F00803A3
:10135000D3600023174A34F9136032F81320590080
:1013600015B2AE42C4BF174E26F81320465E0133B5
:10137000AE42BCBF164D4A53032BEBD170BD0023C8
:101380001449C2F8583134F9135030F9132001339D
:101390002A44022592FBF5F2032B21F8022FF2D109
:1013A000BDE87040FBF734B970BD00BFC01300202A
:1013B000D8240020F6130020BD350020481400205A
:1013C0006C2A0020342600207FC3C901000C014094
:1013D0003A260020DE2B00209C4B2DE9F0411B68B3
:1013E0001A0640F11B819A4E3368B3B9994C94F8B0
:1013F0006C31013B042B00F21181DFE813F0140083
:1014000014001400FE00DA00914B186801F0F1FAA4
:10141000FCF720FF08B1FCF785FB306801F0ECFA1F
:101420000028F1D1E2E7D4F88C218A4D177817B162
:10143000012F11D0F2E0012B00F2F08095F86D2120
:10144000854B0C2101FB02335A78844B306853F8EA
:10145000221001F0CBFA65E03068DFF8F48101F08A
:10146000C2FA002800F0DA8095F86C31022B45D0E2
:10147000032B53D0012B40F0D180794B1968D5F85C
:101480008431CB1AC72B40F2C980D5F88031042BA8
:1014900032D8714A0C20964600FB0323C5F884110C
:1014A000D8F800505E78AF6800236C49D8B251F884
:1014B0002320BA4204D00133082BF6D1002300E0E8
:1014C0000346B34205D0284651F8261001F08EFAA3
:1014D000A4E094F86D310C2101FB03E2566816F884
:1014E000011B19B1284601F08AFAF8E7D4F88031D7
:1014F0000133C4F8803191E002208DE095F86D2130
:10150000554B0C2101FB02335A78544BD8F800009C
:1015100053F8221001F06AFA03207DE0D5F88C31EF
:101520009B780BB9042077E095F888310BB985F8E2
:10153000887194F88831474D012B16D1D5F8803148
:10154000B22B0CD8444A3068134493F83C1001F095
:1015500056FAD5F880310133C5F8803105E0002313
:10156000C5F88031022385F8883194F88831394DE7
:10157000022B19D1D5F880210F2A12D8D5F88C3139
:1015800035495B78306803EB03130B44134493F83D
:10159000F01001F034FAD5F880310133C5F880310C
:1015A00002E0032385F8883194F88831022B35D97D
:1015B000B8E7D4F8743127490133C4F87431D4F84A
:1015C0008C31DB785BB191F86D3105220133DBB2F0
:1015D000B3FBF2F202EB82029B1A81F86D31204BD1
:1015E00000221B680120C4F878311E4B1A701E4A75
:1015F000137823F0020313700EE0194BD4F878210E
:101600001B689B1A40F6C412934207D9174A05205B
:10161000136823F020031360FDF70AF9134B1B68CE
:101620009B0611D50B4AD2F80431D2F89011591A01
:10163000002909DB0B490978042982BF03F512331D
:1016400003F5F873C2F89031BDE8F0812835002029
:10165000D0220020D824002004BB0108ECCC0108D3
:10166000582900204914002048140020C0130020ED
:101670000846F9F71BBC10B50D4C206801F022F8A4
:1016800020680022047A02FB02F3193B634303F64D
:10169000C4135343192193FBF1F3064921F8123087
:1016A0000132072AEFD1BDE81040034900F0C2BF64
:1016B00044140020D00A0020AC2B00200E4B1A78D6
:1016C000772A16D140F2E4725988914211D11A79E1
:1016D000BE2A0ED193F8E0270020EF2A0BD113F891
:1016E000012B5040054A9342F9D1B0FA80F04009ED
:1016F000704700207047704700F80108E4FF0108B8
:101700002DE9F04FE34C40F2E47285B02046002111
:1017100009F03CF9E04B04F53A721A60DF4B002700
:101720001F70DF4B04F2B2721A6077232370032319
:101730006371DC4B4FF42F72A36040F6C413A4F81E
:101740006431012384F8633184F8603184F87C319A
:1017500084F88431052384F8273240F2DC53A4F85E
:10176000963140F24C43A4F8983140F26C73A4F8DF
:101770009A3140F27533A4F89E3140F64303A4F841
:10178000A0312346A4F86C21202284F868216E221F
:1017900084F87A210A2284F87B212B2284F87D2187
:1017A000212284F87E21232284F87F214FF4C872FD
:1017B000A4F88021032FCCBF0122002207F10107EA
:1017C00083F8A22114BF1E220522122F83F8A32121
:1017D00003F10203EED140F27E42A4F8402140F230
:1017E0003A72A4F8422140F27E52A4F8482140F215
:1017F000EA5240F2DC50A4F84A2140F2B4521E23CF
:1018000084F893314FF4FA63A4F8C831A4F8CC31CA
:10181000A4F8D031A4F8D431C82301264FF47A7843
:101820004FF0320ADFF870B2A4F8E6314FF4C87313
:101830004FF0050C192184F8E46184F8E861A4F8FC
:10184000EA31A4F84601A4F84C21A4F8C681A4F812
:10185000CA81A4F8CE81A4F8D281A4F84481A4F866
:101860004EA184F8E16184F8E2C1CDF80CC084F89F
:10187000E311019184F8EE610290A4F8503184F8EC
:10188000F161A4F852A102F00BFEDBF800300199DF
:1018900000252573D9712121597453219F75D9765B
:1018A0002A2237210F275A705F71197299740D22FD
:1018B000222778215A75DDF80CC09F719972362263
:1018C0000E272D214FF028099A701F746422197574
:1018D00035273C211E70DA709F761A779E7783F841
:1018E0000B9083F80C9083F80DA083F817C083F851
:1018F00004A09D731D76DD735D7683F8099083F8EF
:1019000050106949694F196269499F63D962196327
:1019100059636849DF63596499644FF081474B21EB
:101920009F6283F84C1002984FF07F5E462100279B
:1019300083F8526083F85150A3F84E50C3F824E066
:101940001F6484F8B317142184F8B22784F8BA17F7
:10195000A4F8BC0784F8B4A784F8B55784F8B9573D
:1019600084F8B65784F8B75784F8B85783F85C10F2
:101970005149019219661521A3F85850A3F85A50FD
:10198000A3F8565083F8649083F8659083F8681044
:101990004A4983F87860D96649494A4819674A49EB
:1019A000596702F0ABFDDBF800304FF4487183F863
:1019B000146118465E46019AA3F816110A2183F8AD
:1019C000115183F8125183F8139183F8185184F858
:1019D000D81184F8D911A4F8DA8184F8DC51A4F87C
:1019E000DE210E2202FB05326FF0170E82F819E19C
:1019F0004FF0030E82F81AE16FF02F0E82F81BE110
:101A00004FF0070E82F81CE16FF0230E82F81DE103
:101A10004FF0050E82F81EE101354FF05A0E80F8A6
:101A200020E180F821E164224FF0FF0E082D80F8BC
:101A30001F2180F822E14FF0000100F10E00D0D10B
:101A4000C820A3F88A01142083F88C01A3F8902100
:101A50001E204FF4967283F88D01A3F89221012085
:101A6000282283F8891183F88E01A3F894210B466C
:101A7000E2181033C02B1761FAD11448002140221C
:101A800008F084FF0023124FE218D9590433086884
:101A9000382B1FE06C2A00200C140020082900209D
:101AA0004414002000010400CDCC8C3F0AD7233C15
:101AB000CDCCCC3E0000C0400000A0409A99193F18
:101AC000F6287C3FD3D901083D0A773F142D00202A
:101AD00048BC0108224DC2F8A802D4D105F50A700D
:101AE0000021802208F052FF07F13801702205F52D
:101AF0000A7008F042FFFBF7BBFF366800230124A1
:101B0000314605F590604FF4CC7285F8D83785F8EA
:101B1000D64785F8D74708F030FF05F5C360314652
:101B20004FF4CC7208F029FF0E4B1B681A68C5F8F9
:101B3000BE275A68C5F8C2279A68C5F8C6271A682A
:101B4000C5F8CA275A68C5F8CE279A680223C5F88F
:101B5000D22785F8D44485F86C3605B0BDE8F08FFF
:101B60006C2A00204414002038B5144B05461B682D
:101B700098421ADD124B93F8D84714B1012C09D0C2
:101B800017E0104B1B68186988B1A842CCBF012030
:101B9000022038BD7F280CDCFDF718F9C0F17F006A
:101BA000854208DDFDF7F0F805E0002038BD012092
:101BB00038BD022038BD204638BD00BF701000205F
:101BC0006C2A00206C100020074B93F8D837012BAB
:101BD00008D1064A064BD0681B68834234BF0020F8
:101BE00001207047002070476C2A00200C00002064
:101BF0006009002038B5094B93F8D85765B9084CEF
